:100000000C9424080C9455080C9455080C9455082D
:100010000C9455080C9455080C9455080C945508EC
:100020000C9455080C9455080C9455080C945508DC
:100030000C9455080C945B640C9455080C9455086A
:100040000C9455080C9455080C9455080C945508BC
:100050000C9455080C9455080C9455080C94024ABD
:100060000C9455080C9415700C94EC6F0C94550876
:100070000C9455080C9455080C9455080C9455088C
:100080000C9455080C9455080C9455080C9455087C
:100090000C94C36F0C949A6F0C9455080C94816562
:1000A0000C9455080C9455080C945508FEC7000094
:1000B000FCC70000FAC70000F8C70000F6C7000040
:1000C000F4C70000F2C70000F0C700000C94716F85
:1000D0000C94486FEAC700000C941F6F0C94F66EE6
:1000E000E4C700005E324032653265326532653207
:1000F0006532653265326532653265323F1E782180
:10010000DB23E323EB2315251B2515268D26A526AA
:10011000A9266532BC26C8263528102A942BC92C5E
:10012000392D022E7E2E18301F3165326532653230
:1001300065326532653265326532653265325A3113
:1001400065326532653265326532653293324947D0
:100150004C473B473F4745478347504754475A47DB
:100160005E47624768476C477047834776477A47E0
:100170007E47EA66B66750686C687F689268A568D3
:10018000C168D468E7680369166924693769084A51
:10019000D73B3BCE016E84BCBFFDC12F3D6C74319B
:1001A0009ABD56833DDA3D00C77F11BED9E4BB4CF2
:1001B0003E916BAAAABE000000803F07634236B79B
:1001C0009BD8A71A39685618AEBAAB558C1D3CB7E8
:1001D000CC5763BD6DEDFD753EF6177231BF000063
:1001E00000803F08000000BE922449123EABAAAA3C
:1001F0002ABECDCCCC4C3E00000080BEABAAAAAA41
:100200003E00000000BF000000803F000000000032
:10021000084178D3BB4387D1133D190E3CC3BD427F
:1002200082AD2B3E68EC8276BED98FE1A93E4C8030
:10023000EFFFBE01C4FF7F3F0000000000004E4101
:100240004E494E495459494E46CDCCCC3D0AD72350
:100250003C17B7D13877CC2B329595E6241FB14F98
:100260000A000020410000C84200401C4620BCBEDD
:100270004CCA1B0E5AAEC59D7400407A10F35A004A
:10028000A0724E18090010A5D4E80000E8764817BF
:100290000000E40B54020000CA9A3B000000E1F5A4
:1002A00005000080969800000040420F000000A06A
:1002B0008601000000102700000000E80300000095
:1002C000006400000000000A0000000000010000BF
:1002D0000000002C76D888DC674F0823DFC1DFAE32
:1002E00059E1B1B796E5E3E453C63AE651997696FB
:1002F000E8E6C28426EB898C9B62ED407C6FFCEFC4
:10030000BC9C9F40F2BAA56FA5F490055A2AF75CF1
:10031000936B6CF9676DC11BFCE0E40D47FEF520A3
:10032000E6B500D0ED902E0300943577050080846B
:100330001E080000204E0A000000C80C333333337F
:100340000F986E12831141EF8D2114893BE65516EB
:10035000CFFEE6DB18D1844B381BF77C1D901DA423
:10036000BBE424203284725E228100C9F124ECA116
:10037000E53D27696E7075742044535463616C6960
:1003800062726174653A0020766F6C746167653DD6
:1003900000235475726269646974792055707065C0
:1003A00072204C696D69743A200020766F6C74611C
:1003B00067653D0023547572626964697479204CE5
:1003C0006F776572204C696D69743A20002354750B
:1003D00072626964697479204C6F776572204C6928
:1003E0006D69742056696E663A200023434F3220AF
:1003F0004D415820766F6C7420280023434F3220E3
:100400007A65726F20766F6C74202800234F32203B
:1004100063616C6962726174696F6E3A2000235483
:100420007572626964697479204C6F776572204CCB
:10043000696D69742056313A200057694669204930
:10044000503A004D6F74696F6E004D6F74696F6E36
:10045000004E6F2053656E736F7221004E6F204403
:100460005320546865726D6F6D6574657221004428
:100470005320546865726D2E00434F3220436F6ED7
:10048000630053656E736F72206572726F72210024
:10049000234E6F2073656E736F722100434F3220BD
:1004A000436F6E63004D6561737572696E670023FB
:1004B0004E6F2054422073656E736F723F00234E5F
:1004C0006F2073656E736F722100536F756E6420B9
:1004D0004C6576656C004D6561737572696E672E4B
:1004E0002E00234E6F2073656E736F722100536F61
:1004F000756E64204C6576656C00234E6F207365C5
:100500006E736F7220666F722074656D7020262086
:1005100068756D696469747921004E6F2053656E4A
:10052000736F72210020666F722074656D702026D3
:100530002068756D696469747921002353656E7351
:100540006F72204572726F72200053656E736F7206
:10055000204572726F7221002357726F6E6720738D
:10056000656E736F7220666F722074656D702026E1
:100570002068756D6964697479210057726F6E67C0
:100580002053656E736F72210054656D702048753D
:100590006D6964697479004C6967687420496E7488
:1005A000656E7369747900466C616D65204952000F
:1005B000482D6669656C6400536561726368204408
:1005C0006972656374696F6E004E6F2073656E7338
:1005D0006F72210049522054656D706572617475A7
:1005E0007265004D6561737572696E672E2E00230A
:1005F0004E6F2070482073656E736F7221007048D3
:100600002076616C756500496E76616C6964206B5B
:1006100065792100237265706C6965733D006765BB
:100620007453656C665465737442697428293A2062
:10063000006973496E74657272757074456E61629B
:100640006C65642831293A2000676574496E7465C9
:1006500072727570744D617070696E672831293AD5
:100660002000676574496E74657272757074536F9B
:10067000757263652831293A2000676574496E7484
:10068000657272757074536F7572636528293A20AC
:10069000006765745261746528293A20332E31341D
:1006A0003135393F00616363656C2E69734C6F7738
:1006B000506F77657228293A2000616363656C2E5C
:1006C000697341736C65657028293A200061636322
:1006D000656C2E6973546170536F757263654F6EEC
:1006E0005A28293A2000616363656C2E697354614E
:1006F00070536F757263654F6E5928293A200061F7
:100700006363656C2E6973546170536F75726365B2
:100710004F6E5828293A2000616363656C2E697317
:100720004163746976697479536F757263654F6E4E
:100730005A28293A2000616363656C2E697341630E
:10074000746976697479536F757263654F6E592851
:10075000293A200069734163746976697479536F2B
:10076000757263654F6E5828293A20006973546189
:1007700070446574656374696F6E4F6E5A28293BC7
:100780002066616C73653F20006973546170446535
:1007900074656374696F6E4F6E5A28293B207472BA
:1007A00075653F20006973546170446574656374B6
:1007B000696F6E4F6E5928293B2066616C73653FE7
:1007C00020006973546170446574656374696F6E69
:1007D0004F6E5928293B20747275653F200069735C
:1007E000546170446574656374696F6E4F6E582808
:1007F000293B2066616C73653F200069735461700A
:10080000446574656374696F6E4F6E5828293B2088
:10081000747275653F2000676574537570707265FA
:10082000737342697428293B2066616C73653F20AD
:1008300000676574537570707265737342697428CC
:10084000293B20747275653F2000697341637469A8
:1008500076697479416328293A20006973496E6189
:10086000637469766974795A456E61626C6564284F
:10087000293A20006973496E6163746976697479F5
:1008800059456E61626C656428293A200069734994
:100890006E616374697669747958456E61626C65DE
:1008A0006428293A20006973416374697669747910
:1008B0005A456E61626C656428293A20006973416B
:1008C0006374697669747959456E61626C656428F0
:1008D000293A2000697341637469766974795845CF
:1008E0006E61626C656428293A20006765744672FF
:1008F000656546616C6C4475726174696F6E282918
:100900003A20006765744672656546616C6C546890
:10091000726573686F6C6428293A200067657454A7
:10092000696D65496E616374697669747928293ADD
:100930002000676574496E616374697669747954DF
:1009400068726573686F6C6428292000676574415C
:10095000637469766974795468726573686F6C64DE
:1009600028292000676574446F75626C6554617056
:1009700057696E646F7728292000676574446F7526
:10098000626C655461704C6174656E637928293AB4
:1009900020006765745461704475726174696F6E8C
:1009A00028293A2000676574417869734F66667339
:1009B00065742826782C2026792C20267A293A203E
:1009C000006765745461705468726573686F6C6415
:1009D00028293A200058595A2047733A200058597C
:1009E0005A20434F554E54533A2000736574206784
:1009F00061696E735B5D3A006761696E735F6F7208
:100A000069675B5D3A0043616C6962726174696F2A
:100A10006E2050726573737572653D005365612079
:100A20006C6576656C20502863616C63293D0023FA
:100A30004572726F723A7072657373757265204297
:100A40004D503038352C20636865636B20776972B0
:100A5000696E67210049522054656D702073656E80
:100A6000736F7220666F756E6400504D322E3520A4
:100A700073656E736F72206C696B656C7920666F3D
:100A8000756E6400576946692049503A00456455BF
:100A9000484B205345534C6F676765720053656E32
:100AA000736F7220736C6F7420616E642074797040
:100AB000653A0057656C636F6D6520746F204564FF
:100AC00055484B00005EBCE2613FDD83C29C7E2046
:100AD000A3FD1F41009D23BE46DB65F88C11AF329C
:100AE000CA57E97400002100240027002A002D00C5
:100AF0003000330001010000040107010A01000079
:100B00002200250028002B002E00310034000201B5
:100B10000000050108010B01000020002300260051
:100B200029002C002F003200000100000301060103
:100B30000901050505050705080808080202020263
:100B40000A0A080804040404010101010101010169
:100B50000303030303030303040707070C0C0C0C34
:100B60000C0C0C0C0202020206060606060606061D
:100B70000B0B0B0B0B0B0B0B0102102020080810AA
:100B800020401020408002010201080402010102FD
:100B900004081020408080402010080402018004D6
:100BA0000201804020100804020108040201010231
:100BB000040810204080010204081020408000003A
:100BC0000A0B02090C0D0E080703040100000000C7
:100BD0000000000000000000000000000000000015
:100BE00000000000000000000000121110000000D2
:100BF00000000000000000000000000000000000F5
:100C0000000000004F3220436F6E6300234E6F20C0
:100C100073656E736F7220666F7220504D21004EA7
:100C20006F2073656E736F722100206E672F4C000A
:100C3000504D313A322E353A3130004D6561737581
:100C400072696E672E2E00555620496E742E00551F
:100C50005620496E74656E7369747900232D2D2DAD
:100C60002D2D2D2D2D2D2D2D2D2D2D2D2D2D2D2DB4
:100C70002D2D2D2D2D2D2D2D2D2D2D2D2D2D2D2DA4
:100C80002D00235265736F6C7574696F6E3A202066
:100C90002000234D696E2056616C75653A20202036
:100CA0002000234D61782056616C75653A20202024
:100CB000200023556E697175652049443A20202033
:100CC000200023447269766572205665723A2020AE
:100CD00020002353656E736F723A2020202020205D
:100CE0002000232D2D2D2D204D61676E65746963C5
:100CF0002053656E736F72202D2D2D2D2D2D2D2DD2
:100D00002D2D2D2D2D2D2D2D2D2D2D2D00482D66EC
:100D100069656C643A2028002020202020202020B3
:100D200020202020202020200020202020202020E3
:100D300020202020202020202000202020202020D3
:100D400020202020202020202020002020202020C3
:100D500020202020202020202020200020202020B3
:100D600020202020202020202020200020202020A3
:100D7000202020202020202020202000233A5368FB
:100D80006F772F48696465204C4344002A3A5468C1
:100D900069732048656C700044433A436C65617226
:100DA000204C43440044423A5265736574204C6FB2
:100DB000676765720044363A44532054656D70008D
:100DC00044353A555620496E74656E7369747900DE
:100DD00044343A4F3220636F6E632E0044333A43FB
:100DE0004F3220636F6E632E0044323A504D2831EB
:100DF0003A322E353A3130290044323A504D2831BA
:100E00003A322E353A3130292A0044313A5475723B
:100E10006269646974790044303A566F6C74616732
:100E20006500393A6F7220334420616363656C2E2C
:100E300000393A496E636C2E20616E672E00383A95
:100E400070482076616C756500373A4952205465C8
:100E50006D7000373A49522054656D702A00363A59
:100E60004D61676E65746963206669656C64003501
:100E70003A476173204C6576656C00343A495220DC
:100E8000466C616D6500333A4C6967687420496E41
:100E9000742E00323A616E64204865696768740098
:100EA000323A54656D7020507265737375726500C7
:100EB000313A54656D702048756D696469747900C4
:100EC000303A536F756E64204C6576656C00303A2D
:100ED000536F756E64204C6576656C2A0054696D9D
:100EE00065206C617073653A005769466920495006
:100EF0003A0046696E64696E672057694669204901
:100F0000500023616E6F7468657220495220696ECB
:100F10007075743D00236B65793D004F66662061F6
:100F200069722D636F6E6421004974277320746F9A
:100F30006F20636F6F6C210054656D7020697320A2
:100F400066696E6521004973206169722D636F6E59
:100F500064206F6E3F004974277320717569746552
:100F600020686F7421004974277320766572792098
:100F7000686F742120004F6666206169722D636F6F
:100F80006E6421004974277320746F6F20636F6F44
:100F90006C210054656D702069732066696E65214F
:100FA000004973206169722D636F6E64206F6E3F1C
:100FB000004974277320717569746520686F742106
:100FC0000049742773207665727920686F74210058
:100FD00054656D702048756D696469747900416E5F
:100FE000676C65732F003E6128782C792C7A292F45
:100FF000673A004572726F72206E756D626572207D
:10100000666F722074686520617272617920746FF6
:10101000206176726167696E67212F6E004E6F20C6
:1010200073656E736F723F0049522054656D706531
:10103000726174757265004D6561737572696E6772
:101040002E2E0000D18F0F9211241FBECFEFD1E2C0
:10105000DEBFCDBF00E00CBF1CE0A0E0B2E0E6E6E2
:10106000FDE301E00BBF02C007900D92A030B10775
:10107000D9F722E1A0E0BCE001C01D92A03CB2077C
:10108000E1F718E0C3E2D8E000E006C021970109CB
:10109000802FFE010E94ED9BC232D10780E008073D
:1010A000A9F70E94F1860C94A29E0C9400002F9246
:1010B0003F924F925F926F927F928F929F92AF92E8
:1010C000BF92CF92DF92EF92FF920F931F93CF9335
:1010D000DF93CDB7DEB7EA970FB6F894DEBF0FBE49
:1010E000CDBF10913812112321F0109238120C94B8
:1010F000A11D8091461190914711019709F050C0B0
:1011000060E070E082E491E10E94566B082E000CD2
:10111000990B0E94419E892B09F442C061E775E05A
:10112000CE0183960E94976DBE016D5D7F4F82E474
:1011300091E10E94676B811127C06DE779E0CE01D4
:1011400045960E94976DBE016B5E7F4F82E491E1F0
:101150000E94676B811114C066ED79E0CE010196A3
:101160000E94976DBE016F5F7F4F82E491E10E9404
:10117000676B11E0811110E0CE0101960E94CD6CE9
:10118000CE0145960E94CD6CCE0183960E94CD6C17
:10119000112331F062E471E186E391E10E94B86CC1
:1011A0008091461190914711049708F042C068EB76
:1011B00077E0CE0101960E94976DBE016F5F7F4F71
:1011C00082E491E10E94676B182FCE0101960E9484
:1011D000CD6C112371F161E070E082E491E10E9435
:1011E000566B80330CF484516AE270E0681B71091D
:1011F00087FD73954AE0CE0101960E945C6DBE01A9
:101200006F5F7F4F82E491E10E94826BCE01019675
:101210000E94CD6C62E471E186E391E10E94B86CBA
:1012200082E491E10E94EC6ACB010E94BA1D0C9409
:10123000A11D63E775E0CE0145960E94976DBE0142
:101240006B5E7F4F82E491E10E94676B811116C053
:1012500067E775E0CE0101960E94976DBE016F5F52
:101260007F4F82E491E10E94676B11E0811101C020
:1012700010E0CE0101960E94CD6C01C011E0CE01BC
:1012800045960E94CD6C112309F456C36BE775E0B7
:10129000CE0101960E94976DCE0101960E949E7C20
:1012A000CE0101960E94CD6C67E875E0CE010196F3
:1012B0000E94976D6FE172E1CE0101960E94266C4B
:1012C000BC01CE0145960E948F6DCE0145960E94CD
:1012D0009E7CCE0145960E94CD6CCE0101960E9467
:1012E000CD6C609170047091710480917204909142
:1012F00073040E940F9720E030E048EC52E40E9413
:101300005F99AB01BC0122E0CE0145960E94016DC0
:101310006DE975E0CE0101960E94976DBE016B5E8E
:101320007F4FCE0101960E94266C6EEF76E00E9400
:101330000F6CBC01CE0183960E948F6DCE01839607
:101340000E949E7CCE0183960E94CD6CCE010196B8
:101350000E94CD6CCE0145960E94CD6C40916C04EC
:1013600050916D0460916E0470916F0424E0CE0181
:1013700045960E94016D62EB75E0CE0101960E94D8
:10138000976DBE016B5E7F4FCE0101960E94266C69
:10139000BC01CE0183960E948F6DCE0183960E9480
:1013A0009E7CCE0183960E94CD6CCE0101960E9458
:1013B000CD6CCE0145960E94CD6C40916004509159
:1013C0006104609162047091630422E0CE018F9603
:1013D0000E94016D409158045091590460915A0443
:1013E00070915B0423E0CE0189960E94016D4091CB
:1013F000640450916504609166047091670422E072
:10140000CE0183960E94016D40915C0450915D0471
:1014100060915E0470915F0423E0CE0145960E94C6
:10142000016D6FEC75E0CE0101960E94976DBE01D3
:101430006B5E7F4FCE0101960E94266C64EE75E0D4
:101440000E940F6CBE016D5D7F4F0E94266C67EE9F
:1014500075E00E940F6CBE01675D7F4F0E94266C95
:1014600064EE75E00E940F6CBE01615D7F4F0E94CB
:10147000266C6DEE75E00E940F6CBC01CE01C59626
:101480000E948F6DCE01C5960E949E7CCE01C596AE
:101490000E94CD6CCE0101960E94CD6CCE01459686
:1014A0000E94CD6CCE0183960E94CD6CCE018996B0
:1014B0000E94CD6CCE018F960E94CD6C4091C404E9
:1014C0005091C5046091C6047091C70423E0CE0119
:1014D00083960E94016D20915404309155044091EF
:1014E00056045091570460E070E080E291E40E945D
:1014F0000D9BAB01BC0121E0CE0145960E94D26C50
:1015000062EF75E0CE0101960E94976DBE016B5EA1
:101510007F4FCE0101960E94266C65E076E00E9426
:101520000F6CBE016D5D7F4F0E94266C6BE076E014
:101530000E940F6CBC01CE0189960E948F6DCE0176
:1015400089960E949E7CCE0189960E94CD6CCE0128
:1015500001960E94CD6CCE0145960E94CD6CCE01C5
:1015600083960E94CD6C4091C0045091C10460915B
:10157000C2047091C30423E0CE0183960E94016DE2
:1015800020915004309151044091520450915304E1
:1015900060E070E080E291E40E940D9BAB01BC0131
:1015A00021E0CE0145960E94D26C6EE076E0CE013D
:1015B00001960E94976DBE016B5E7F4FCE01019632
:1015C0000E94266C65E076E00E940F6CBE016D5DA6
:1015D0007F4F0E94266C6BE076E00E940F6CBC018E
:1015E000CE0189960E948F6DCE0189960E949E7CC5
:1015F000CE0189960E94CD6CCE0101960E94CD6CE1
:10160000CE0145960E94CD6CCE0183960E94CD6C92
:1016100040914C0450914D0460914E0470914F04E0
:1016200022E0CE0145960E94016D61E276E0CE0196
:1016300001960E94976DBE016B5E7F4FCE010196B1
:101640000E94266C67E376E00E940F6CBC01CE011D
:1016500083960E948F6DCE0183960E949E7CCE0160
:1016600083960E94CD6CCE0101960E94CD6CCE0176
:1016700045960E94CD6C4091480450914904609178
:101680004A0470914B0422E0CE0145960E94016D00
:101690006EE376E0CE0101960E94976DBE016B5E0F
:1016A0007F4FCE0101960E94266C6BE076E00E948F
:1016B0000F6CBC01CE0183960E948F6DCE01839684
:1016C0000E949E7CCE0183960E94CD6CCE01019635
:1016D0000E94CD6CCE0145960E94CD6C16E3C12EC2
:1016E00014E0D12E01E010E087E1E82E809134046F
:1016F00090913504801791070CF44FC0F601A1902A
:10170000B1906F014AE0B501CE0183960E945C6DF5
:101710004AE0B801CE0145960E945C6D61E576E035
:10172000CE0101960E94976DBE016B5E7F4FCE0188
:1017300001960E94266C6EE176E00E940F6CBE015D
:101740006D5D7F4F0E94266C69E576E00E940F6C0C
:10175000EA9CB001EB9C700D1124645E7D4F0E94E9
:101760000F6CBC01CE0189960E948F6DCE018996C7
:101770000E949E7CCE0189960E94CD6CCE0101967E
:101780000E94CD6CCE0145960E94CD6CCE01839611
:101790000E94CD6C0F5F1F4FA9CF80911F0D9091BC
:1017A000200D892B71F46FE576E0CE0101960E9441
:1017B000976DCE0101960E949E7CCE0101960E94FB
:1017C000CD6C80911F0D9091200D019771F46EE604
:1017D00076E0CE0101960E94976DCE0101960E949F
:1017E0009E7CCE0101960E94CD6C80911F0D909140
:1017F000200D029771F468E776E0CE0101960E9411
:10180000976DCE0101960E949E7CCE0101960E94AA
:10181000CD6C60914604709147044AE0CE01459634
:101820000E945C6D6AE876E0CE0101960E94976D99
:10183000BE016B5E7F4FCE0101960E94266CBC01FB
:10184000CE0183960E948F6DCE0183960E949E7C6E
:10185000CE0183960E94CD6CCE0101960E94CD6C84
:10186000CE0145960E94CD6C40911802509119020C
:1018700060911A0270911B0222E0CE0145960E94EF
:10188000016D67EA76E0CE0101960E94976DBE0178
:101890006B5E7F4FCE0101960E94266C6CEE78E065
:1018A0000E940F6CBC01CE0183960E948F6DCE0109
:1018B00083960E949E7CCE0183960E94CD6CCE01C1
:1018C00001960E94CD6CCE0145960E94CD6C409150
:1018D000140250911502609116027091170222E0D5
:1018E000CE0145960E94016D67EB76E0CE01019630
:1018F0000E94976DBE016B5E7F4FCE0101960E94E4
:10190000266C6CEE78E00E940F6CBC01CE018396D1
:101910000E948F6DCE0183960E949E7CCE0183969D
:101920000E94CD6CCE0101960E94CD6CCE014596F1
:101930000E94CD6C10921302809146119091471134
:101940008330910508F092C08130910541F460E048
:1019500070E082E491E10E94566BF82E62C002971B
:1019600009F05FC068EB77E0CE0101960E94976DA9
:10197000BE016F5F7F4F82E491E10E94676B182F79
:10198000CE0101960E94CD6C112309F44AC061E09A
:1019900070E082E491E10E94566B1A8219821C82E7
:1019A0001B821E821D828D8B1E8ABE016B5E7F4F45
:1019B000CE0101960E94A36CBE016F5F7F4F86E34C
:1019C00091E10E94826BCE0101960E94CD6C60E095
:1019D00070E082E491E10E94566BF82E80913B0CFE
:1019E0008823F9F067EC76E0CE0101960E94976DAE
:1019F00062E471E1CE0101960E94266C6AEC79E006
:101A00000E940F6CBC0182EA9FE00E94F66DCE013D
:101A100001960E94CD6C66E371E182EA9FE00E942C
:101A2000E56E8F2D0F2C000C990B0E94419E892B87
:101A3000B1F00E94C44E0E94CC566AEC79E0CE010F
:101A400001960E94976D4AE050E060E070E0CE01A0
:101A500001960E949757CE0101960E94CD6C8F2D62
:101A60000E9464850E94F6490C948A1D21E030E0B2
:101A700040E050E062E471E1CE0101960E94AB6D5E
:101A8000BE016F5F7F4F84E291E10E94826BCE01C5
:101A900001960E94CD6C6AEF76E0CE0145960E94D9
:101AA000976DBE016B5E7F4F82E491E10E94676B90
:101AB000811116C062ED79E0CE0101960E94976D0A
:101AC000BE016F5F7F4F82E491E10E94676B11E07E
:101AD000811101C010E0CE0101960E94CD6C01C0C1
:101AE00011E0CE0145960E94CD6C112309F4BCC0D3
:101AF0008091461190914711409710F00C94A11DD0
:101B000042E050E062E471E1CE0101960E948C5EF9
:101B1000BE016F5F7F4F84E291E10E94826BCE0134
:101B200001960E94CD6C64E271E1CE0101960E94A3
:101B30008F6DCE0101960E94EE58CE0101960E9453
:101B4000CD6C0E94928420E030E048EC52E40E9488
:101B50006E970E94F899AB01BC01409370045093BA
:101B6000710460937204709373042AE0CE010196AD
:101B70000E94306DCE0101960E94EE58CE01019672
:101B80000E94CD6C60917004709171048091720418
:101B9000909173048B019C0100591F45214031092C
:101BA00001341C492105310588F06DEC76E0CE0149
:101BB00001960E94976D64E271E1CE0101960E9448
:101BC000266C60EE76E00E940F6CB6C119821A8214
:101BD0001B821C821D821E821F8218860E940F9704
:101BE00020E030E048EC52E40E945F998E010F5FE4
:101BF0001F4F22E047E00E943B92BC018AE291E144
:101C00000E94A36C60EF76E0CE0145960E94976D2E
:101C10006AE271E1CE0145960E94266C6DEF76E096
:101C20000E940F6CBC018AE291E10E94B86CCE0167
:101C300045960E94CD6C1092650C1092640C8091B8
:101C4000700490917104A0917204B0917304809318
:101C5000A90C9093AA0CA093AB0CB093AC0C80E0B1
:101C600090E00E94376271C162E077E0CE01459654
:101C70000E94976DBE016B5E7F4F82E491E10E94EE
:101C8000676B811116C068E077E0CE0101960E9473
:101C9000976DBE016F5F7F4F82E491E10E94676B99
:101CA00011E0811101C010E0CE0101960E94CD6CBF
:101CB00001C011E0CE0145960E94CD6C112309F4BC
:101CC00065C026E030E045E050E062E471E1CE011D
:101CD00001960E94AB6DBE016F5F7F4F84E291E180
:101CE0000E94826BCE0101960E94CD6C84E291E14C
:101CF0000E94EC6A6B017C0165E376E0CE010196FF
:101D00000E94976DCE0101960E949E84AC014F5FA8
:101D10005F4F62E471E1CE0145960E948C5EBE0188
:101D20006B5E7F4F84E291E10E94826BCE0145960B
:101D30000E94CD6CCE0101960E94CD6C84E291E1AF
:101D40000E94EC6ADB01E4E3F4E041E050E0209122
:101D5000340430913504241735075CF02281338137
:101D60002A173B0711F4138212824F5F5F4F32969E
:101D7000EECF9601220F331FF901EC5CFB4F71830C
:101D8000608382E090E00E9417501CC56EE077E00F
:101D9000CE0145960E94976DBE016B5E7F4F82E437
:101DA00091E10E94676B811116C064E177E0CE017A
:101DB00001960E94976DBE016F5F7F4F82E491E1B3
:101DC0000E94676B11E0811101C010E0CE01019605
:101DD0000E94CD6C01C011E0CE0145960E94CD6CF1
:101DE000112339F1E4E3F4E081E090E02091340440
:101DF000309135042817390774F0863091051CF4AA
:101E00009383828305C09C012E5F3F4F33832283DF
:101E100001963296EBCF82E090E00E94175010922C
:101E2000650C1092640C80E090E00E9437620C9484
:101E3000761D6AE177E0CE0145960E94976DBE015E
:101E40006B5E7F4F82E491E10E94676B811116C047
:101E500061E277E0CE0101960E94976DBE016F5F4F
:101E60007F4F82E491E10E94676B11E0811101C014
:101E700010E0CE0101960E94CD6C01C011E0CE01B0
:101E800045960E94CD6C1123F9F08091A70C90919A
:101E9000A80C892BA1F481E090E09093A80C80938A
:101EA000A70C8EED93E09093650C8093640C0E94D8
:101EB000686268EC70E080E090E00E94BE49E0E07B
:101EC000F0E019950C94781D68E277E0CE01459614
:101ED0000E94976DBE016B5E7F4F82E491E10E948C
:101EE000676B811116C060E377E0CE0101960E9416
:101EF000976DBE016F5F7F4F82E491E10E94676B37
:101F000011E0811101C010E0CE0101960E94CD6C5C
:101F100001C011E0CE0145960E94CD6C112381F1E4
:101F200068E377E0CE0101960E94976D69E172E166
:101F3000CE0101960E94266CBC018AE291E10E94CA
:101F4000B86CCE0101960E94CD6C6CE97AE0CE01AE
:101F500001960E94976D6AE271E1CE0101960E949E
:101F6000266CBC01CE0145960E948F6DCE01459630
:101F70000E949E7CCE0145960E94CD6C0C94721DF1
:101F800062E477E0CE0145960E94976DBE016B5EDC
:101F90007F4F82E491E10E94676B811116C069E472
:101FA00077E0CE0101960E94976DBE016F5F7F4F73
:101FB00082E491E10E94676B11E0811101C010E0A1
:101FC000CE0101960E94CD6C01C011E0CE01459674
:101FD0000E94CD6C112349F06FE875E0CE010196A7
:101FE0000E94976D6FE172E1A3CF60E577E0CE01CB
:101FF00045960E94976DBE016B5E7F4F82E491E132
:102000000E94676B811116C065E577E0CE010196ED
:102010000E94976DBE016F5F7F4F82E491E10E9445
:10202000676B11E0811101C010E0CE0101960E94A2
:10203000CD6C01C011E0CE0145960E94CD6C1123FC
:10204000C1F165E376E0CE0101960E94976DCE0165
:1020500001960E949E84AC014F5F5F4F62E471E184
:10206000CE0145960E948C5EBE016B5E7F4F84E27E
:1020700091E10E94826BCE0145960E94CD6CCE010B
:1020800001960E94CD6C84E291E10E94EC6A611598
:10209000710521F481E08093120207C0613071055F
:1020A00011F00C94761D109212020E94D34E0C94E3
:1020B000761D6AE577E0CE0145960E94976DBE01D8
:1020C0006B5E7F4F82E491E10E94676B811116C0C5
:1020D0006EE577E0CE0101960E94976DBE016F5FBD
:1020E0007F4F82E491E10E94676B11E0811101C092
:1020F00010E0CE0101960E94CD6C01C011E0CE012E
:1021000045960E94CD6C112309F424C143E050E0B0
:1021100062E471E1CE0101960E948C5EBE016F5FA8
:102120007F4F84E291E10E94826BCE0101960E9472
:10213000CD6C64E271E1CE0101960E948F6DCE01FB
:1021400001960E94EE58CE0101960E94CD6C10922D
:10215000650C1092640C64E271E185E292E10E94E8
:10216000B86C64E271E18FE192E10E94B86C85EC99
:102170009CE0009739F048E050E0BC0185E292E134
:102180000E940B4783E29DE0009739F04CE050E05D
:10219000BC018FE192E10E940B478091640C909109
:1021A000650C0E94376262E677E0CE0101960E94DC
:1021B000976D6FE172E1CE0101960E94266CBC0121
:1021C000CE0183960E948F6DCE0101960E94CD6C48
:1021D00080911F0D9091200D892B39F4BE016D5D0A
:1021E0007F4F8BEC9DE00E94F66D80911F0D9091CA
:1021F000200D029709F09BC06FE172E1CE01899634
:102200000E948F6D6AE677E0CE0101960E94976D7D
:10221000CE0101960E944D8FCE0101960E94CD6C99
:1022200064EF71E080E090E00E94BE496DE677E0E7
:10223000CE0101960E94976DCE0101960E944D8FAE
:10224000CE0101960E94CD6C64EF71E080E090E0D9
:102250000E94BE4966E777E0CE0101960E94976D25
:10226000CE0101960E944D8FCE0101960E94CD6C49
:1022700064EF71E080E090E00E94BE496FE777E094
:10228000CE0101960E94976DCE0101960E944D8F5E
:10229000CE0101960E94CD6C64EF71E080E090E089
:1022A0000E94BE496DE877E0CE0101960E94976DCD
:1022B000CE0101960E944D8FCE0101960E94CD6CF9
:1022C00064EF71E080E090E00E94BE4962E677E052
:1022D000CE0101960E94976DBE01675D7F4FCE01D2
:1022E00001960E94266CBC01CE0145960E948F6D1E
:1022F000CE0101960E94CD6CCE0145960E94F76AF0
:10230000BE016B5E7F4FCE0101960E948F6DCE01A4
:1023100001960E944D8FCE0101960E94CD6CCE0198
:1023200045960E94CD6CCE0189960E94CD6C65ECDD
:102330007CE0CE0101960E94976DCE0101960E942D
:10234000EE58CE0101960E94CD6C10921302CE0180
:1023500083960EC46BE977E0CE0145960E94976D97
:10236000BE016B5E7F4F82E491E10E94676B811139
:1023700016C060EA77E0CE0101960E94976DBE011B
:102380006F5F7F4F82E491E10E94676B11E08111E2
:1023900001C010E0CE0101960E94CD6C01C011E099
:1023A000CE0145960E94CD6C112309F468C044E02B
:1023B00050E062E471E1CE0101960E948C5EBE01A4
:1023C0006F5F7F4F84E291E10E94826BCE010196A4
:1023D0000E94CD6C65EA77E0CE0145960E94976D2C
:1023E00064E271E1CE0145960E94266CBC01CE01EB
:1023F00001960E948F6DCE0145960E94CD6C809112
:102400001F0D9091200D892B39F4BE016F5F7F4F16
:102410008BEC9DE00E94F66D68EB7BE080E090E045
:102420000E94BE4980911F0D9091200D029779F472
:10243000BE016F5F7F4FCE0145960E948F6DCE012A
:1024400045960E944D8FCE0145960E94CD6C68EB5B
:102450007BE080E090E00E94BE49BE016F5F7F4F4D
:10246000CE0145960E948F6DCE0145960E94EE5892
:10247000CE0145960E94CD6C1092130277C36CEA90
:1024800077E0CE0145960E94976DBE016B5E7F4F4F
:1024900082E491E10E94676B811116C060EB77E0E6
:1024A000CE0101960E94976DBE016F5F7F4F82E45F
:1024B00091E10E94676B11E0811101C010E0CE0133
:1024C00001960E94CD6C01C011E0CE0145960E949C
:1024D000CD6C112309F456C062E471E184E291E10C
:1024E0000E94B86C81E08093130262E471E1CE0136
:1024F00001960E948F6DCE0101960E94EE58CE018A
:1025000001960E94CD6C80911F0D9091200D029735
:10251000A1F064E271E18BEC9DE00E94F66D68EB46
:102520007BE080E090E00E94BE490E94B57C60EDB7
:1025300077E080E090E00E94BE4980911F0D90916D
:10254000200D029771F464E271E1CE0101960E94C0
:102550008F6DCE0101960E944D8FCE0101960E9493
:10256000CD6C8091461190914711892B11F40C94F8
:10257000761D6CE97AE0CE0101960E94976D62E4C7
:1025800071E1EBCC64EB77E0CE0145960E94976D4C
:10259000BE016B5E7F4F82E491E10E94676B811107
:1025A00016C06AEB77E0CE0101960E94976DBE01DE
:1025B0006F5F7F4F82E491E10E94676B11E08111B0
:1025C00001C010E0CE0101960E94CD6C01C011E067
:1025D000CE0145960E94CD6C112309F45CC0809118
:1025E0001F0D9091200D019711F00C94761DCE01D6
:1025F00001960E946C768D819E81009711F40C9457
:10260000721DE981FA812081222311F40C94721D3C
:10261000079710F40C94721D6AE374E0CE0145969E
:102620000E94876D48EC50E06FEF7FEFCE0145963A
:102630000E949757CE0145960E94CD6CBE016F5FF8
:102640007F4FCE0145960E948F6D40ED57E06FEFB2
:102650007FEFCE0145960E941C57CE0145960E9401
:10266000CD6C60EC77E0CE0145960E94976D62E4F8
:1026700071E1CE0145960E94266CBC01CE01839685
:102680000E948F6DCE0183960E949E7CCE01839620
:102690000E94CD6C6FCC6EEC77E0CE0145960E9427
:1026A000976DBE016B5E7F4F82E491E10E94676B84
:1026B000811116C063ED77E0CE0101960E94976DFF
:1026C000BE016F5F7F4F82E491E10E94676B11E072
:1026D000811101C010E0CE0101960E94CD6C01C0B5
:1026E00011E0CE0145960E94CD6C1123F1F025E05A
:1026F00030E044E050E062E471E1CE0101960E94D6
:10270000AB6DBE016F5F7F4F84E291E10E94826BEF
:10271000CE0101960E94CD6C84E291E10E94EC6AA8
:102720007093200D60931F0D4DC068ED77E0CE01D2
:1027300045960E94976DBE016B5E7F4F82E491E1EA
:102740000E94676B811116C06DED77E0CE01019696
:102750000E94976DBE016F5F7F4F82E491E10E94FE
:10276000676B11E0811101C010E0CE0101960E945B
:10277000CD6C01C011E0CE0145960E94CD6C1123B5
:1027800081F126E030E044E050E062E471E1CE0106
:1027900001960E94AB6DBE016F5F7F4F84E291E1B5
:1027A0000E94826BCE0101960E94CD6C84E291E181
:1027B0000E94EC6A7093220D6093210D7093470480
:1027C0006093460462E471E1CE0101960E948F6D30
:1027D000CE0101960E94EE58CE0101960E94CD6C6A
:1027E0001ECB62EE77E0CE0145960E94976DBE014A
:1027F0006B5E7F4F82E491E10E94676B811116C08E
:1028000069EE77E0CE0101960E94976DBE016F5F81
:102810007F4F82E491E10E94676B11E0811101C05A
:1028200010E0CE0101960E94CD6C01C011E0CE01F6
:1028300045960E94CD6C112369F127E030E046E017
:1028400050E062E471E1CE0101960E94AB6DBE01E1
:102850006F5F7F4F84E291E10E94826BCE0101960F
:102860000E94CD6C84E291E10E94EC6A672B19F41E
:1028700010923B0C03C081E080933B0C62E471E159
:10288000CE0101960E948F6DCE0101960E94EE58F6
:102890000C94721D60EF77E0CE0183960E94976DD5
:1028A000BE016D5D7F4F82E491E10E94676B8111F3
:1028B00035C063EF77E0CE0145960E94976DBE016B
:1028C0006B5E7F4F82E491E10E94676B811117C0BC
:1028D00066EF77E0CE0101960E94976DBE016F5FB3
:1028E0007F4F82E491E10E94676BFF24F394811192
:1028F00001C0F12CCE0101960E94CD6C02C0FF24D4
:10290000F3948E010B5E1F4FC8010E94CD6CCE0167
:1029100083960E94CD6CF11005C02DC1CE01839627
:102920000E94CD6C0AE010E0C12CD12C7601AA24C3
:10293000AA9483E0B82E6EE170E080E090E00E94FF
:10294000BE49809110020E947449B5010E94DA9B31
:10295000072E000C880B990B0E940F9720E030E0A7
:1029600040EA50E40E946E979B01AC01C701B6019A
:102970000E9499986B017C0101501109E1F620E059
:1029800030E040E251E40E945F996B017C0169EF05
:1029900077E0CE0145960E94976DBE016B5E7F4F3A
:1029A00082E491E10E94676B81110C949B1D6DEF95
:1029B00077E0CE0101960E94976DBE016F5F7F4F59
:1029C00082E491E10E94676B11E0811101C010E087
:1029D000CE0101960E94CD6CCE0145960E94CD6C31
:1029E000112309F43FC020E030E040E650E4C70185
:1029F000B6010E946E979B01AC0160E070E080E838
:102A000090E40E949898AB01BC0140930C02509353
:102A10000D0260930E0270930F0222E0CE01019628
:102A20000E94016DBE016F5F7F4F8AE291E10E94BB
:102A3000826BCE0101960E94CD6C61E078E0CE0100
:102A400001960E94976D6AE271E1CE0101960E94A3
:102A5000266CBC018AE291E10E94B86CCE0101961D
:102A60000E94CD6C60E178E0CE0145960E94976DA2
:102A7000BE016B5E7F4F82E491E10E94676B811122
:102A80000C949E1D65E178E0CE0101960E94976D41
:102A9000BE016F5F7F4F82E491E10E94676B11E09E
:102AA000811101C010E0CE0101960E94CD6CCE01D3
:102AB00045960E94CD6C112309F43FC020E030E020
:102AC00040E650E4C701B6010E946E979B01AC013D
:102AD00060E070E080E291E40E949898AB01BC0154
:102AE000409308025093090260930A0270930B020C
:102AF00022E0CE0101960E94016DBE016F5F7F4F03
:102B00008AE291E10E94826BCE0101960E94CD6C17
:102B10006AE178E0CE0101960E94976D6AE271E168
:102B2000CE0101960E94266CBC018AE291E10E94CE
:102B3000B86CCE0101960E94CD6C6CE97AE0CE01B2
:102B400001960E94976D6AE271E1CE0101960E94A2
:102B5000266CBC01CE0145960E948F6DCE01459634
:102B60000E949E7CCE0145960E94CD6CCE010196BE
:102B70000E94CD6CBDC76AE278E0CE0101960E944A
:102B8000976DBE016F5F7F4F82E491E10E94676B9A
:102B9000F82ECE0101960E94CD6CFF2009F468C08A
:102BA0008091461190914711079708F4A1C746E01C
:102BB00050E062E471E1CE0101960E948C5EBE019C
:102BC0006F5F7F4F84E291E10E94826BCE0101969C
:102BD0000E94CD6C0E949284AB01BC01409318020C
:102BE0005093190260931A0270931B0221E0C801EE
:102BF0000E94016D67EA76E0CE0101960E94976D12
:102C0000B801CE0101960E94266C6CEE78E00E941D
:102C10000F6CBC018AE291E10E94B86CCE01019672
:102C20000E94CD6CC8010E94CD6C6AE271E1CE01B8
:102C300001960E948F6DCE0101960E949E7CCE016E
:102C400001960E94CD6C0E94F64928EE33E040E0E8
:102C500050E00E946798CA01B9010E940D976093E5
:102C6000000C7093010C8093020C9093030C40C7EE
:102C700061E378E0CE0101960E94976DBE016F5F1F
:102C80007F4F82E491E10E94676BF82ECE0101969E
:102C90000E94CD6CFF20C1F18091461190914711A7
:102CA000079708F425C746E050E062E471E1CE01E1
:102CB00001960E948C5EBE016F5F7F4F84E291E1BE
:102CC0000E94826BCE0101960E94CD6C0E9492847C
:102CD000AB01BC014093140250931502609316029D
:102CE0007093170221E0C8010E94016D67EB76E046
:102CF000CE0101960E94976DB801CE0101960E9407
:102D0000266C6CEE78E083C368E378E0C8010E942B
:102D1000976DB80182E491E10E94676B811117C041
:102D20006CE378E0CE0101960E94976DBE016F5F63
:102D30007F4F82E491E10E94676BFF24F39481113D
:102D400001C0F12CCE0101960E94CD6C02C0FF247F
:102D5000F394C8010E94CD6CFF2009F455C0809106
:102D60000602909107020E94467D60935C04709376
:102D70005D0480935E0490935F046093BD0C709338
:102D8000BE0C8093BF0C9093C00C80E090E0A0E854
:102D9000BFE38093640490936504A0936604B093AA
:102DA00067048093B50C9093B60CA093B70CB093C6
:102DB000B80C80913B0C882381F06EE174E082EACC
:102DC0009FE00E94046E60915C0470915D048091AC
:102DD0005E0490915F040E94EC431092650C109287
:102DE000640C80E090E00E94376240915C04509156
:102DF0005D0460915E0470915F0422E0C8010E944E
:102E0000016D60E478E04FC669E478E0C8010E9493
:102E1000976DB80182E491E10E94676B811117C040
:102E20006FE478E0CE0101960E94976DBE016F5F5E
:102E30007F4F82E491E10E94676BFF24F39481113C
:102E400001C0F12CCE0101960E94CD6C02C0FF247E
:102E5000F394C8010E94CD6CFF2009F4B8C08091A2
:102E60004611909147110797E8F046E050E062E480
:102E700071E1CE0101960E948C5EBE016F5F7F4FB3
:102E800084E291E10E94826BCE0101960E94CD6C9A
:102E90000E94928460934C0470934D0480934E047E
:102EA00090934F04809104029091050299270E940B
:102EB0005451BC01990F880B990B0E940F972DE07C
:102EC00038E643E55BE30E946E976B017C0120913D
:102ED000A8043091A9044091AA045091AB040E9427
:102EE000099718164CF060919004709191048091AC
:102EF0009204909193041BC02091BC043091BD04B6
:102F00004091BE045091BF04C701B6010E944E9A81
:102F100087FF05C0C701B6010E94666108C06091C5
:102F2000A4047091A5048091A6049091A70420E0C8
:102F300030E048EC52E40E946E976B017C0120E087
:102F400030E0A9010E940997181634F0C12CD12C49
:102F5000A8EAEA2EA1E4FA2EC0924C04D0924D04C5
:102F6000E0924E04F0924F04C092DD0CD092DE0C41
:102F7000E092DF0CF092E00C80913B0C882381F012
:102F80006CE074E082EA9FE00E94046E60914C0461
:102F900070914D0480914E0490914F040E94EC4337
:102FA0001092650C1092640C80E090E00E943762F1
:102FB00040914C0450914D0460914E0470914F0427
:102FC00022E0C8010E94016D65E578E06CC56FE5FF
:102FD00078E0C8010E94976DB80182E491E10E94F7
:102FE000676B811117C064E678E0CE0101960E94FC
:102FF000976DBE016F5F7F4F82E491E10E94676B26
:10300000FF24F394811101C0F12CCE0101960E949E
:10301000CD6C02C0FF24F394C8010E94CD6CFF2048
:1030200009F494C080914611909147110697F8F0E9
:1030300045E050E062E471E1CE0101960E948C5EB1
:10304000BE016F5F7F4F84E291E10E94826BCE01EF
:1030500001960E94CD6C0E9492840E948F9A609388
:1030600054047093550480935604909357048091B0
:10307000C8049091C9040E94928F20E030E048E09B
:1030800051E40E945F996093C4047093C5048093D7
:10309000C6049093C7046093CD0C7093CE0C8093BC
:1030A000CF0C9093D00C8091540490915504A09132
:1030B0005604B09157048093D50C9093D60CA093EE
:1030C000D70CB093D80C80913B0C882341F16BEF67
:1030D00073E082EA9FE00E94046E209154043091D4
:1030E0005504409156045091570460E070E080E22E
:1030F00091E40E940D9B41E050E00E941F6069E650
:1031000078E082EA9FE00E94F56E6091C4047091BD
:10311000C5048091C6049091C7040E94EC431092AC
:10312000650C1092640C80E090E00E943762409140
:10313000C4045091C5046091C6047091C70423E093
:10314000C8010E94016D60E778E0BEC06BE778E0DF
:10315000C8010E94976DB80182E491E10E94676BFB
:10316000811117C060E878E0CE0101960E94976D4A
:10317000BE016F5F7F4F82E491E10E94676BFF2485
:10318000F394811101C0F12CCE0101960E94CD6C07
:1031900002C0FF24F394C8010E94CD6CFF2009F403
:1031A0009FC080914611909147110697F8F045E035
:1031B00050E062E471E1CE0101960E948C5EBE0196
:1031C0006F5F7F4F84E291E10E94826BCE01019696
:1031D0000E94CD6C0E9492840E948F9A609350044A
:1031E0007093510480935204909353048091C804C7
:1031F0009091C9040E94928F20E030E048E051E4B1
:103200000E945F996093C0047093C1048093C204CC
:103210009093C3046093D10C7093D20C8093D30C21
:103220009093D40C8091500490915104A091520439
:10323000B09153048093D90C9093DA0CA093DB0CDB
:10324000B093DC0C80913B0C882341F16BEE73E072
:1032500082EA9FE00E94046E209150043091510454
:10326000409152045091530460E070E080E291E498
:103270000E940D9B41E050E00E941F6069E678E0EB
:1032800082EA9FE00E94F56E6091C0047091C104D3
:103290008091C2049091C3040E94EC431092650C8B
:1032A0001092640C80E090E00E9437624091C0046C
:1032B0005091C1046091C2047091C30423E0C8011D
:1032C0000E94016D65E878E0CE0101960E94976D3D
:1032D000B801CE0101960E94266C69E778E097C09C
:1032E0006EE878E0C8010E94976DB80182E491E130
:1032F0000E94676B811117C062E978E0CE010196E8
:103300000E94976DBE016F5F7F4F82E491E10E9442
:10331000676BFF24F394811101C0F12CCE0101965B
:103320000E94CD6C02C0FF24F394C8010E94CD6CB2
:10333000FF2009F46FC07090020260E0872D0E94A8
:103340003549F9E1AF2EB12CC12CD12C7601872D56
:103350000E947449BC01990F880B990B0E940F972A
:103360009B01AC01C701B6010E9499986B017C01D9
:103370006AE070E080E090E00E94BE49F1E0AF1AA0
:10338000B10829F720E030E040EA50E4C701B60177
:103390000E946E9720E030E040E85AE30E946E976A
:1033A00020E030E048EC51E40E945F9960934804CB
:1033B0007093490480934A0490934B046093F30CF8
:1033C0007093F40C8093F50C9093F60C1092650CAE
:1033D0001092640C80E090E00E94376240914804B3
:1033E0005091490460914A0470914B0422E0C80155
:1033F0000E94016D6EE376E0CE0101960E94976D0A
:10340000B801CE0101960E94266C6BE076E00E9426
:103410000F6C52C366E978E0C8010E94976DB8014D
:1034200082E491E10E94676B811117C06AE978E03C
:10343000CE0101960E94976DBE016F5F7F4F82E4BF
:1034400091E10E94676BFF24F394811101C0F12C7C
:10345000CE0101960E94CD6C02C0FF24F394C801F6
:103460000E94CD6CFF2009F43BC126E030E044E02F
:1034700050E062E471E1CE0101960E94AB6DBE01A5
:103480006F5F7F4F84E291E10E94826BCE010196D3
:103490000E94CD6C84E291E10E94EC6A4B015C01D8
:1034A0001B0165E376E0CE0101960E94976DCE0187
:1034B00001960E949E84AC014F5F5F4F62E471E110
:1034C000C8010E948C5EB80184E291E10E94826B87
:1034D000C8010E94CD6CCE0101960E94CD6CF09087
:1034E00000020E9492842B013C01640141E0C41A55
:1034F000D10880913B0C8823B9F063E773E082EA3E
:103500009FE00E94046E4AE050E0B40182EA9FE02E
:103510000E94CC6E6AEC79E082EA9FE00E94F56E30
:10352000C301B2010E94EC436F2DC8010E948E4D71
:1035300018870F831D821E82198289E08A8381E0A9
:103540008B838C831C8A1B8ACE0101960E94EA4CD5
:10355000CE0101960E947D4BCE0101960E94FD4452
:10356000EE80F12C6BE0E616F1041CF0EAE0EE2EA2
:10357000F12C7BE58716910408F44CC07CE3A72E60
:103580007CE0B72E3501212C312C2101C12CD12C0E
:10359000CE14DF04B9F06C2DCE0101960E947C4C54
:1035A0009B01AC01F30161937193819391933F016E
:1035B000C201B1010E9499981B012C01FFEFCF1AA3
:1035C000DF0AE6CFB7010F2C000C880B990B0E9485
:1035D0000F979B01AC01C201B1010E945F992B01C1
:1035E0003C01C12CD12CCE14DF0409F457C0F501E5
:1035F0002081318142815381C301B2010E94989898
:10360000F50161937193819391935F01FFEFCF1A5D
:10361000DF0AE9CF121413040CF5E214F30424F4C6
:10362000670141E0C41AD1086C2DCE0101960E94B9
:103630007C4C9B01AC01C601880F991F880F991F14
:10364000BC01645C734F6B01C301B2010E94989886
:10365000F601608371838283938320C02328F1F471
:103660009CE3A92E9CE0B92EC12CD12CCE14DF04F2
:10367000A9F06C2DCE0101960E947C4C9B01AC01FF
:10368000C301B2010E949898F501619371938193EF
:1036900091935F01FFEFCF1ADF0AE8CFECE3FCE084
:1036A000A7EFBCE041915191619171914D935D9370
:1036B0006D937D934CE0E436F407A1F71092650C0E
:1036C0001092640C80E090E00E94376244E050E089
:1036D00062E471E1C8010E948C5E6EE978E0E3C1AA
:1036E0006FEB78E0C8010E94976DB80182E491E128
:1036F0000E94676B811117C063EC78E0CE010196E0
:103700000E94976DBE016F5F7F4F82E491E10E943E
:10371000676BFF24F394811101C0F12CCE01019657
:103720000E94CD6C02C0FF24F394C8010E94CD6CAE
:10373000FF2009F455C080910602909107020E9473
:10374000467D609358047093590480935A04909373
:103750005B046093C10C7093C20C8093C30C909374
:10376000C40C80E090E5A3ECB7E4809360049093F0
:103770006104A0936204B09363048093B90C9093A6
:10378000BA0CA093BB0CB093BC0C80913B0C88236B
:1037900081F06DEC73E082EA9FE00E94046E60911C
:1037A00058047091590480915A0490915B040E94CE
:1037B000EC431092650C1092640C80E090E00E9443
:1037C0003762409158045091590460915A047091A5
:1037D0005B0422E0C8010E94016D67EC78E063C1E0
:1037E00062ED78E0C8010E94976DB80182E491E132
:1037F0000E94676B811117C066ED78E0CE010196DB
:103800000E94976DBE016F5F7F4F82E491E10E943D
:10381000676BFF24F394811101C0F12CCE01019656
:103820000E94CD6C02C0FF24F394C8010E94CD6CAD
:10383000FF2009F484C080914611909147110497AC
:10384000E8F044E050E062E471E1CE0101960E94AC
:103850008C5EBE016F5F7F4F84E291E10E94826BBC
:10386000CE0101960E94CD6C0E9492846093640404
:103870007093650480936604909367048091640458
:1038800090916504A0916604B09167048093B50C93
:103890009093B60CA093B70CB093B80C80913B0CEE
:1038A000882391F064EB73E082EA9FE00E94046E4B
:1038B000609164047091650480916604909167043E
:1038C00042E050E00E941F60809106029091070242
:1038D0000E94467D60935C0470935D0480935E0457
:1038E00090935F046093BD0C7093BE0C8093BF0CEB
:1038F0009093C00C80913B0C882381F06AEA73E0BE
:1039000082EA9FE00E94046E60915C0470915D0405
:1039100080915E0490915F040E94EC431092650CCC
:103920001092640C80E090E00E94376240915C0449
:1039300050915D0460915E0470915F04AEC062EED0
:1039400078E0C8010E94976DB80182E491E10E947D
:10395000676B811117C066EE78E0CE0101960E9478
:10396000976DBE016F5F7F4F82E491E10E94676BAC
:10397000FF24F394811101C0F12CCE0101960E9425
:10398000CD6C02C0FF24F394C8010E94CD6CFF20CF
:1039900009F4AEC080914611909147110497E8F068
:1039A00044E050E062E471E1CE0101960E948C5E39
:1039B000BE016F5F7F4F84E291E10E94826BCE0176
:1039C00001960E94CD6C0E94928460936004709373
:1039D00061048093620490936304809160049091E9
:1039E0006104A0916204B09163048093B90C909338
:1039F000BA0CA093BB0CB093BC0C80913B0C8823F9
:103A000091F061E973E082EA9FE00E94046E6091A8
:103A1000600470916104809162049091630442E0BB
:103A200050E00E941F6080910602909107020E9460
:103A3000467D609358047093590480935A04909380
:103A40005B046093C10C7093C20C8093C30C909381
:103A5000C40C80913B0C882381F067E873E082EA14
:103A60009FE00E94046E6091580470915904809107
:103A70005A0490915B040E94EC431092650C1092E2
:103A8000640C80E090E00E943762409158045091AD
:103A9000590460915A0470915B0422E0C8010E94AD
:103AA000016D6AED78E0CE0101960E94976DB80134
:103AB000CE0101960E94266CBC018AE291E10E942F
:103AC000B86CCE0101960E94CD6CC8010E94CD6CED
:103AD0006AE271E1CE0101960E948F6DCE010196DE
:103AE0000E949E7CCE0101960E94CD6C1092130222
:103AF00080911302882371F062E471E1CE01019696
:103B00000E948F6DCE0101960E94EE58CE01019663
:103B10000E94CD6C0E94F6496093040C7093050CD2
:103B20008093060C9093070C67E57BE082E491E1BB
:103B30000E94A36C06C011E00C94EC1411E00C94EC
:103B40005715EA960FB6F894DEBF0FBECDBFDF91D2
:103B5000CF911F910F91FF90EF90DF90CF90BF908A
:103B6000AF909F908F907F906F905F904F903F901D
:103B70002F9008952F923F924F925F926F927F9273
:103B80008F929F92AF92BF92CF92DF92EF92FF926D
:103B90000F931F93CF93DF93CDB7DEB7CA54D109EC
:103BA0000FB6F894DEBF0FBECDBF1C01E090330C02
:103BB000F090340C80913B0C882349F064E176E06E
:103BC00082EA9FE00E94046EC1010E947743810156
:103BD0000B5F1F4F0530110508F18091330C909158
:103BE000340C8215930519F10E94CC560E94C44EE4
:103BF0003092340C2092330C4AE0B101CE01019690
:103C00000E945C6DBE016F5F7F4F86E391E10E9471
:103C1000826BCE0101960E94CD6C09C02EEF221658
:103C20002FEF320621F40E94D34E0C94183367E52F
:103C30007BE08AE291E10E94A36C0530110590F0CF
:103C40006AEC79E0CE0101960E94976D4AE050E05F
:103C50006FEF7FEFCE0101960E949757CE0101963C
:103C60000E94CD6CF1017996E533F10510F00C94CA
:103C700065328827EE58FF4F8F4F0C94ED9B809153
:103C8000B912882309F442C188E69EE00E943E7082
:103C900061E080912F040E94354960E080912D04FD
:103CA0000E9435490E9454426093350C7093360C43
:103CB0008093370C9093380C0E94654E0E94824E80
:103CC000AB01BC0123E0CE0145960E94016DBE010F
:103CD0006B5E7F4FCE0101960E948F6D6EED7AE094
:103CE000CE0101960E940F6CBC0184E291E10E941A
:103CF000B86CCE0101960E94CD6CCE0145960E9413
:103D0000CD6C67E279E0CE0101960E94976D64E286
:103D100071E1CE0101960E94266CBC018AE291E11C
:103D20000E94B86CCE0101960E94CD6C0E94824E1A
:103D30009B01AC0128966FAF289729963FAF299732
:103D40002A964FAF2A972B965FAF2B970E949949DF
:103D50002B013C016EE170E080E090E00E94BE49E2
:103D60000E94824E6B017C010E9499494B015C01CB
:103D700084189508A608B70828962FAD2897299685
:103D80003FAD29972A964FAD2A972B965FAD2B977B
:103D900081ED881687E09806A104B1040CF43FC0B9
:103DA000C701B6010E9498986B017C0120E030E0C9
:103DB000A9010E944E9A18165CF426EA3BE944ECED
:103DC0005BE3C701B6010E94099787FF0BC027C0BC
:103DD00026EA3BE944EC5BEBC701B6010E944E9A30
:103DE0001816ECF0C501B40128EE33E040E050E0D5
:103DF0000E943B98CA01B9010E940F974B015C01D8
:103E000020E030E04AE754E4C701B6010E946E9713
:103E1000A50194010E945F99AB01BC0103C040E081
:103E200050E0BA0122E0CE0145960E94016DBE012C
:103E30006B5E7F4FCE0101960E948F6D6AEE78E037
:103E4000CE0101960E940F6CBC018EE191E10E94AF
:103E5000B86CCE0101960E94CD6CCE0145960E94B1
:103E6000CD6C6EEE78E0CE0101960E94976D6EE10A
:103E700071E1CE0101960E94266CBC018AE291E1BB
:103E80000E94586CCE0101960E94CD6C6AEC79E0DC
:103E9000CE0101960E94976D6EE171E1CE0101960F
:103EA0000E94266CBC0184E291E10E94586CCE0114
:103EB00001960E94CD6C63E474E0CE0101960E94ED
:103EC000876D4AE050E060E070E0CE0101960E940C
:103ED0004D58CE0101960E94CD6C64E271E1CE0195
:103EE00001960E948F6D45E050E06FEF7FEFCE01AD
:103EF00001960E941C57CE0101960E94CD6C62EF84
:103F000078E08AE291E10E944A6CEBC1C090140211
:103F1000D0901502E0901602F09017020E94F64928
:103F20006BAF7CAF8DAF9EAF88E69EE00E943E7087
:103F300061E080912F040E94354960E080912D045A
:103F40000E9435490E9454426093350C7093360CA0
:103F50008093370C9093380C0E94654E0E94824EDD
:103F600023966CAF7DAF8EAF9FAF23970E94994988
:103F70004B015C016AE070E080E090E00E94BE4985
:103F800065E079E08AE291E10E94A36C20E030E0F4
:103F90004AE754E4C701B6010E946E9727966CAFBA
:103FA0007DAF8EAF9FAF2797412C512C3201C12C92
:103FB000D12C7601C701B6010E940F9727962CAD30
:103FC0003DAD4EAD5FAD27970E94099787FF89C130
:103FD0000E94F6492BAD3CAD4DAD5EAD621B730B3F
:103FE000840B950B0E940D9720E030E04AE754E4E3
:103FF0000E945F99AB01BC0123E0CE0101960E94B3
:10400000016DBE016F5F7F4F84E291E10E94826B80
:10401000CE0101960E94CD6C0E94824E6B017C0104
:104020000E9499499B01AC01281939094A095B0989
:1040300049015A0131ED831637E09306A104B1041A
:104040000CF443C020E030E0A901C701B6010E9492
:104050004E9A18165CF426EA3BE944EC5BE3C70190
:10406000B6010E94099787FF0BC02FC026EA3BE9E3
:1040700044EC5BEBC701B6010E944E9A18162CF176
:10408000C501B40128EE33E040E050E00E943B98C7
:10409000CA01B9010E940F974B015C0123962CAD18
:1040A0003DAD4EAD5FAD2397C701B6010E94989814
:1040B00020E030E04AE754E40E946E97A5019401A5
:1040C0000E945F994B015C0103C0812C912C54012B
:1040D00064E271E1CE0101960E948F6D6CEE78E092
:1040E000CE0101960E940F6CBC0184E291E10E9416
:1040F000B86CCE0101960E94CD6C23E0B701A601F9
:10410000CE0145960E94016DBE016B5E7F4FCE01D0
:1041100001960E948F6D63E279E0CE0101960E94C4
:104120000F6CBC018EE191E10E94B86CCE0101964A
:104130000E94CD6CCE0145960E94CD6C22E0B50167
:10414000A401CE0101960E94016D65E27BE0CE01E3
:1041500045960E94976D64E271E1CE0145960E94FA
:10416000266C66E279E00E940F6C6EE171E10E94BC
:10417000266C6FEE78E00E940F6CBE016F5F7F4F80
:104180000E94266C6AEE78E00E940F6CBC018AE205
:1041900091E10E94586CCE0145960E94CD6CCE01F3
:1041A00001960E94CD6C20E030E0A901C501B40168
:1041B0000E944E9A87FD06C06AEC79E08EE191E19B
:1041C0000E944A6C22E0B501A401CE0145960E94EE
:1041D000016DBE016B5E7F4FCE0101960E948F6D17
:1041E0006AEE78E0CE0101960E940F6CBC018EE170
:1041F00091E10E94586CCE0101960E94CD6CCE01D7
:1042000045960E94CD6C6AE271E1CE0101960E9452
:104210008F6DCE0101960E949E7CCE0101960E9478
:10422000CD6CC301B20125E030E040E050E00E94D7
:104230003B98672B682B692B21F56AE474E0CE016B
:1042400001960E94876D45E050E060E070E0CE018D
:1042500001960E944D58CE0101960E94CD6C6EE1F0
:1042600071E1CE0101960E948F6D45E050E06FEF45
:104270007FEFCE0101960E941C57CE0101960E944D
:10428000CD6C67E57BE08AE291E10E94A36C65E07A
:1042900070E080E090E00E94BE490E94F6496B0108
:1042A0007C012BAD3CAD4DAD5EADC21AD30AE40A24
:1042B000F50A0E94824E23966CAF7DAF8EAF9FAF02
:1042C00023970E9499494B015C016AE070E080E00D
:1042D00090E00E94BE493FEF431A530A630A730AF3
:1042E00069CE60E080912F040E9435490C9493328E
:1042F000F090000267E57BE0CE01C5960E94976DC5
:104300008E010B5E1F4F6F2DC8010E948E4D1887C6
:104310000F831D821E82198289E08A8381E08B834C
:104320008C831C8A1B8ACE0101960E94EA4CCE0126
:1043300001960E947D4BCE0101960E94FD440E81A4
:1043400010E00330110509F46AC16FE674E0CE0194
:10435000C5960E945E6C67E57BE08AE291E10E946F
:10436000A36CBE016B5C7F4FCE0183960E948F6D64
:104370004AE050E060E070E0CE0183960E944D5824
:10438000CE0183960E94CD6C61E080E00E94165FB2
:1043900069E379E0CE01C5960E94A36C4CE3A42E9C
:1043A0004CE0B42ECC24C394D12CE12CF12CE0169B
:1043B000F1060CF0ECC06E2DCE0101960E947C4CF3
:1043C000D5012D913D914D915D915D010E9499988E
:1043D0002B013C0120E030E04CEF52EC0E940997A9
:1043E00087FF21C04AE0B601CE0183960E945C6D32
:1043F0006BE677E0CE0189960E94976DBE016D5DF8
:104400007F4FCE0189960E94266C6AE279E00E9475
:104410000F6CBC018AE291E10E94586CCE01899632
:104420000E94CD6C45C022E0B301A201CE0183966B
:104430000E94016D4AE0B601CE0189960E945C6D32
:104440006BE677E0CE018F960E94976DBE01675DA7
:104450007F4FCE018F960E94266C65E376E00E9426
:104460000F6CBE016D5D7F4F0E94266CBC018EE11A
:1044700091E10E94B86CCE018F960E94CD6CCE0166
:1044800089960E94CD6CCE0183960E94CD6C6EE120
:1044900071E1CE0183960E948F6D6AEC79E0CE01C6
:1044A00083960E940F6CBC018AE291E10E94586CD5
:1044B000CE0183960E94CD6C0130110559F4E114B0
:1044C000F10409F05DC06AE271E1CE01C5960E9477
:1044D000B86C56C00230110511F522E0B301A201FB
:1044E000CE0189960E94016DBE01675D7F4FCE01AE
:1044F00083960E948F6D6AEC79E0CE0183960E94CC
:104500000F6CBC01CE01C5960E94586CCE018396FB
:104510000E94CD6CCE0189960E94CD6C31C00330D3
:10452000110571F16EE171E1CE0183960E948F6DEC
:1045300044E150E06FEF7FEFCE0183960E941C575D
:10454000CE0183960E94CD6C66ED79E0CE01839614
:104550000E94976DCE0183960E94F056CE018396FD
:104560000E94CD6C80911202882351F08091E20468
:10457000882331F060ED77E080E090E00E94BE4952
:10458000BFEFEB1AFB0AEFEFCE1ADE0A10CFCE0117
:10459000C5960E94F76A8AE291E10E94F76A0115C6
:1045A0001105A9F46CE574E08AE291E10E945E6C69
:1045B00061E574E0CE0183960E94876D4AE050E089
:1045C0006FEF7FEFCE0183960E941C57ECC0043042
:1045D000110514F00C94B532BE016B5C7F4FCE0117
:1045E00083960E948F6D4AE050E06FEF7FEFCE011F
:1045F00083960E941C57CE0183960E94CD6C66ED77
:1046000079E0CE0183960E94976DCE0183960E9439
:10461000F056CE0183960E94CD6C0C94B53266E3C1
:1046200079E0CE01C5960E94A36CBE016B5C7F4F02
:10463000CE0183960E948F6D4AE050E060E070E00A
:10464000CE0183960E944D58CE0183960E94CD6C78
:1046500067E57BE08AE291E10E94A36C6AE271E186
:10466000CE01C5960E94B86C00E010E0602FCE012C
:1046700001960E947C4C6B017C0122E0AB01BC01E5
:10468000CE010115110569F483960E94016DBE01EA
:104690006D5D7F4F8BE292E10E94F66DCE018396B5
:1046A0001BC089960E94016DBE01675D7F4FCE01E0
:1046B00083960E948F6D6AEC79E0CE0183960E940A
:1046C0000F6CBC01CE01C5960E94586CCE0183963A
:1046D0000E94CD6CCE0189960E94CD6C22E0B7017C
:1046E000A601CE0189960E94016DBE01675D7F4FD4
:1046F000CE0183960E948F6D6AEC79E0CE0183969D
:104700000E940F6CBC018AE291E10E94586CCE01BC
:1047100083960E94CD6CCE0189960E94CD6C0F5F6E
:104720001F4F0330110509F0A1CFCE01C5960E949D
:10473000F76ABE016B5C7F4FCE0183960E948F6D3E
:104740004AE050E06FEF7FEFCE0183960E941C5746
:10475000CE0183960E94CD6C66ED79E0CE01839602
:104760000E94976DCE0183960E94F056CE018396EB
:104770000E94CD6C8AE291E10E94F76A6CE379E0D5
:10478000CE0183960E94976D6AE271E1CE01839615
:104790000E94266C66E479E00E940F6CBC018AE2FC
:1047A00091E10E94B86CCE0183960E94CD6CCE013F
:1047B000C5960C94913280910202909103020E945E
:1047C00076510C94933280910402909105020E94DC
:1047D00001560C9493320E94CC5665EA74E08AE24A
:1047E00091E10E945E6C6AE271E1CE0101960E9445
:1047F0008F6D4AE050E060E070E0CE0101960E94CB
:104800004D58CE0101960E94CD6C6CE974E084E2B3
:1048100091E10E945E6C64E271E1CE0101960E941A
:104820008F6D44E150E06FEF7FEFCE0101960E9463
:104830001C57CE0101960E94CD6C80910C0C90917A
:104840000D0C8230910549F40E94CD8381111AC06C
:1048500010920D0C10920C0C15C0892B99F40E942B
:10486000CD83882339F082E090E090930D0C809303
:104870000C0C08C00E94CD838111F5CF0E94CD831E
:104880008111F1CF80910C0C90910D0C029741F1A8
:1048900060E974E08AE291E10E945E6C6AE271E193
:1048A000CE0101960E948F6D4AE050E060E070E01A
:1048B000CE0101960E944D58CE0101960E94CD6C0A
:1048C0006AE271E1CE0101960E948F6D6AEC79E097
:1048D000CE0101960E940F6C64E271E10C94302DC0
:1048E0008AE090E00E94FE4E6B017C0120E030E007
:1048F000A9010E940997181634F08AE090E00E94FE
:10490000FE4E6B017C010BE010E020E030E042ED58
:1049100053E4C701B6010E940997181684F420E0F9
:1049200030E0A901C701B6010E9409971816BCF032
:1049300062E874E08AE291E10E945E6C41C001503D
:10494000110969F368EC70E080E090E00E94BE49D4
:1049500083E090E00E94FE4E6B017C01D6CF20E008
:1049600030E048EC52E4C701B6010E94099787FF86
:1049700002C021E001C020E0B701A601CE010196EE
:104980000E94016D69E579E0CE0145960E94976D20
:10499000BE016F5F7F4FCE0145960E94266C6EE58B
:1049A00079E00E940F6CBC018AE291E10E94B86C30
:1049B000CE0145960E94CD6CCE0101960E94CD6C31
:1049C0006AE271E1CE0101960E948F6D42E350E0F0
:1049D0006FEF7FEFCE0101960E941C57CE0101962A
:1049E0000E94CD6C69E774E084E291E10E945E6C04
:1049F00064E271E1CE0101960E948F6D42E350E0C6
:104A000060E070E0CE0101960E944D58CE01019603
:104A10000E94CD6C8091B912882311F40C949332CA
:104A200060E273E080E090E08CC10E94F6490E9451
:104A3000EF530C949332009106021091070262E644
:104A400079E084E291E10E94A36C0E94CC5664E27A
:104A500071E1CE0101960E948F6D4AE050E06FEF48
:104A60007FEFCE0101960E944D58CE0101960E9423
:104A7000CD6CC8010E94467D23966CAF7DAF8EAF92
:104A80009FAF239780905C0490905D04A0905E049B
:104A9000B0905F04A501940160915804709159048D
:104AA00080915A0490915B040E9498982B013C01DC
:104AB00020E030E0A9010E940997882309F451C041
:104AC000C0906404D0906504E0906604F0906704A0
:104AD00020E030E0A901C701B6010E94099718162D
:104AE0000CF03FC020916004309161044091620459
:104AF000509163042BAF3CAF4DAF5EAFC701B60121
:104B00000E940997882369F1A70196016BAD7CADDE
:104B10008DAD9EAD0E945F990E949A9A6BAF7CAF5B
:104B20008DAF9EAFA501940123966CAD7DAD8EAD8A
:104B30009FAD23970E949898A30192010E945F99CC
:104B40002BAD3CAD4DAD5EAD0E946E970E94CC99F1
:104B50009B01AC01C701B6010E946E976B017C01FD
:104B600003C0C12CD12C760164E271E1CE01019623
:104B70000E948F6D4AE050E060E070E0CE01019647
:104B80000E944D58CE0101960E94CD6C20E030E687
:104B90004AEE56E4C701B6010E944E9A18163CF43C
:104BA0006FEA74E08AE291E10E945E6C25C021E028
:104BB000B701A601CE0145960E94016D6CE679E031
:104BC000CE0101960E94976DBE016B5E7F4FCE01B4
:104BD00001960E94266C60E779E00E940F6CBC0190
:104BE0008AE291E10E94B86CCE0101960E94CD6CE0
:104BF000CE0145960E94CD6C6AE271E1CE0101962C
:104C00000E948F6D4AE050E06FEF7FEFCE0101967A
:104C10000E941C57CE0101960E94CD6C64E670E0A4
:104C200080E090E00E94BE49F5CE00918E04109184
:104C30008F040E94CC56C8010E9454518C0162E33B
:104C400070E080E090E00E94BE49B801110F880B2F
:104C5000990B0E940F9720E030E040EA50E40E9458
:104C60006E9720E030EC4FE754E40E945F99AB016F
:104C7000BC0123E0CE0101960E94016D61EE7AE055
:104C8000CE0145960E94976DBE016F5F7F4FCE01AA
:104C900045960E94266C6BE076E00E940F6CBC018A
:104CA0008AE291E10E94B86CCE0145960E94CD6CDB
:104CB000CE0101960E94CD6C64E779E084E291E137
:104CC0000E94A36C64E271E1CE0101960E948F6D97
:104CD0004AE050E068E070E0CE0101960E944D5835
:104CE000CE0101960E94CD6C6AE271E1CE0101967F
:104CF0000E948F6D4AE050E06FEF7FEFCE0101968A
:104D00000E941C57CE0101960E94CD6C64E271E1B5
:104D10008AE291E10E94586C7DCE9091320C81E044
:104D200089278093320C8091B912882331F06AE28E
:104D300071E18BEC9DE00E94E56E68EC70E080E034
:104D400090E00E94BE490C9493321092B9120C94D8
:104D5000933281E08093B91266E371E18CE391E1D3
:104D60000E94B86C8091330C9091340C9093831214
:104D7000809382120C94933280913812882321F010
:104D8000109238120C9493320E94B2660C949332B3
:104D900085E09FE00E943E7040E052EC61E070E0F0
:104DA00085E09FE00E94255E8CED95E0A0E0B0E0FC
:104DB0008093090F90930A0FA0930B0FB0930C0FE1
:104DC00064E670E080E090E00E94BE4980910C0CA7
:104DD00090910D0C019759F483E090E00E9452539A
:104DE00081111EC010920D0C10920C0C19C081E0A4
:104DF00090E00E945253882339F081E090E0909334
:104E00000D0C80930C0C0CC083E090E00E94525378
:104E10008111F3CF83E090E00E9452538111EDCFD6
:104E200080910C0C90910D0C0197D9F06EEE74E00E
:104E300084E291E10E945E6C64E271E1CE01019630
:104E40000E948F6D44E150E06FEF7FEFCE0101963D
:104E50000E941C57CE0101960E94CD6C62EE74E058
:104E6000D0C066ED74E08AE291E10E945E6C6AE275
:104E700071E1CE0101960E948F6DCE0101960E94D4
:104E8000EE58CE0101960E94CD6C62E370E080E0A6
:104E900090E00E94BE496AE271E1CE0101960E9453
:104EA0008F6D42E350E06FEF7FEFCE0101960E94DD
:104EB0004D58CE0101960E94CD6C6AEC74E084E2FC
:104EC00091E10E945E6C64E271E1CE0101960E9464
:104ED0008F6D44E150E06FEF7FEFCE0101960E94AD
:104EE0001C57CE0101960E94CD6C8BEB8D8B8AEA0C
:104EF0008E8B81E08F8B412C512C32011CAE1BAE6E
:104F0000C12CD12C0AE010E0C601B8010E94DA9B46
:104F1000892B49F443E050E0BE016B5E7F4F85E092
:104F20009FE00E94826965E070E080E090E00E946E
:104F3000BE493FEFC31AD30AE12CF12C812C912CEE
:104F4000540185E09FE00E94F769892B61F444E0F9
:104F500084169104A104B10434F02BAD3CAD24308F
:104F6000310544F00CC036E0E316F10414F40C945F
:104F7000BD32F3CF40E9C41641E0D40629F6C3019F
:104F8000B2010E940F9720E030E040E251E40E941D
:104F90005F9920E030E040E85EE30E946E976B018D
:104FA0007C0120E030E040EA51E40E944E9A18165D
:104FB00034F521E0B701A601CE0101960E94016DF2
:104FC0006DEE77E0CE0145960E94976DBE016F5F52
:104FD0007F4FCE0145960E94266C6CE779E00E94D7
:104FE0000F6CBC018AE291E10E94B86CCE0145963B
:104FF0000E94CD6CCE0101960E94CD6C06C06EEB76
:1050000074E08AE291E10E945E6C6AE271E1CE0195
:1050100001960E948F6D4AE050E060E070E0CE01A2
:1050200001960E944D58CE0101960E94CD6C6AE215
:1050300071E1CE0101960E948F6D6AEC79E0CE019C
:1050400001960E940F6C64E271E10E94266CBC0123
:105050008AE291E10E94B86CCE0101960E94CD6C6B
:1050600085E09FE00E943E70D5CC69E875E0CE01F6
:1050700001960E94876D4AE050E06FEF7FEFCE010E
:1050800001960E941C57CE0101960E94CD6C609142
:105090008C0470918D0480914604909147040E9485
:1050A0009477B4E18B2E912CA12CB12CE12CF12C16
:1050B0008FEFE81AF80AC501B4010E94BE49609159
:1050C0008C0470918D0480914604909147040E9455
:1050D00094778C0193E0E916F10434F454E1850EE1
:1050E000911CA11CB11CE4CFAEE1EA16F1041CF442
:1050F000012BA1F704C00115110509F00DC1809124
:105100004604909147048B309105C9F48091881131
:1051100090918911A0918A11B0918B118093B51251
:105120009093B612A093B712B093B81280918411E5
:1051300090918511A0918611B09187111DC0863183
:10514000910521F30C9701F58091A8129091A91275
:10515000A091AA12B091AB128093B5129093B6129F
:10516000A093B712B093B8128091A4129091A51297
:10517000A091A612B091A7128093B1129093B2128F
:10518000A093B312B093B4124091B5125091B612DD
:105190006091B7127091B81221E0CE0101960E9481
:1051A000016D69E379E0CE0145960E94976DBE01DD
:1051B0006F5F7F4FCE0145960E94266CBC018AE24C
:1051C00091E10E94B86CCE0145960E94CD6CCE0153
:1051D00001960E94CD6C4091B1125091B212609133
:1051E000B3127091B41221E0CE0101960E94016DBC
:1051F0006FE779E0CE0145960E94976DBE016F5F23
:105200007F4FCE0145960E94266CBC018AE291E157
:105210000E94586CCE0145960E94CD6CCE0101963D
:105220000E94CD6C61E07BE08AE291E10E944A6CD1
:1052300067E57BE0CE0101960E94976D44E150E066
:1052400060E070E0CE0101960E944D58CE010196BB
:105250000E94CD6CC090B512D090B612E090B712FB
:10526000F090B81220E030E0A901C701B6010E9419
:105270004E9A20E030E040E05FE387FD05C0C701C3
:10528000B6010E94999804C0C701B6010E9498987F
:105290000E94F8992AE0AB01BC01CE0101960E9460
:1052A000306DBE016F5F7F4F84E291E10E94826B9F
:1052B000CE0101960E94CD6C60E087E00E94165FEF
:1052C00064E271E18BE292E10E94F66D6FED8BE298
:1052D00092E10E94EF6D65E879E08BE292E10E9435
:1052E000F56E6091B1127091B2128091B3129091EB
:1052F000B4120E94F8994AE050E08BE292E10E94D9
:10530000CC6E61E07BE08BE292E10E94F56E64E698
:1053100070E080E090E015CD0F3FBFEF1B07ACF0D1
:105320006BE775E0CE0101960E94876D4AE050E080
:1053300060E070E0CE0101960E944D58CE010196CA
:105340000E94CD6C68E575E065C00E3FEFEF1E076B
:1053500009F44CC06AE475E0CE0101960E94876DA5
:105360004AE050E060E070E0CE0101960E944D58A6
:10537000CE0101960E94CD6C6BE375E08AE291E16B
:105380000E945E6C4AE0B801CE0101960E945C6DFD
:10539000BE016F5F7F4F8AE291E10E94586CCE019F
:1053A00001960E94CD6C00912E1110912F110B5E71
:1053B0001F4FB8018AE291E10E94BB6B882311F470
:1053C0000C94933220912A1130912B1180912E113F
:1053D00090912F1165E275E0820F931F0E948392D6
:1053E00010932F1100932E110C9493326AE175E003
:1053F000CE0101960E94876D4AE050E060E070E0C7
:10540000CE0101960E944D58CE0101960E94CD6CAE
:105410006AEF74E08AE291E10E945E6C0C94933230
:1054200080913104882311F40C94933267E57BE07A
:10543000CE0101960E94976D4AE050E061E070E075
:10544000CE0101960E944D58CE0101960E94CD6C6E
:105450000E94CC560E947A402B013C010E9454428B
:105460004B015C0160917004709171048091720431
:10547000909173040E940F979B01AC0128966FAF27
:10548000289729963FAF29972A964FAF2A972B96B0
:105490005FAF2B970E947A400E940F9728962FADFE
:1054A000289729963FAD29972A964FAD2A972B9694
:1054B0005FAD2B970E945F9921E03EED42E45EE3F1
:1054C0000E940D9B9B01AC0160E070E080E89FE3CF
:1054D0000E94989820E03AE24DE257E40E946E97CD
:1054E0006B017C01C301B2010E940F9720E030E004
:1054F00048EC52E40E945F99AB01BC0122E0CE016E
:1055000001960E94016DBE016F5F7F4F8EE191E1B8
:105510000E94826BCE0101960E94CD6C6EEF76E008
:105520008EE191E10E944A6C6EE171E184E291E1C9
:105530000E94B86C6AEF76E0CE0101960E94976DEA
:105540006EE171E1CE0101960E94266CBC018EE1F4
:1055500091E10E94B86CCE0101960E94CD6C69E386
:1055600079E08AE291E10E94A36C21E0B501A401F7
:10557000CE0101960E94016DBE016F5F7F4F8AE2EE
:1055800091E10E94586CCE0101960E94CD6C68E8B2
:1055900079E08AE291E10E944A6C21E0B701A6011C
:1055A000CE0145960E94016DBE016B5E7F4FCE011C
:1055B00001960E948F6D6EED7AE0CE0101960E94F9
:1055C0000F6CBC018AE291E10E94586CCE010196F9
:1055D0000E94CD6CCE0145960E94CD6C6EE171E1CA
:1055E000CE0101960E948F6D6AEC79E0CE010196A2
:1055F0000E940F6C6AE271E10E94266CBC018AE293
:1056000091E10E94B86CCE0101960E94CD6C64E2DB
:1056100071E1CE0101960E948F6D4AE050E060E09A
:1056200070E0CE0101960E944D58CE0101960E9475
:10563000CD6C21E0B501A401CE0101960E94016D5F
:10564000BE016F5F7F4F80E391E10E94826BCE01CC
:1056500001960E94CD6C60E371E1CE0101960E943B
:105660008F6D4AE050E06FEF7FEFCE0101960E9410
:105670001C57CE0101960E94CD6C65E070E080E081
:1056800090E00E94BE4965E879E0CE0101960E9453
:10569000976DCE0101960E94F056CE0101960E94B0
:1056A000CD6C21E0B701A601CE0145960E94016DA7
:1056B000BE016B5E7F4FCE0101960E948F6D6EED35
:1056C0007AE0CE0101960E940F6CBC0180E391E16B
:1056D0000E94B86CCE0101960E94CD6CCE01459619
:1056E0000E94CD6C60E371E1CE0101960E948F6D46
:1056F0004AE050E068EF7FEFCE0101960E941C5710
:10570000CE0101960E94CD6C65E070E080E090E0F3
:105710000E94BE498091B912882309F404C768E544
:1057200072E080E090E00DCB8091B912882331F0D7
:10573000A2E04A2E512C612C712C05C0FEE14F2EA7
:10574000512C612C712C67E975E08AE291E10E948D
:105750005E6C6AE271E1CE0101960E948F6D4AE0B3
:1057600050E06FEF7FEFCE0101960E941C57CE01F3
:1057700001960E94CD6C812C912C5401C12CD12C0E
:10578000760183E20E94FB5E87E090E00E94F75E74
:105790000E94F55E66E970E080E090E00E94BE49FC
:1057A00083E20E94FB5E80E290E00E94F75E0E942E
:1057B000F55E66E970E080E090E00E94BE4962E03C
:1057C00070E083E290E00E94014040E050E0BA01C6
:1057D00080917F0D90E02091800D821B9109181619
:1057E00019062CF58FE390E12A964FAF2A972B9656
:1057F0005FAF2B9728966FAF289729967FAF299791
:105800000E94DE632A964FAD2A972B965FAD2B97A9
:1058100028966FAD289729967FAD2997762F652F0B
:10582000542F4427480F511D611D711DD1CFCB014D
:10583000BA010E940F972AE939E949E95FE30E941A
:105840005F990E94F899AB01BC01C416D506E60623
:10585000F70614F46A017B012AE0CE0145960E9406
:10586000306DBE016B5E7F4FCE0101960E948F6D41
:105870006EE879E0CE0101960E940F6CBC0184E2D3
:1058800091E10E94B86CCE0101960E94CD6CCE01D0
:1058900045960E94CD6C64E271E1CE0101960E94B2
:1058A0008F6D4EE150E060E070E0CE0101960E9405
:1058B0009757CE0101960E94CD6CFFEF8F1A9F0A79
:1058C000AF0ABF0A481459046A047B040CF059CF8C
:1058D0002AE0B701A601CE0145960E94306DBE01B7
:1058E0006B5E7F4FCE0101960E948F6D6EE879E06E
:1058F000CE0101960E940F6CBC0184E291E10E94EE
:10590000B86CCE0101960E94CD6CCE0145960E94E6
:10591000CD6C64E271E1CE0101960E948F6D4AE088
:1059200050E060E070E0CE0101960E944D58CE013B
:1059300001960E94CD6C2AE0B701A601CE01019626
:105940000E94306D62E979E0CE0145960E94976D24
:10595000BE016F5F7F4FCE0145960E94266C65E9C0
:1059600079E00E940F6C6AE271E10E94266CBC0132
:105970008AE291E10E94B86CCE0145960E94CD6CFE
:10598000CE0101960E94CD6C62E370E080E090E071
:10599000D8C900918A0410918B0481E0809385041A
:1059A00064E670E080E090E00E94BE490E94CC5620
:1059B000C8010E94545160E074E0681B790B4AE012
:1059C000CE0101960E945C6D6AE979E0CE014596B0
:1059D0000E94976DBE016F5F7F4FCE0145960E947A
:1059E000266CBC018AE291E10E94B86CCE0145961A
:1059F0000E94CD6CCE0101960E94CD6C60E087E0E4
:105A00000E94165F67EA75E0CE0101960E94876DDD
:105A100042E350E068E070E0CE0101960E944D58EC
:105A2000CE0101960E94CD6C6AE271E1CE01019631
:105A30000E948F6D42E350E06FEF7FEFCE01019641
:105A40000E941C57CE0101960E94CD6C61EA79E05C
:105A5000CE0101960E94976D6AE271E1CE01019636
:105A60000E94266CBC018AE291E10E94B86C0C9401
:105A7000062580918804909189040E9454518C01DC
:105A800090930F0C80930E0C62E370E080E090E046
:105A90000E94BE494AE0B801CE0101960E945C6DA9
:105AA000BE016F5F7F4F8AE291E10E94826BCE015F
:105AB00001960E94CD6C8091821190918311892B67
:105AC00009F45EC06EE771E1CE0145960E948F6DCC
:105AD000BE016B5E7F4FCE0101960E948F6D44E147
:105AE00050E060E070E0CE0101960E944D58CE017A
:105AF00001960E94CD6C6BEA79E0CE0101960E947E
:105B0000976D6AE271E1CE0101960E94266CBC019C
:105B100084E291E10E94B86CCE0101960E94CD6CA6
:105B200064E271E1CE0101960E948F6D44E150E084
:105B30006FEF7FEFCE0101960E941C57CE010196B8
:105B40000E94CD6CBE016B5E7F4FCE0101960E941C
:105B50008F6D6AEC79E0CE0101960E940F6C64E2D1
:105B600071E10E94266CBC018AE291E10E94B86C4E
:105B7000CE0101960E94CD6CCE0145960C9408256D
:105B800066EB79E084E291E10E94A36C64E271E14A
:105B9000CE0101960E948F6D44E150E060E070E01C
:105BA000CE0101960E944D58CE0101960E94CD6C07
:105BB0006AE979E0CE0101960E94976D6AE271E18F
:105BC000CE0101960E94266CBC0184E291E10E9404
:105BD000B86CCE0101960E94CD6C64E271E1CE01F9
:105BE00001960E948F6D44E150E06FEF7FEFCE0190
:105BF00001960E941C57CE0101960E94CD6C6BEA63
:105C000079E026CF80913104882309F48CC48091F7
:105C1000B912882329F082E090E00E941A5983C4C7
:105C2000C0901402D0901502E0901602F090170276
:105C300020E030E040E450E4C701B6010E944E9AF3
:105C400018166CF420E030E04AEF54E4C701B601C6
:105C50000E946E970E94F8996B017C0106C030E3A8
:105C6000C32E35E7D32EE12CF12C0E94CC5660E0F8
:105C700080E00E94165F68EB75E08BE292E10E9483
:105C8000046E61E080E00E94165F60EB75E08BE2DD
:105C900092E10E94046E64E670E080E090E00E9471
:105CA000BE490E94F6496093080C7093090C8093DA
:105CB0000A0C90930B0C0E94F6490091080C10916D
:105CC000090C20910A0C30910B0CDC01CB01801BDC
:105CD000910BA20BB30B8C159D05AE05BF050CF007
:105CE00022C483E090E00E941A590E94F64964E1C0
:105CF00070E080E090E00E94BE49DDCF8091B91253
:105D0000811102C00E94CC568091320490913304DC
:105D1000029751F08091390C90913A0C009709F458
:105D200080C1039709F47DC163EE75E084E291E1DF
:105D30000E945E6C64E271E1CE0101960E948F6D5B
:105D400044E150E060E070E0CE0101960E944D58C1
:105D5000CE0101960E94CD6C64ED75E084E291E184
:105D60000E945E6C64E271E1CE0101960E948F6D2B
:105D700044E150E06FEF7FEFCE0101960E941C5787
:105D8000CE0101960E94CD6C87E00E94BE3FBC010F
:105D900080E090E00E940D972AE037ED43EA5CE353
:105DA0000E946E9723E333E948E853E40E949898F1
:105DB0004B015C010E94ED3F6B017C0104E010E0AF
:105DC00020E030E048EC52E4C701B6010E944E9A50
:105DD00018167CF40150110909F4D5C064E670E08E
:105DE00080E090E00E94BE490E94ED3F6B017C0183
:105DF000E7CF21E0B501A401CE0101960E94016D1B
:105E00006CEC79E0CE0145960E94976DBE016F5F04
:105E10007F4FCE0145960E94266CBC018AE291E13B
:105E20000E94B86CCE0145960E94CD6CCE010196C1
:105E30000E94CD6C6AE271E1CE0101960E948F6DE5
:105E400042E350E06FEF7FEFCE0101960E941C57B6
:105E5000CE0101960E94CD6C66ED79E0CE010196EF
:105E60000E94976DCE0101960E94F056CE010196D8
:105E70000E94CD6C65ED79E08AE291E10E944A6C66
:105E800021E0B701A601CE0101960E94016D69E3F0
:105E900079E0CE0145960E94976DBE016F5F7F4FFE
:105EA000CE0145960E94266CBC0180E391E10E94E0
:105EB000B86CCE0145960E94CD6CCE0101960E9431
:105EC000CD6C6AEC79E0CE0101960E94976D60E39B
:105ED00071E1CE0101960E94266CBC0184E291E141
:105EE0000E94B86CCE0101960E94CD6C64E271E113
:105EF000CE0101960E948F6D4AE050E060E070E0B4
:105F0000CE0101960E949757CE0101960E94CD6C5A
:105F100066ED79E0CE0101960E94976DCE01019663
:105F20000E94F056CE0101960E94CD6C65ED79E09D
:105F300080E391E10E944A6C60E371E1CE01019639
:105F40000E948F6D6AEC79E0CE0101960E940F6C81
:105F50006AE271E10E94266CBC018AE291E10E9432
:105F6000B86CCE0101960E94CD6C8091390C909155
:105F70003A0C039709F044C084E090E090933A0C07
:105F80008093390C3DC069EC75E084E291E10E9498
:105F90005E6C64E271E1CE0101960E948F6D4AE071
:105FA00050E060E070E0CE0101960E944D58CE01B5
:105FB00001960E94CD6C6AEB79E0CE0101960E94B9
:105FC000976D64E271E1CE0101960E94266CBC01DE
:105FD0008AE291E10E94B86CCE0101960E94CD6CDC
:105FE0008091390C90913A0C049721F410923A0C5C
:105FF0001092390C81E090E0909333048093320446
:1060000064E670E080E090E00E94BE498091B912A1
:10601000882349F060E273E080E090E00E94BE498E
:1060200002C00E94B2818BEC9DE00E948E6A7BC20E
:106030006EEF75E084E291E10E945E6C64E271E1D2
:10604000CE0101960E948F6D4AE050E060E070E062
:10605000CE0101960E944D58CE0101960E94CD6C52
:106060001091100280912A0C81110DC00E94F649F6
:106070006093260C7093270C8093280C9093290C26
:1060800081E080932A0C80911E0C81110DC00E942A
:10609000F64960931A0C70931B0C80931C0C909320
:1060A0001D0C81E080931E0C1092190C1092180C9C
:1060B0004091180C5091190C5CAF4BAF4832510510
:1060C0000CF087C0812F0E947449EBADFCADEE0F40
:1060D000FF1FE15DF24F918380830E94466020E0C4
:1060E00030E040EA50E40E946E9720E030E040E863
:1060F0005AE30E946E974B015C016093140C7093FD
:10610000150C8093160C9093170CC0900C02D09035
:106110000D02E0900E02F0900F02A701960160912F
:1061200008027091090280910A0290910B020E946C
:1061300098989B01AC0160E070E080EC90E40E94D4
:1061400098982B013C0120E030E0A9010E940997BA
:1061500020E030E040E650E4811105C0C501B40103
:106160000E946E971EC0C501B4010E946E97A701E0
:1061700096010E94999820E030E040E850E40E94A7
:106180009898A30192010E945F9920E030E040ECD2
:1061900050E40E946E9720E030E040E850E40E9416
:1061A00099986093100C7093110C8093120C90933B
:1061B000130C64E170E080E090E00E94BE49EBAC1B
:1061C000FCAC2FEFE21AF20AF092190CE092180CD4
:1061D0006FCFC090100CD090110CE090120CF0908A
:1061E000130C20E030E0A901C701B6010E944E9ACD
:1061F00087FD1EC022E0B701A601CE0101960E94D4
:10620000016D68ED79E0CE0145960E94976DBE0163
:106210006F5F7F4FCE0145960E94266CBC018AE2DB
:1062200091E10E94B86CCE0145960E94CD6C65C18B
:106230006FEE75E08AE291E10E945E6C62C180912E
:106240003104882309F46FC18091B912811127C0EC
:10625000C0901402D0901502E0901602F090170240
:1062600020E030E04AE754E4C701B6010E946E978F
:106270000E94F8994B015C0120E030E040EA50E4D4
:10628000C701B6010E946E9720E030E040EA50E47A
:106290000E9499980E94F899A501940108C021E0F4
:1062A00030E040E050E06AE070E080E090E00E9482
:1062B0006D7D39C180911F0D9091200D0097F1F5F2
:1062C00081E090E09093200D80931F0D6CED79E0BC
:1062D000CE0101960E94976DCE0101960E94EE5864
:1062E000CE0101960E94CD6C65EE79E0CE0101965B
:1062F0000E94976D6FE172E1CE0101960E94266CBB
:10630000BC01CE0145960E948F6D48EC50E06FEFC6
:106310007FEFCE0145960E944D58CE0145960E94D2
:10632000CD6CCE0101960E94CD6C8BEC9DE00E945D
:106330003E7040E052EC61E070E078C0029799F561
:106340001092200D10921F0D6BEE79E0CE01019698
:106350000E94976DCE0101960E94EE58CE010196E3
:106360000E94CD6C69EF79E0CE0101960E94976D95
:106370006FE172E1CE0101960E94266CBC01CE0154
:1063800045960E948F6D48EC50E06FEF7FEFCE0195
:1063900045960E944D58CE0145960E94CD6CCE0187
:1063A00001960E94CD6C80911F0D9091200D019758
:1063B000A9F582E090E09093200D80931F0D6DEF82
:1063C00079E0CE0101960E94976DCE0101960E9460
:1063D000EE58CE0101960E94CD6C6EE07AE0CE01BF
:1063E00001960E94976D6FE172E1CE0101960E94C5
:1063F000266CBC01CE0145960E948F6D48EC50E0A2
:106400006FEF7FEFCE0145960E944D58CE01459625
:106410000E94CD6CCE0101960E94CD6C8BEC9DE06C
:106420000E943E7040E855E260E070E08BEC9DE039
:106430000E94255E1092650C1092640C80E090E042
:106440000E94376263E17AE0CE0101960E94976D67
:1064500069E172E1CE0101960E94266CBC01CE0179
:1064600045960E948F6D40ED57E06FEF7FEFCE01B4
:1064700045960E941C57CE0145960E94CD6C4FC098
:106480008091A70C9091A80C892BA1F481E090E059
:106490009093A80C8093A70C8EED93E09093650CDD
:1064A0008093640C0E94686268EC70E080E090E089
:1064B0000E94BE49E0E0F0E0199535C00E94638378
:1064C0000E94CC560E94C44E2EC0F092340CE09232
:1064D000330C67E076E08AE291E10E945E6C67E54A
:1064E0007BE0CE0101960E94976D4AE050E060E0AB
:1064F00070E0CE0101960E944D58CE0101960E9497
:10650000CD6C6AE271E1CE0101960E948F6D4AE086
:1065100050E06FEF7FEFCE0101960E941C57CE0135
:1065200001960E94CD6C80912E1190912F110097B1
:10653000A9F0419728F4F2E02F1631040CF065C061
:106540006AE271E1CE0101960E948F6DCE01019643
:106550000E949E7CCE0101960E94CD6C64E670E0A4
:1065600080E090E00E94BE4963C066E479E08AE280
:1065700091E10E944A6C0C94D72385E09FE00E9431
:10658000F769892B71F085E09FE00E94D569E1E011
:10659000F0E0EC0FFD1FEE0DFF1D80834FEFE41ABE
:1065A000F40A65E070E080E090E00E94BE4956E0A9
:1065B000E516F10419F599818D8998131FC09A8108
:1065C0008E8998131BC09B818F89981317C02C81CB
:1065D0008D8190E0A0E0B0E0BA2FA92F982F8827F6
:1065E000820F911DA11DB11D480E591E6A1E7B1EF2
:1065F0002BAD3CAD2F5F3F4F3CAF2BAF3FEF831A2E
:10660000930AA30AB30A0C94A1276AE271E1CE01AE
:1066100001960E948F6D4AE050E06FEF7FEFCE0150
:1066200001960E941C57CE0101960E94CD6C88CF26
:10663000C65BDF4F0FB6F894DEBF0FBECDBFDF9154
:10664000CF911F910F91FF90EF90DF90CF90BF906F
:10665000AF909F908F907F906F905F904F903F9002
:106660002F9008952F923F924F925F926F927F9258
:106670008F929F92AF92BF92CF92DF92EF92FF9252
:106680000F931F93CF93DF93CDB7DEB728970FB645
:10669000F894DEBF0FBECDBFFC0182E590E1938789
:1066A000828780914F1090E09587848780911C119C
:1066B00090E09787868780914B10853009F0B7C3AB
:1066C0008091541090915510885891098D359105FD
:1066D00088F480914F10843041F48091561090914D
:1066E00057108097479708F407C280914F10843461
:1066F00008F0E8C180914F108A3108F448C08091B9
:10670000521090915310843F914050F4118610869E
:106710008FEF9FEFDC0184839583A683B78351C0FD
:10672000809154109091551085974B9780F518E5FE
:10673000E12E10E1F12E82E090E040E050E0BA015D
:106740008C010F5F1F4F20914F1030E0021713078D
:106750006CF4970122503109D9012D913C912750B9
:1067600031092730310508F40AC2C801019795950F
:106770008795918780870C971CF41186108607C037
:10678000448355836683778384E090E01CC18091C5
:106790004F108A3108F448C08091521090915310E4
:1067A0008032934008F4B2CF8091541090915510EC
:1067B000C697869708F403C237C04483558366831F
:1067C00077838BE090E0FFC0D7012D913C9125525B
:1067D00031092B31310508F004C2440F551F661FE3
:1067E000771F41600296B4E0EB0EF11C8C010F5F45
:1067F0001F4F20914F1030E00217130764F49701E8
:1068000022503109D9012D913C912C5031092B3066
:106810003105D0F2C80101979595879591878087BA
:106820000C975CF61186108680914F10823208F426
:106830004CC080915410909155100697079708F01E
:1068400044C048E5C42E40E1D42E82E090E040E010
:1068500050E0BA018C010F5F1F4F20914F1030E0C4
:10686000021713070CF5D6011297ED90FC901197C3
:106870009D01BEE1EB1AF108A7E1EA16F10408F068
:10688000BEC1440F551F661F771F4160D6012D9171
:106890003C91B4E0CB0ED11C235031092530310599
:1068A00010F40296D7CFC8010197959587959187E7
:1068B000808740971CF41186108607C04483558357
:1068C000668377838CE090E07EC07F011C821B8210
:1068D00081E090E09A83898380914F108D3008F495
:1068E00075C029E733E0AE014D5F5F4FBE016F5FBA
:1068F0007F4FCF010E94F084892B09F067C029E700
:1069000033E0AE014D5F5F4FBE016F5F7F4FC70148
:106910000E94F084019709F059C029E733E0AE01E5
:106920004D5F5F4FBE016F5F7F4FC7010E94F084D4
:10693000892B09F04BC0812C912C540100E010E010
:1069400080914F1090E029813A81281739077CF512
:1069500029E733E0AE014D5F5F4FBE016F5F7F4FB0
:10696000C7010E94F0846C0129E733E0AE014D5F5E
:106970005F4FBE016F5F7F4FC7010E94F084E1E06F
:10698000CE16D10449F4892B09F5880C991CAA1C50
:10699000BB1C689480F808C0CD28C1F40197B1F4FD
:1069A000880C991CAA1CBB1C0F5F1F4FC9CFD701B5
:1069B00019961C930E931897F70184829582A682EC
:1069C000B78281E090E09183808329C21C821B8280
:1069D00081E090E09A838983D7011C968D919C91E8
:1069E0001D97181619060CF061C01A96ED91FC91CE
:1069F0001B9782E090E09A838983828193818997B3
:106A00004E9708F053C083E090E09A838983848195
:106A100095810B970A9708F049C02CEB31E0AE0145
:106A20004D5F5F4FBE016F5F7F4FC7010E94F084D3
:106A3000892BE1F52CEB31E0AE014D5F5F4FBE01DC
:106A40006F5F7F4FC7010E94F084019779F5412C59
:106A5000512C320100E010E029813A81D7011C96C7
:106A60008D919C911D97281739070CF010C12CEBC4
:106A700031E0AE014D5F5F4FBE016F5F7F4FC701D9
:106A80000E94F0845C010330110509F0C6C02CEBB4
:106A900031E0AE014D5F5F4FBE016F5F7F4FC701B9
:106AA0000E94F084A816B90609F4B7C0D7011A9657
:106AB000ED91FC911B9782819381C697869708F48C
:106AC000F2C03EC1809156109091571082549109A6
:106AD0008E9708F00FCE20E030E0C12CD12C76014B
:106AE000A901485A5F4EDA014D915C914950510914
:106AF0004930510598F0FECD809158109091591071
:106B00000997099708F0F1CD118610868FEF9FEF56
:106B1000DC0184839583A683B7838CC1B901665A4F
:106B20007F4EDB014D915C91475151094231510536
:106B3000C0F4D701C601880F991FAA1FBB1F6C01A3
:106B40007D016894C0F82C5F3F4F2038310541F635
:106B500020E230E031872087C482D582E682F78246
:106B600069C1DB014D915C91465051094730510597
:106B700008F0C0CDCC0CDD1CEE1CFF1CE4CFD7010F
:106B80002D913C91235131092F30310550F4440FA0
:106B9000551F661F771F41600296B4E0EB0EF11C93
:106BA000CFCDD7012D913C912A50310929303105A3
:106BB00008F0EDCD440F551F661F771FEDCF809174
:106BC000561090915710C697869708F02DCE8AE5FB
:106BD000E82E80E1F82E83E090E040E050E0BA013A
:106BE00005CED7012D913C912C5031092A30310529
:106BF00008F01ACE440F551F661F771FF3CDD90139
:106C00002D913C912C5031092B30310508F05DCE8F
:106C1000440F551F661F771F39CE2CEB31E0AE01B4
:106C20004D5F5F4FBE016F5F7F4FC7010E94F084D1
:106C30006C010330110579F42CEB31E0AE014D5FAE
:106C40005F4FBE016F5F7F4FC7010E94F084C8167F
:106C5000D90609F02BCFA114B10459F4CA94CD2858
:106C600009F024CF440C551C661C771C689440F82E
:106C70000BC0AA94AB2809F019CFCD2809F016CF84
:106C8000440C551C661C771C0F5F1F4FE5CE1996F0
:106C90001C930E931897F70144825582668277827F
:106CA00082E090E090CE848195814B97459708F0E3
:106CB00047C0DF0116966F0126ECC20ED11C20E002
:106CC00030E040E050E060E070E080E090E00D9166
:106CD0001C911197095011090830110588F5129679
:106CE0000D911C911397015111090D301105D8F424
:106CF00001E00E94F59B21601496AC15BD0539F7A3
:106D0000F701248335834683578300E20E94109C59
:106D10002283338385E090E09183808380E390E059
:106D2000918780877CC012960D911C911397045017
:106D300011090530110520F401E00E94F59BDCCF1C
:106D400080914F10893340F0828193818957910956
:106D50008335910508F47CC180914F10823209F48B
:106D60006CC082819381895791098335910508F41C
:106D7000E6C1828193818C549109C59708F064C063
:106D800080914F10843031F48481958180974797AA
:106D900008F434C280914F10843408F455C08481C3
:106DA000958189549109C39708F04EC09F012A5FCD
:106DB0003F4FAF014A575F4F812C912C5401D901AD
:106DC0006D917C916950710969307105E8F5D901BF
:106DD00012966D917C91139766517109613171051D
:106DE00008F022C2D501C401880F991FAA1FBB1F3A
:106DF0004C015D01689480F82C5F3F4F24173507E4
:106E0000F1F620E230E0F70131872087D701848254
:106E10009582A682B78287E090E08D939C9381E073
:106E200090E0BFC282E080934B1010924F1080E040
:106E300090E0B7C283E090E0C6CD828193810A974B
:106E4000099708F460C18DCF80914F10863460F1AE
:106E5000828193810C970B9708F4F6C125C0D90164
:106E600012966D917C9113976E517109673171057E
:106E700008F01EC2D501C401880F991FAA1FBB1FAD
:106E80004C015D01689480F84E5F5F4F2C5F3F4F6F
:106E90004534510509F4F3C1D9016D917C916C50D1
:106EA00071096B307105D8F280914F10883578F1F7
:106EB00082819381855891098B35910508F408C228
:106EC00026C0BC016F5F7F4FD8012D913C912750A8
:106ED00031092730310508F00AC2440F551F4160BF
:106EE00002960C5F1F4F20914F1030E02450310963
:106EF000821793070CF004C2980122503109D9017E
:106F00002D913C912950310928303105D0F28091E2
:106F10004F108032E1F48281938106970697B8F48E
:106F2000848195810997099790F49F012A5F3F4FCB
:106F3000AF01425C5F4F812C912C5401D9016D91BE
:106F40007C91665071096630710508F4F3C1D70170
:106F50001C962D903C901D97B6E02B1631040CF436
:106F600061CF8F010A5F1F4F73E0C72ED12CE5EC74
:106F70008E2EEDE99E2EECE1AE2EE1E8BE2EF8015C
:106F80006081718134976080718080E090E00E9420
:106F90000D976D837E838F839887B30180E090E0A7
:106FA0000E940D972B013C012DEC3CEC4CE45FE37F
:106FB0000E946E979B01AC016D817E818F819885C7
:106FC0000E94099787FD19C02DEC3CEC4CE45FE36F
:106FD0006D817E818F8198850E946E979B01AC01A7
:106FE000C301B2010E940997E82F880FFF0BEE271B
:106FF000FF0FEE1FFF27319602C0E0E0F0E0A50191
:10700000940163E971E080E091E00E94B79B4F0139
:10701000FF0FAA08BB0886269726A826B926FFEFE9
:10702000CF1ADF0A0E5F1F4FC214D30409F0A7CF97
:10703000D70114968D929D92AD92BC92179780E2E3
:1070400090E019969C938E9318978FEF9FEFE5CE63
:1070500084819581CA97899708F07ECE9F012A5F27
:107060003F4F812C912C540143E050E0D9016D91A8
:107070007C916A5071096930710508F06DCED901B3
:1070800012966D917C91139766517109613171056A
:1070900050F5D501C401880F991FAA1FBB1F4C01D1
:1070A0005D01689480F84E5F5F4F2C5F3F4F4B331C
:1070B0005105E1F69F012A583F4FD9012D913C918E
:1070C0002A5031092930310508F046CE2CE130E054
:1070D000F70131872087D70184829582A682B78203
:1070E0008AE090E09ACED90112966D917C91139727
:1070F000665071096730710508F02ECE880C991C16
:10710000AA1CBB1CD0CF20914F10CF01820F911D24
:10711000820F911DDC0112978D919C910A9709971E
:1071200008F01FCEF701118610868FEF9FEFDC016C
:1071300084839583A683B78386E090E044CC8091D6
:107140004F10813208F415CE84819581CA978997B2
:1071500008F00FCE9F012A5F3F4F812C912C5401E4
:1071600043E050E0D9016D917C916A50710969301A
:10717000710508F0FECDD90112966D917C9113979F
:10718000665171096131710570F112966D917C91B2
:107190001397665071096730710508F0EACD880CC5
:1071A000991CAA1CBB1C4E5F5F4F2C5F3F4F4332A4
:1071B0005105C1F69F012A5B3F4FD9012D913C91AA
:1071C0002A5031092930310508F0D3CD20E130E0D3
:1071D000F70131872087D70184829582A682B78202
:1071E00086E090E01ACED501C401880F991FAA1F2E
:1071F000BB1F4C015D01689480F8D5CF86819781D3
:107200000997099708F0C6CDD70119961C921E92CE
:1072100018978FEF9FEFDC01F70184839583A68396
:10722000B78387E090E0CFCBD90112966D917C9126
:107230001397665071096730710508F005CE880C08
:10724000991CAA1CBB1CD8CD8481958109970997EC
:1072500008F02ACE868197818C974F9708F024CE2C
:107260008085918589974D9708F01ECE9F01265FF6
:107270003F4F812C912C540145E050E00DCE9F01F1
:1072800026573F4FD9012D913C912C5031092B307D
:10729000310508F009CE20E230E0F7013187208780
:1072A000D70184829582A682B78288E090E0B5CD2E
:1072B000D90112966D917C911397695071096930CB
:1072C000710508F0F1CD880C991CAA1CBB1CDCCD03
:1072D00084819581825491098E9708F018CE8F0190
:1072E000045C1F4F8DE190E040E050E0FCCDD80100
:1072F0002D913C912851310922313105C0F0CB014B
:10730000019795958795D70119969C938E93189719
:107310008A970CF4FCCD052E000C660B770BF70159
:10732000448355836683778389E090E04CCB440F98
:10733000551FD6CDD90112966D917C911397695145
:10734000710963317105E8F4D501C401880F991FF3
:10735000AA1FBB1F4C015D01689480F82C5F3F4F52
:107360002417350709F0EACD2EE030E0F701318728
:107370002087D70184829582A682B7828FE090E031
:107380004CCDD90112966D917C911397695071097A
:107390006930710508F0DBCD880C991CAA1CBB1C58
:1073A000DDCF28960FB6F894DEBF0FBECDBFDF91BC
:1073B000CF911F910F91FF90EF90DF90CF90BF90F2
:1073C000AF909F908F907F906F905F904F903F9085
:1073D0002F9008954F925F926F927F928F929F921B
:1073E000AF92BF92DF92EF92FF920F931F93CF93D2
:1073F000DF93CDB7DEB7A9970FB6F894DEBF0FBE07
:10740000CDBFD82E882351F080913B0C882331F0DA
:1074100067E57BE082EA9FE00E94D56E0E942060D3
:1074200060E08DE20E94A74360E18DE20E94A743E5
:1074300068E08DE20E94A74340909411509095110E
:10744000609096117090971149825A826B827C826B
:107450008090981190909911A0909A11B0909B11E2
:107460008D829E82AF82B88680919C1190919D11F1
:10747000A0919E11B0919F118EA39FA3A8A7B9A719
:1074800089879A87AB87BC87DD20A1F180913B0C6F
:10749000882381F17E019DE0E90EF11C68EF79E01F
:1074A000C7010E94876DC7010E94EE58C7010E9464
:1074B000CD6C8E010F5F1F4FD8016D917D918D9125
:1074C0009D918D0146E050E00E941F606AEC79E0DA
:1074D00082EA9FE00E94F56E0E151F0569F767E5C9
:1074E0007BE0C8010E94976DC8010E94EE58C80158
:1074F0000E94CD6C23E938E144E85FE3C301B201A7
:107500000E946E972B013C016D877E878F87988B39
:1075100022E430E645E85FE3C501B4010E946E97BE
:107520004B015C01698B7A8B8B8B9C8B25E83BEE46
:1075300041E95FE36EA17FA188A599A50E946E979E
:107540006D8B7E8B8F8B988F4092941150929511FA
:107550006092961170929711809298119092991161
:10756000A0929A11B0929B1160939C1170939D11FF
:1075700080939E1190939F11DD2009F4A7C0809104
:107580003B0C882309F4A2C07E01B9E1EB0EF11C8B
:107590006BEE79E0C7010E94876DC7010E94EE582B
:1075A000C7010E94CD6C8E01035F1F4FF8016191EE
:1075B0007191819191918F0142E050E00E941F6092
:1075C0006AEC79E082EA9FE00E94F56E0E151F05D5
:1075D00069F767E57BE0C8010E94976DC8010E94CA
:1075E000EE58C8010E94CD6C40EA51E166E070E0BF
:1075F00082E30E943D438090A111912C982C882415
:107600008091A011882AA090A311B12CBA2CAA2491
:107610008091A211A82AE090A511F12CFE2CEE2455
:107620008091A411E82A6EED79E082EA9FE00E9441
:10763000046E4AE050E0B40182EA9FE00E94CC6E02
:107640006AEC79E082EA9FE00E94F56E4AE050E041
:10765000B50182EA9FE00E94CC6E6AEC79E082EA92
:107660009FE00E94F56E4AE050E0B70182EA9FE099
:107670000E94CC6E67E57BE082EA9FE00E94D56EB7
:10768000C8010E94FB4365ED79E082EA9FE00E9419
:10769000046E7E01F5E2EF0EF11CD8016D917D9133
:1076A0008D919D918D014AE050E00E941F606AEC2F
:1076B00079E082EA9FE00E94F56E0E151F0569F7DA
:1076C00067E57BE082EA9FE00E94D56E61E08DE194
:1076D0000E94A743DD20A1F080913B0C882381F01C
:1076E00061EC79E082EA9FE00E94046EAE014B5D9E
:1076F0005F4F61E070E08DE1C0D78DA190E0F7D7DA
:1077000062E08EE10E94A74363E08FE10E94A743FD
:1077100064E080E20E94A743DD2009F44DC080911F
:107720003B0C882309F448C065EA79E082EA9FE0CF
:107730000E94046EAE014B5D5F4F61E070E08EE130
:107740009CD7ADA0B12CAE014B5D5F4F61E070E006
:107750008FE193D7EDA0F12CAE014B5D5F4F61E05F
:1077600070E080E28AD70DA110E04AE050E0B50158
:1077700082EA9FE00E94CC6E6AEC79E082EA9FE0A8
:107780000E94F56E4AE050E0B70182EA9FE00E9455
:10779000CC6E6AEC79E082EA9FE00E94F56E4AE0E6
:1077A00050E0B80182EA9FE00E94CC6E67E57BE082
:1077B00082EA9FE00E94D56E65E081E2C8D7DD20B5
:1077C000A1F080913B0C882381F062E979E082EAA4
:1077D0009FE00E94046EAE014B5D5F4F61E070E080
:1077E00081E24BD78DA190E082D766E082E2AFD7ED
:1077F000DD20A1F080913B0C882381F06AE779E0DD
:1078000082EA9FE00E94046EAE014B5D5F4F61E033
:1078100070E082E232D78DA190E069D767E083E221
:1078200096D7DD20A1F080913B0C882381F064E69F
:1078300079E082EA9FE00E94046EAE014B5D5F4FEB
:1078400061E070E083E219D78DA190E050D768E045
:1078500084E27DD7DD20A1F080913B0C882381F06C
:107860006CE479E082EA9FE00E94046EAE014B5D19
:107870005F4F61E070E084E200D78DA190E037D7E0
:1078800069E085E264D7DD20A1F080913B0C88237C
:1078900081F062E379E082EA9FE00E94046EAE012B
:1078A0004B5D5F4F61E070E085E2E7D68DA190E02F
:1078B0001ED76AE086E24BD7DD20A1F080913B0C19
:1078C000882381F06CE179E082EA9FE00E94046EF7
:1078D000AE014B5D5F4F61E070E086E2CED68DA1D8
:1078E00090E005D76BE088E232D7DD20A1F08091EF
:1078F0003B0C882381F063E079E082EA9FE00E94FC
:10790000046EAE014B5D5F4F61E070E088E2B5D67A
:107910008DA190E0ECD66CE089E219D7DD2009F466
:1079200069C080913B0C882309F464C06BEE78E059
:1079300082EA9FE00E94046EAE014B5D5F4F61E002
:1079400070E089E29AD68DA190E0D1D664ED78E01E
:1079500082EA9FE00E94046E66E070E087E2DDD676
:1079600090E0C5D66DEB78E082EA9FE00E94046E5D
:1079700065E070E087E2D1D690E0B9D666EA78E0BB
:1079800082EA9FE00E94046E64E070E087E2C5D660
:1079900090E0ADD66DE878E082EA9FE00E94046E48
:1079A00062E070E087E2B9D690E0A1D664E778E0C3
:1079B00082EA9FE00E94046E61E070E087E2ADD64B
:1079C00090E095D66BE578E082EA9FE00E94046E35
:1079D00060E070E087E2A1D690E089D66AE478E0C2
:1079E00082EA9FE00E94046E63E070E087E295D631
:1079F00090E07DD641E067E070E087E2BDD641E0EF
:107A000063E070E087E2B8D641E063E070E08AE2CC
:107A1000B3D6DD2081F080913B0C882361F061E3D7
:107A200078E082EA9FE00E94046E63E070E08AE200
:107A300074D690E05CD640E063E070E08AE29CD6C9
:107A4000DD2081F080913B0C882361F067E178E0D4
:107A500082EA9FE00E94046E63E070E08AE25DD6F5
:107A600090E045D641E062E070E08AE285D6DD2014
:107A700081F080913B0C882361F06BEF77E082EA24
:107A80009FE00E94046E62E070E08AE246D690E0D9
:107A90002ED640E062E070E08AE26ED6DD2081F012
:107AA00080913B0C882361F06EED77E082EA9FE0E5
:107AB0000E94046E62E070E08AE22FD690E017D652
:107AC00041E061E070E08AE257D6DD2081F08091EC
:107AD0003B0C882361F062EC77E082EA9FE00E9431
:107AE000046E61E070E08AE218D690E000D640E0D3
:107AF00061E070E08AE240D6DD2081F080913B0CAD
:107B0000882361F065EA77E082EA9FE00E94046ED4
:107B100061E070E08AE201D690E0E9D541E060E002
:107B200070E08AE229D6DD2081F080913B0C882329
:107B300061F069E877E082EA9FE00E94046E60E00D
:107B400070E08AE2EAD590E0D2D540E060E070E0F3
:107B50008AE212D6DD2081F080913B0C882361F00F
:107B60006CE677E082EA9FE00E94046E60E070E0DD
:107B70008AE2D3D590E0BBD541E066E070E087E2D1
:107B8000FBD541E065E070E087E2F6D541E064E0D6
:107B900070E087E2F1D540E062E070E087E2ECD58A
:107BA00040E061E070E087E2E7D540E060E070E04F
:107BB00087E2E2D5DD2009F465C080913B0C882383
:107BC00009F460C064E577E082EA9FE00E94046EF9
:107BD00066E070E08BE2A1D590E089D566E377E0BE
:107BE00082EA9FE00E94046E65E070E08BE295D52A
:107BF00090E07DD568E177E082EA9FE00E94046E24
:107C000064E070E08BE289D590E071D56FEF76E0AB
:107C100082EA9FE00E94046E62E070E08BE27DD514
:107C200090E065D566EE76E082EA9FE00E94046E01
:107C300061E070E08BE271D590E059D56DEC76E0B3
:107C400082EA9FE00E94046E60E070E08BE265D5FE
:107C500090E04DD56AEB76E082EA9FE00E94046EE8
:107C600063E070E08BE259D590E041D565EA76E0BB
:107C700082EA9FE00E94046E64E070E08CE24DD5E1
:107C800090E035D540E064E070E08CE275D5AE015F
:107C90004B5D5F4F61E070E08CE2EFD46DA1607FDF
:107CA00066608CE254D5DD2009F45EC080913B0C07
:107CB000882309F459C061E976E082EA9FE00E94D6
:107CC000046EAE014B5D5F4F61E070E08CE2D5D495
:107CD0006DA16F7070E066507109072E000C880B63
:107CE000990B0E940F979B01AC0160E070E080E06F
:107CF00090E40E940D9B20E030E048EC50E40E94AC
:107D00006E976AD56AE776E082EA9FE00E94046E89
:107D1000AE014B5D5F4F61E070E080E3AED44DA1FA
:107D200050E060E070E02AE082EA9FE00E943D6E51
:107D300082EA9FE00E94D26E62E676E082EA9FE0ED
:107D40000E94046E61E070E080E3E7D490E0CFD45D
:107D500069E476E082EA9FE00E94046E61E070E0F0
:107D60008FE2DBD490E0C3D441E061E070E08FE2C9
:107D700003D5DD2081F080913B0C882361F061E325
:107D800076E082EA9FE00E94046E61E070E08EE29D
:107D9000C4D490E0ACD441E061E070E08EE2ECD479
:107DA00040E067E070E081E3E7D4DD2009F451C0F2
:107DB00080913B0C882309F44CC06EE176E082EAA6
:107DC0009FE00E94046E67E070E081E3A6D490E03B
:107DD0008ED468E17AE082EA9FE00E94F56EAE01FF
:107DE0004B5D5F4F61E070E080E047D48DA10E9461
:107DF0005D6567E57BE082EA9FE00E94D56E0DE15C
:107E000010E064E47AE082EA9FE00E94F56E40E1CF
:107E100050E0B80182EA9FE00E94CC6E6DE678E007
:107E200082EA9FE00E94F56EAE014B5D5F4F61E01C
:107E300070E0802F22D48DA10E945D6567E57BE014
:107E400082EA9FE00E94D56E0F5F1F4F0A33110533
:107E5000C1F6A9960FB6F894DEBF0FBECDBFDF9175
:107E6000CF911F910F91FF90EF90DF90BF90AF9057
:107E70009F908F907F906F905F904F90089596E0C5
:107E8000899FD0011124AA55BE4E90967C936E9383
:107E90005F9791E091969C93919790911212E09147
:107EA0001312F0911412992339F0309751F0811187
:107EB00008C08091C21104C0309719F05C968C9173
:107EC000199408950F931F93CF93DF93C82FD62F44
:107ED00086E0C89FF0011124EA55FE4E11A2878D5D
:107EE00090A181309105E9F01CF4892B49F041C043
:107EF00082309105A1F10397E1F560E070E033C0B5
:107F00006623B9F161E070E08C2FB9DF0E94F64979
:107F10006093FE117093FF118093001290930112F1
:107F200028C00E94F6490091FE111091FF11209186
:107F3000001230910112AB01BC01401B510B620BCE
:107F4000730B8091101290911112A0E0B0E0841791
:107F50009507A607B70718F462E070E004C0D111D6
:107F600008C063E070E08C2FDF91CF911F910F91DB
:107F700086CFDF91CF911F910F9108950F931F939B
:107F8000CF93DF931F92CDB7DEB7682F8091181281
:107F900069830E94FB5E69818FE390E10E942964FE
:107FA00080E00E94985E63E0809118120E949363C3
:107FB0008FE390E10E94DE638C018FE390E10E94E9
:107FC000DE6320E030E0382FC901802B912B0F9029
:107FD000DF91CF911F910F91089586E0CFDFBC0113
:107FE00080E090E00E940D972AE037ED43EA5CE3E1
:107FF0000E946E9723E333E948E853E40C94989881
:108000000895613208F060E20E944F631092800D83
:1080100080937F0D08951F93CF93DF931F92CDB769
:10802000DEB7682F87E769830E94FB5E69818FE373
:1080300090E10E9429640E94F55E87E70E94FB5E42
:1080400061E070E087E790E0DCDF8FE390E10E9481
:10805000DE63182F0E94F55E812F0F90DF91CF9184
:108060001F9108950F931F93CF93DF931F92CDB766
:10807000DEB7682F87E769830E94FB5E69818FE323
:1080800090E10E9429640E94F55E87E70E94FB5EF2
:1080900062E070E087E790E0B4DF8FE390E10E9458
:1080A000DE6300E010E0182F8FE390E10E94DE63B2
:1080B000082B192B0E94F55EC8010F90DF91CF911C
:1080C0001F910F91089587E70E94FB5E64EF8FE395
:1080D00090E10E9429646EE28FE390E10E9429649E
:1080E0000E94F55E65E070E080E090E00E94BE498D
:1080F00086EFB8CF3F924F925F926F927F928F92AE
:108100009F92AF92BF92CF92DF92EF92FF920F9326
:108110001F93CF93DF93CDB7DEB728970FB6F894B0
:10812000DEBF0FBECDBFCFDF6C01E12CF12C109173
:1081300048111295110F110F107C1C5C87E70E94EB
:10814000FB5E64EF8FE390E10E942964612F8FE36F
:1081500090E10E9429640E94F55E8091481181118E
:1081600005C065E070E080E090E012C0813029F445
:1081700068E070E080E090E00BC0823029F46EE0AF
:1081800070E080E090E004C06AE170E080E090E0A0
:108190000E94BE4986EF66DF4C01A12CB12CBA2C9F
:1081A000A92C982C882488EF36DF882A3090481133
:1081B00080915D1190915E11A7019601281B390BEA
:1081C00041095109A0915B11B0915C110E9457982F
:1081D0006B017C01AFE0F594E794D794C794AA951E
:1081E000D1F76091551170915611CB01770FAA0B01
:1081F000BB0BBC01CD01BBE0660F771F881F991F29
:10820000BA95D1F720915711309158118901330F48
:10821000220B330BA90198012C0D3D1D4E1D5F1D36
:108220000E943B98C20ED31EE41EF51E20EAC21A1D
:108230002FE0D20AE108F108A7019601C701B601B3
:108240000E94B79B9B01AC011CE055954795379563
:1082500027951A95D1F729833A834B835C83009144
:10826000491110914A11A0914D11B0914E11A701E1
:1082700096010E9461982B013C018DE075946794F2
:10828000579447948A95D1F7A0914F11B09150110E
:1082900029813A814B815C810E946198BB2797FDBF
:1082A000B095AB2F840D951DA61DB71D0296A11D7F
:1082B000B11D32E0B595A795979587953A95D1F779
:1082C0009C01AD0130584F4F5F4FA0915911B091B3
:1082D0005A110E9457982B013C014FE07694679405
:1082E000579447944A95D1F788E090E08319910913
:1082F000A501940104C056954795379527958A9511
:10830000D2F72D833E834F8358874801110FAA0867
:10831000BB0852E0880C991CAA1CBB1C5A95D1F7CB
:10832000A0915111B091521129813A814B815C8108
:108330000E9461989B01AC016BE05595479537957C
:1083400027956A95D1F729833A834B835C83A09163
:108350004B11B0914C11A70196010E946198DC016C
:10836000CB017BE0B595A795979587957A95D1F741
:1083700029813A814B815C81820F931FA41FB51F15
:10838000880D991DAA1DBB1D032C04C0880F991FC1
:10839000AA1FBB1F0A94D2F7BC01CD016E5F7F4FAD
:1083A0008F4F9F4F24E030E040E050E00E943B9828
:1083B0008D819E81AF81B885821B930BA40BB50B79
:1083C0009C01AD0180E593ECA0E0B0E0BC01CD01E3
:1083D00004C096958795779567953A94D2F70E9451
:1083E000B79B97FD0BC0660F771F881F991FA301CE
:1083F00092010E94679869017A010AC0A301920163
:108400000E94679869017A01CC0CDD1CEE1CFF1CF0
:108410009927F7FC9A958F2D7E2D6D2D9B01AC0130
:108420000E94B79B9B01AC01AEEDBBE00E94579848
:108430004C01BB2497FCB094AB2CA3E4B3EEA70192
:1084400096010E946398BB2797FDB095AB2F880DCE
:10845000991DAA1DBB1D8153914FAF4FBF4F44E0E3
:10846000B595A795979587954A95D1F7BC01CD010C
:108470006C0D7D1D8E1D9F1D28960FB6F894DEBFD6
:108480000FBECDBFDF91CF911F910F91FF90EF9065
:10849000DF90CF90BF90AF909F908F907F906F9024
:1084A0005F904F903F900895CF92DF92EF92FF92AE
:1084B0000F931F9308DEAC0160E070E0E8E4F1E1A7
:1084C000858996899A01AB01281B390B410951090D
:1084D000A389B4890E9457986B017C018FE0F594C1
:1084E000E794D794C7948A95D1F765857685CB01B3
:1084F000770FAA0BBB0BBC01CD012BE0660F771FDA
:10850000881F991F2A95D1F7278530898901330F54
:10851000220B330BA90198012C0D3D1D4E1D5F1D33
:108520000E943B98D701C601820F931FA41FB51F5D
:108530000896A11DB11DBC01CD0134E0959587952C
:10854000779567953A95D1F70E940F9720E030E034
:1085500040E251E40E945F991F910F91FF90EF90CC
:10856000DF90CF9008958F929F92AF92BF92EF923B
:10857000FF920F931F93CF93DF93D82FC62F1092A4
:108580008C1110928D1110928E1110928F111092E9
:10859000901161E06AD660E08D2F35D66C2F70E0C7
:1085A00080E090E0EBD660E08D2F5FD68BE990E025
:1085B0000197F1F700E911E08D2FFBD5892B31F4FC
:1085C00001501109C9F78EEF9FEF4CC000E911E08F
:1085D0008D2FEFD5019721F401501109C9F7F3CF81
:1085E00018E2C0E800E020E9E22EFF24F3948D2F8A
:1085F000E0D5892B29F481E0E81AF108C1F7E3CF2F
:1086000098D64B015C0190E9E92EFF24F3948D2F5D
:10861000D0D5019729F481E0E81AF108C1F7D3CF4A
:1086200088D6DC01CB0188199909AA09BB09899769
:10863000A105B10538F0E02FF0E0EC57FE4E808543
:108640008C2B80872C2F30E035952795211531050F
:1086500011F0C22F02C00F5FC0E8115009F0C3CF64
:1086600080E090E0DF91CF911F910F91FF90EF900C
:10867000BF90AF909F908F900895EF92FF920F93CD
:108680001F93CF93DF93C82F8B017A0183E50E945C
:10869000FB5E6C2F8FE390E10E9429640E94F55EDF
:1086A00083E50E94FB5EB80183E590E0AADCE70168
:1086B000CE018E199F0930917F0D2091800D3217C8
:1086C00031F08FE390E10E94DE638993F1CF801750
:1086D000910729F01092921181E080939311DF911C
:1086E000CF911F910F91FF90EF900C94F55ECF9377
:1086F000DF93AC01990F660B770B2AE030E082EA3A
:108700009FE00E94856EEC0182EA9FE00E94D26E9B
:108710008C0F9D1FDF91CF9108951F93CF93DF930F
:108720001F92CDB7DEB7162FAE014F5F5F4F61E0EE
:1087300070E0A3DF898190E002C0959587951A9536
:10874000E2F781700F90DF91CF911F910895CF9341
:10875000DF93D82FC62F83E50E94FB5E6D2F8FE33A
:1087600090E10E9429646C2F8FE390E10E942964BC
:10877000DF91CF910C94F55EFF920F931F93CF93EF
:10878000DF931F92CDB7DEB7182F062FF42EAE0160
:108790004F5F5F4F61E070E070DF8981FF2049F03B
:1087A00041E050E001C0440F0A95EAF7482B4983A5
:1087B00009C021E030E001C0220F0A95EAF72095B8
:1087C000282329836981812FC2DF0F90DF91CF9108
:1087D0001F910F91FF900895CF93DF9342E00E9485
:1087E000415FEC0182EA9FE00E94D26E8C0F9D1FD8
:1087F000DF91CF910895AF92BF92CF92DF92EF9227
:10880000FF921F93CF93DF93CDB7DEB72A970FB6B2
:10881000F894DEBF0FBECDBF182F40EA51E166E0ED
:1088200070E082E39F8329DF2091A11130E0322F95
:1088300022278091A011282B3A8329832091A3110C
:1088400030E0322F22278091A211282B3C832B83EA
:108850002091A51130E0322F22278091A411282BDE
:108860003E832D839E012F5F3F4F590154E9C52E52
:1088700051E1D52EE12E9F81F92EF5016191719183
:108880005F01F60121913191419151916F01072EC4
:10889000000C880B990B2F83388749875A870E94D1
:1088A0000F972F81388549855A850E946E97F70169
:1088B00061937193819391937F01F0EACF16F1E177
:1088C000DF06D9F62A960FB6F894DEBF0FBECDBFED
:1088D000DF91CF911F91FF90EF90DF90CF90BF90ED
:1088E000AF900895AF92BF92CF92DF92EF92FF9236
:1088F0000F931F93CF93DF931F92CDB7DEB75C0129
:10890000D62EE72EFC018585811104C0C501BFD696
:10891000811106C0F50113861586148680E061C0BA
:1089200040E060EFC50147D601E0F12CC12C11E019
:10893000C501EED5682FC5016983EAD5698161302B
:1089400019F48130B9F432C04F2D50E068131BC0C8
:10895000F5018385181730F4E40FF51F8381802318
:1089600049F402C0181731F060E0193058F4F501ED
:10897000148708C0F501EF0DF11D8381802B8383DF
:1089800061E009C0C12EF501E40FF51F9381802F2E
:10899000809589238383C501DFD51F5F000F11F404
:1089A000F39401E0F7E0FF1508F0C2CF113408F4AA
:1089B000B1CFF501C386C11002C081E08587F50102
:1089C0008381882309F4A6CFD5011396ED2DFE2DC2
:1089D0009501255F3F4F8D918193A217B307D9F77A
:1089E00081E00F90DF91CF911F910F91FF90EF9059
:1089F000DF90CF90BF90AF9008959F92AF92BF92BB
:108A0000CF92DF92EF92FF920F931F93CF93DF935A
:108A1000CDB7DEB761970FB6F894DEBF0FBECDBFFE
:108A20008C018CE0F8018183C12CD12C2FE5E22E42
:108A30003FE7B32E4FE1A42E5FE3952EF80184812A
:108A400090E0C816D9060CF093C04C2DBE01665FAD
:108A50007F4FC80121D5F8018181893038F0F82E87
:108A6000FCE0F81728F49CE0F92E02C089E0F82E0B
:108A70008A85803131F0BE01665F7F4FC8010FD714
:108A800001C08CE08F1509F46FC0AE014F5F5F4FDE
:108A9000BE01665F7F4FC80199D6882309F464C080
:108AA0008A85803109F460C08BE0F81651F0ECE063
:108AB000FE1629F0FAE0FF1206C09D8205C0BD82B5
:108AC00003C0ED8201C0AD82F80186819781DFD5B8
:108AD000BE01665F7F4FF80186819781ADD540E08A
:108AE0006EE4F8018681978166D540E06B81F801DC
:108AF0008681978160D540E06C81F80186819781FD
:108B00005AD58A85803131F040E06D81F801868147
:108B1000978151D5F80186819781B9D5BE01665FED
:108B20007F4FF8018681978187D5F801408168E4FD
:108B30008681978140D564E170E080E090E01ED4AA
:108B4000F8018081882329F06AE070E080E090E0FD
:108B500015D4F801868197819AD5F8018181F8169C
:108B600008F4F82EF801F182FFEFCF1ADF0A66CF82
:108B700061960FB6F894DEBF0FBECDBFDF91CF91E7
:108B80001F910F91FF90EF90DF90CF90BF90AF902B
:108B90009F9008956F927F928F929F92AF92BF9213
:108BA000CF92DF92EF92FF920F931F93CF93DF93B9
:108BB00081E0809312121AD40091021210910312D4
:108BC0002091041230910512AB01BC01401B510BE6
:108BD000620B730B80910E1290910F12A0E0B0E027
:108BE00084179507A607B70708F003C1C0E0809176
:108BF0000C12C81758F4E0910812F0910912EC0F0A
:108C0000F11D62E0808131D3CF5FF1CF712C812CD7
:108C1000912C5401839480910D12781608F05AC05B
:108C2000072D10E0E0910A12F0910B12E00FF11FF6
:108C300061E080811AD3E0910A12F0910B12E00FEB
:108C4000F11F60E08081DFD2D501C401072C04C090
:108C5000880F991FAA1FBB1F0A94D2F76C017C01D1
:108C6000E094F094612C80910C126816F0F4C62DFB
:108C7000D0E0E0910812F0910912EC0FFD1F808105
:108C800098D22496CC0FDD1FCA55DE4E892B29F4CD
:108C9000888199818C299D2904C0888199818E21A0
:108CA0009F21998388836394DECFE0910A12F0912B
:108CB0000B12E00FF11F61E08081A5D280910A12B2
:108CC00090910B12FC01E00FF11F60E08081CDD28A
:108CD0007394A1CFE2ECF1E18FEF9FEF2381348118
:108CE000232B21F41082928381831582369621E111
:108CF000EE3FF20799F710E096E0F92E80910C1202
:108D0000181708F051C000E0C12FD0E0CC0FDD1FD4
:108D1000C255DE4E20910D12021708F043C0688143
:108D20007981002E02C0769567950A94E2F761700A
:108D30007727129F90011124200F311DE091061218
:108D4000F0910712E20FF31F4081E6EAF1E180E0C3
:108D5000A58DB68DA217B30711F461701AC08F5F8D
:108D600036968A30A9F7672BD9F0E2ECF1E180E082
:108D700090E0508151110FC0F89EF001F99EF00D66
:108D80001124EA55FE4E448F368F258F10A2178E80
:108D900061E098D805C0019636968A30910549F76A
:108DA0000F5FB8CF1F5FAACF80E090E0C0E0FC016A
:108DB000EA55FE4E21A12111C1E006968C339105A2
:108DC000B1F714D3609302127093031280930412CC
:108DD00090930512CC2369F08091C711882349F044
:108DE0008091C5119091C611019719F48091C2111B
:108DF00003C01092121280E0DF91CF911F910F916A
:108E0000FF90EF90DF90CF90BF90AF909F908F90AA
:108E10007F906F9008950F931F93CF93DF93FC0182
:108E2000248135812115310519F4FB01108211C00F
:108E3000EA0121972C173D0708F4E9018B01FC0199
:108E400060817181AE01C8010E94799EC00FD11F5F
:108E50001882DF91CF911F910F91089590E0FC014E
:108E60003197E231F10508F04EC08827E955FF4FF0
:108E70008F4F0C94ED9B809180008F7703C0809181
:108E800080008F7D80938000089580918000877F8F
:108E9000F9CF84B58F7702C084B58F7D84BD0895E6
:108EA0008091B0008F7703C08091B0008F7D809358
:108EB000B0000895809190008F7707C08091900056
:108EC0008F7D03C080919000877F809390000895EC
:108ED0008091A0008F7707C08091A0008F7D03C094
:108EE0008091A000877F8093A00008958091200149
:108EF0008F7707C0809120018F7D03C08091200172
:108F0000877F809320010895DC0180E0615090F01C
:108F10009D919827E92FEF70F0E0EC53F54F2491E5
:108F200092959F70E92FF0E0EC52F54FE4918E2F6F
:108F30008227ECCF08950F931F93CF93DF938C017B
:108F4000EB0188E2FB0111928A95E9F74BE050E0D2
:108F500063ED7AE0CE010E94799E1B8681E090E06D
:108F6000A0E0B0E08C879D87AE87BF87F801858938
:108F70009689A789B08D888B998BAA8BBB8B82E051
:108F800090E0A0E0B0E08C8B9D8BAE8BBF8B1CA2E1
:108F90001DA21EA21FA280E090E0A8E4B4E4888F86
:108FA000998FAA8FBB8F80E090E0A8E4B4EC8C8FFF
:108FB0009D8FAE8FBF8F8DEC9CECACE4BEE388A39D
:108FC00099A3AAA3BBA3DF91CF911F910F910895FD
:108FD0004F925F926F927F928F929F92AF92BF92C9
:108FE000CF92DF92EF92FF920F931F93CF93DF9375
:108FF0008C01EB0184E2FB0111928A95E9F78EE185
:109000000E94FB5E83E090E00E94F75E0E94F55EA6
:1090100066E08EE10E94936380917F0D90E0209145
:10902000800D821B910986309105ECF38FE390E16E
:109030000E94DE63882E8FE390E10E94DE63982E0B
:109040008FE390E10E94DE63682E8FE390E10E943F
:10905000DE63782E8FE390E10E94DE63482E8FE37B
:1090600090E10E94DE63582EB82CA12CB50169292D
:10907000072E000C880B990B0E940F974B015C0187
:10908000F8016583768387839087D42CC12CB60141
:109090006529072E000C880B990B0E940F97F80189
:1090A0006187728783879487F62CE12CB701672943
:1090B000072E000C880B990B0E940F97F80165870B
:1090C00076878787908B118A128A138A148A84E2A2
:1090D00090E0A0E0B0E088839983AA83BB83858970
:1090E0009689A789B08D8C839D83AE83BF8382E0F0
:1090F00090E0A0E0B0E088879987AA87BB87188AAC
:10910000198A1A8A1B8AC0908104D0908204E09048
:109110008304F0908404A7019601C501B4010E9464
:109120005F9920E030E048EC52E40E946E976C8B2F
:109130007D8B8E8B9F8BA7019601F80161857285CF
:10914000838594850E945F9920E030E048EC52E4EA
:109150000E946E97688F798F8A8F9B8F20917D04F4
:1091600030917E0440917F0450918004F801658520
:109170007685878590890E945F9920E030E048ECF1
:1091800052E40E946E976C8F7D8F8E8F9F8F81E04F
:10919000DF91CF911F910F91FF90EF90DF90CF90D3
:1091A000BF90AF909F908F907F906F905F904F9007
:1091B0000895CF93DF93282F30E0F901E254F44F64
:1091C0008491F901E858F44FD491F901EE5CF44F21
:1091D000C491CC2389F0811141DEEC2FF0E0EE0F39
:1091E000FF1FE85EF44FA591B491EC91ED2381E06F
:1091F00090E021F480E002C080E090E0DF91CF9128
:109200000895862FD6CF1F93CF93DF93282F30E07A
:10921000F901E254F44F8491F901E858F44FD491E4
:10922000F901EE5CF44FC491CC23C1F0162F8111EB
:1092300015DEEC2FF0E0EE0FFF1FE250F54FA59189
:10924000B4918FB7F894111105C09C91ED2FE09562
:10925000E92302C0EC91ED2BEC938FBFDF91CF910E
:109260001F910895862F642FCECFCF93DF9390E088
:10927000FC01E858F44F2491FC01EE5CF44F84911A
:10928000882361F190E0880F991FFC01EC51F54FA4
:10929000C591D491FC01E250F54FA591B4916111B3
:1092A00009C09FB7F8948881209582238883EC9128
:1092B0002E230BC0623061F49FB7F8943881822F5F
:1092C000809583238883EC912E2B2C939FBF06C01F
:1092D0008FB7F894E8812E2B28838FBFDF91CF9131
:1092E0000895862F642FC1CF863308F0865390915E
:1092F0007B00282F2870977F922B90937B0087709C
:109300002091850490E4299F90011124822B809361
:109310007C0080917A00806480937A0080917A004A
:1093200086FDFCCF809178002091790090E0922B0F
:1093300008953FB7F89480916B0C90916C0CA091BC
:109340006D0CB0916E0C26B5A89B05C02F3F19F08F
:109350000196A11DB11D3FBFBA2FA92F982F8827B5
:10936000820F911DA11DB11DBC01CD0142E0660F10
:10937000771F881F991F4A95D1F708958F929F9262
:10938000AF92BF92CF92DF92EF92FF926B017C017E
:10939000D0DF4B015C01C114D104E104F104E9F018
:1093A000C8DFDC01CB0188199909AA09BB09883EED
:1093B0009340A105B10578F321E0C21AD108E10874
:1093C000F10888EE880E83E0981EA11CB11CC11420
:1093D000D104E104F10421F7DECFFF90EF90DF909C
:1093E000CF90BF90AF909F908F9008952FB7F89433
:1093F0006091670C7091680C8091690C90916A0C77
:109400002FBF08951F920F920FB60F9211242F9322
:109410003F938F939F93AF93BF938091670C9091ED
:10942000680CA091690CB0916A0C3091660C23E035
:10943000230F2D3720F40196A11DB11D05C026E88C
:10944000230F0296A11DB11D2093660C8093670C1B
:109450009093680CA093690CB0936A0C80916B0C8C
:1094600090916C0CA0916D0CB0916E0C0196A11DA9
:10947000B11D80936B0C90936C0CA0936D0CB0930A
:109480006E0CBF91AF919F918F913F912F910F9053
:109490000FBE0F901F901895DF92EF92FF920F93DF
:1094A0001F93CF93DF937C018B01D42EDC011696A2
:1094B000ED91FC911797138615861486DF011B9694
:1094C00033961E92AE17BF07E1F7C0E0B801D7018F
:1094D00016968D919C91179705DAD82F811102C0AD
:1094E000D0E00DC0CD1107C067E0C8010DDDF80167
:1094F0009781891721F0CF5FDC1690F3E7CF8D2F8E
:10950000DF91CF911F910F91FF90EF90DF90089521
:10951000FC0190810180F281E02DF8948181892BFA
:1095200081832281892F809528232283A7E0B0E0C0
:109530001197F1F7218182238183A3E2B0E0119793
:10954000F1F780817894EFECF0E03197F1F7982310
:1095500081E009F480E00895FC0190810180F281AE
:10956000E02D892F809560FF12C0F894228182231C
:1095700082838181892B8183A3E2B0E01197F1F787
:109580008281982B9283789487ED90E011C0F894B3
:109590002281822382838181892B8183AFEFB0E096
:1095A0001197F1F78281982B928378948FE090E065
:1095B0000197F1F70895CF92DF92EF92FF920F9308
:1095C0001F93CF93DF931F92CDB7DEB76C01E62ECA
:1095D00008E010E0FF24F39461E08F2D8E2109F460
:1095E00060E0C6014983B8DFFF0C015011094981D1
:1095F0000115110589F7411115C0F894D60111968E
:10960000ED91FC91129791818C91809589238183B2
:109610001196ED91FC91129792818C9180958923FE
:10962000828378940F90DF91CF911F910F91FF90DB
:10963000EF90DF90CF900895CF92DF92EF92FF925C
:109640000F931F93CF93DF931F92CDB7DEB78C019B
:10965000F62E40E065E57983AEDFCF2C7981D72EF9
:10966000760188E0E80EF11CF60161916F0140E09F
:10967000C801A1DFCE14DF04B9F70F90DF91CF91BD
:109680001F910F91FF90EF90DF90CF900895FC0114
:1096900090810180F281E02DF8948181292F20951D
:1096A0008223818378948DE743E050E0815021F15B
:1096B000DA011197F1F730813923C1F3F8948281EF
:1096C000822382838181892B81837894ABE7B7E001
:1096D0001197F1F7F894818128232183A3E1B1E068
:1096E0001197F1F78081982381E009F080E0789468
:1096F000E3E6F6E03197F1F708958F929F92AF92EB
:10970000BF92CF92DF92EF92FF920F931F93CF936E
:10971000DF93EC018E819F81BADF40E06CEC8E819B
:109720009F8149DF488164E48E819F8144DF8A8183
:10973000882309F43EC0E981E950E33040F4F0E0C9
:10974000EE0FFF1FE751FB4F0081118102C00EEEAB
:1097500012E08B818823E1F08881811119C046DEF7
:109760004B015C016801110FEE08FF088E819F819B
:10977000CFDE8130F1F03ADEDC01CB018C199D099E
:10978000AE09BF0988159905AA05BB0578F311C074
:10979000B801110F880B990BDF91CF911F910F9199
:1097A000FF90EF90DF90CF90BF90AF909F908F9001
:1097B000E5CDDF91CF911F910F91FF90EF90DF905A
:1097C000CF90BF90AF909F908F9008954F925F92EF
:1097D0006F927F928F929F92AF92BF92CF92DF92C1
:1097E000EF92FF920F931F93CF93DF931F921F92DD
:1097F000CDB7DEB72C018A01FC0186819781698390
:109800007A8345DF69817A818823A1F1F20186811B
:10981000978112DF40E06EEBF20186819781CBDE0B
:1098200078014801F9E08F0E911CF2016680778083
:1098300088E0A82EB12CCC24C394D12CC30168DEBF
:109840008111DC28CC0CF1E0AF1AB108B9F7F701AF
:10985000D1927F01E815F90541F7F20186819781E0
:1098600016DF813039F468E0C8014EDB91E0F80181
:109870002085821390E0892F0F900F90DF91CF9178
:109880001F910F91FF90EF90DF90CF90BF90AF901E
:109890009F908F907F906F905F904F900895CF939F
:1098A000DF93CDB7DEB729970FB6F894DEBF0FBEB2
:1098B000CDBFAE014F5F5F4F89DF882389F08D8177
:1098C0008F3361F020F48F3159F489E00CC08F356B
:1098D00019F08F3739F004C08BE005C08AE003C06F
:1098E00080E001C08CE029960FB6F894DEBF0FBE71
:1098F000CDBFDF91CF9108950F931F93CF93DF9347
:10990000CDB7DEB761970FB6F894DEBF0FBECDBFFF
:109910008C01462FBE01665F7F4FBEDD811105C001
:1099200060E070E08EEF92EC4AC0AE014F5F5F4F97
:10993000BE01665F7F4FC80149DF882359F1698105
:1099400048E0649FB00111248A81282F30E0322F33
:109950002227330F330F330F262B372B8A85803185
:10996000E1F4688570E08F81AB01481B5109CA01A1
:109970009695982F8827979587950E94DA9B605136
:109980007109207F53E0220F331F5A95E1F7620FD0
:10999000731F04C060E874EE01C0B901613854EE71
:1099A00075070CF4BDCF072E000C880B990B0E9495
:1099B0000F9720E030E040E05CE30E946E976196F4
:1099C0000FB6F894DEBF0FBECDBFDF91CF911F91D0
:1099D0000F910895EF92FF920F931F93CF93DF9310
:1099E000CDB7DEB728970FB6F894DEBF0FBECDBF58
:1099F0008C01DC011696ED91FC9117971386158664
:109A00001486DF011B9633961E92AE17BF07E1F74F
:109A1000F80114821582EE24E394BE016F5F7F4F3C
:109A2000F801868197810E947244882309F469C0F5
:109A300067E0CE01019668DA98858913EECFD801E8
:109A40008C91811121C016968D919C9117971FDEE4
:109A5000BE016F5F7F4FF80186819781EDDD40E0A9
:109A600064EBD80116968D919C911797A4DDF801AF
:109A7000868197814DDDF82ED80116968D919C91A7
:109A8000179705DEFF20B1F1F801F180898180315F
:109A9000A1F1BE016F5F7F4FC80101DF8F1520F478
:109AA000D80111968C910AC08981803111F48CE023
:109AB00005C0BE016F5F7F4FC801F1DEF8018183F1
:109AC00084818F5F84838981883261F030F48031B2
:109AD00049F0823209F0A1CF05C08B3319F08234EE
:109AE00009F09BCFD80115968C9115978F5F15962D
:109AF0008C9393CFD801EC92C7CFBCE0BF1580F216
:109B0000D6CF28960FB6F894DEBF0FBECDBFDF913B
:109B1000CF911F910F91FF90EF9008950F931F9396
:109B2000CF93DF93EC01162F60E0812F9EDB612F36
:109B300070E0FB01E858F44FE491E883FB01EE5C30
:109B4000F44FE491F0E0EE0FFF1FE85EF44F8591D3
:109B500094919A8389831B861D861C86FE013B9601
:109B60008E010D5F1F4F1292E017F107E1F7DF91B1
:109B7000CF911F910F9108950F931F93CF93DF9370
:109B80001F92CDB7DEB78C01FC01848169830E94EE
:109B9000FB5EF80183856981862B90E00E94F75E69
:109BA0000F90DF91CF911F910F910C94F55E0F9361
:109BB0001F93CF938C01C62FDFDF6C2F6460C80129
:109BC000DBDF6C2F6B7FC801D7DF83EC90E0019760
:109BD000F1F7CF911F910F9108950F931F93CF939A
:109BE0008C01C62F607F6160E2DF80E1C89FB00119
:109BF00011246160C801DBDF81E090E0CF911F910B
:109C00000F9108950F931F9360E080912F04FBDA6A
:109C100083E090E00197F1F761E080912F04F3DA9F
:109C200083E290E00197F1F760E080912F04EBDA96
:109C300080912D0490912E049927FC01E858F44F4F
:109C40006491FC01EE5CF44FE491F0E0EE0FFF1F35
:109C5000E85EF44F8591949100E412E42FE030E047
:109C6000462F0E94AC86611571058105910549F06A
:109C7000DC01CB010196A11DB11DBC01CD019F707E
:109C800003C060E070E0CB010E940D9720E030E05F
:109C900048EC52E40E945F992091730C3091740C4F
:109CA0004091750C5091760C0E946E9720E030E444
:109CB0004CE156E40E945F9920E030E040E05FE331
:109CC0000E946E971F910F91089523E333E948E8AE
:109CD00053E40E945F9920E030E040E85FE30E9497
:109CE00099980E945D9B26E636EA45EA53E40E9475
:109CF0006E976093730C7093740C8093750C9093B3
:109D0000760C0895CF92DF92EF92FF927BDF6B018A
:109D10007C0120E030E040E050E40E944E9A1816AA
:109D20001CF470DF6B017C0120E030E040E050E487
:109D3000C701B6010E944E9A18161CF463DF6B012E
:109D40007C0120E030E040E050E4C701B6010E9411
:109D50004E9A18161CF456DF6B017C0120E030E0AF
:109D600040E050E4C701B6010E944E9A18162CF448
:109D7000FF90EF90DF90CF9045CFC701B601FF90E5
:109D8000EF90DF90CF90089581E08093E20480917E
:109D90001202882339F088E08093361260E08BE26B
:109DA00092E1EACE08958091120281110FC081E004
:109DB000809312028093E20480913112982F946074
:109DC000909331128C600E94055F17C08091E2046D
:109DD000882399F01092361260E08BE292E1CCDE9B
:109DE0001092E204809131128B7F8093311288604F
:109DF0000E94055F109212020895C6CF2F923F92E3
:109E00004F925F926F927F928F929F92AF92BF928A
:109E1000CF92DF92EF92FF920F931F93CF93DF9336
:109E2000CDB7DEB764970FB6F894DEBF0FBECDBFD7
:109E30007C0185E09FE00E943E7040E855E260E0D2
:109E400070E085E09FE00E94255E64E670E080E0BF
:109E500090E094DA8CED95E0A0E0B0E08093090FFB
:109E600090930A0FA0930B0FB0930C0F64E670E071
:109E700080E090E083DA8FEF898381E08A8386E84F
:109E80008B831C821D821E821F82188689E7898728
:109E9000C701880F991F9C8B8B8B212C312CC12CD7
:109EA000D12C812C912C5401CE14DF044CF085E090
:109EB0009FE00E943E70C114D10499F1760131C037
:109EC0008B899C892816390694F785E09FE00E94CB
:109ED000C66908974CF049E050E0BE016F5F7F4FC4
:109EE00085E09FE00E94826965E070E080E090E09C
:109EF00045DA00E010E0412C512C320185E09FE072
:109F00000E94F769892B31F484E0481651046104FA
:109F100071041CF4023011057CF19FEF291A390AF3
:109F2000C3CFC501B4010E940F974B015C01B7017B
:109F3000FF0C880B990B0E940F979B01AC01C50188
:109F4000B4010E945F9964960FB6F894DEBF0FBE0D
:109F5000CDBFDF91CF911F910F91FF90EF90DF90D8
:109F6000CF90BF90AF909F908F907F906F905F90B9
:109F70004F903F902F90089585E09FE00E94F769F1
:109F8000892B69F085E09FE00E94D569EAE0F0E066
:109F9000EC0FFD1FE00FF11F80830F5F1F4F65E087
:109FA00070E080E090E0EAD902301105D1F59A85A1
:109FB0008981981336C09B858B81981332C085E0C8
:109FC0009FE00E94F769892B31F494E0491651040F
:109FD000610471048CF40930110589F085E09FE07B
:109FE0000E94D569EAE0F0E0EC0FFD1FE00FF11FE1
:109FF00080830F5F1F4FE3CF043011057CF02D8568
:10A000008C8590E0982F8827820F911D092E000CD7
:10A01000AA0BBB0B880E991EAA1EBB1E8FEFC81A77
:10A02000D80A9FEF491A590A690A790A67CF2F920D
:10A030003F924F925F926F927F928F929F92AF92D8
:10A04000BF92CF92DF92EF92FF920F931F93CF9325
:10A05000DF9300D01F92CDB7DEB76C0143EF54E021
:10A0600086E394E09A83898303EE1CE0EE24E39474
:10A07000F12C66246394712C22E1222E312C33E1E1
:10A08000432E512C60E1A62EB12C71E1872E912C2C
:10A0900080913404909135048E159F050CF4EDC029
:10A0A00091E0C916D10431F4F80180819181E981F0
:10A0B000FA8109C0F2E0CF16D10439F4E981FA81BE
:10A0C00080819181F80191838083E981FA81808187
:10A0D0009181009741F4FA018281938190938F04DA
:10A0E00080938E0429C08130910541F4FA01828168
:10A0F000938190938D0480938C041EC082309105CF
:10A1000041F4FA018281938190938B0480938A04B5
:10A1100013C0039789F4FA01828193819093890493
:10A120008093880467E57BE08EE791E14B835C8355
:10A130000E94A36C5C814B81E981FA8181919191AC
:10A14000FA83E9838430910541F4FA012281338155
:10A1500030931102209310022CC08530910541F4F8
:10A16000FA0122813381309307022093060221C035
:10A170008630910541F4FA01228133813093C9047C
:10A180002093C80421C08730910541F4FA0122814F
:10A190003381309305022093040221C08A30910557
:10A1A00041F4FA012281338130938704209386049D
:10A1B0003FC08531910541F4FA012281338130930A
:10A1C00003022093020234C08631910541F4FA0162
:10A1D00022813381309301022093000229C087310C
:10A1E000910531F5FA01228133812830310549F496
:10A1F000B0923004A0922F0490922E0480922D04ED
:10A2000017C02730310549F43092300420922F04D2
:10A2100050922E0440922D040BC02630310541F49B
:10A220007092300460922F0410922E0410922D042C
:10A230009C012B5031092A303105B8F4FA012281F2
:10A2400033813093890420938804F7E1F89FB001AB
:10A25000F99F700D1124645E7D4F8EE791E14B8371
:10A260005C830E94A36C5C814B812FEFE21AF20A9F
:10A270004E5F5F4F0E5F1F4F0BCF0F900F900F90F1
:10A280000F90DF91CF911F910F91FF90EF90DF9092
:10A29000CF90BF90AF909F908F907F906F905F9086
:10A2A0004F903F902F900895FF920F931F93CF935D
:10A2B000DF93F82E0AE010E0C0E0D0E08F2D14D834
:10A2C000C80FD91F65E070E080E090E057D80150DA
:10A2D0001109A1F7CE016AE070E00E94C69BCB0194
:10A2E000DF91CF911F910F91FF9008952F923F9290
:10A2F0004F925F926F927F928F929F92AF92BF9296
:10A30000CF92DF92EF92FF920F931F93CF93DF9341
:10A31000CDB7DEB763970FB6F894DEBF0FBECDBFE3
:10A320008B8B60E00E9435498091B912882329F017
:10A3300082E090E0A0E0B0E004C08FE090E0A0E018
:10A34000B0E08F87988BA98BBA8B6FE47CE08AE2B0
:10A3500091E10E945E6C6AE271E1CE0101960E9479
:10A360008F6D4AE050E06FEF7FEFCE01019695D6FA
:10A37000CE0101960E94CD6CC12CD12C7601312CDE
:10A380001D861E86212C02E310E0412C512C320147
:10A390008B890E947449092E000CAA0BBB0B480E36
:10A3A000591E6A1E7B1E65E070E080E090E00E940E
:10A3B000BE490150110961F780904804909049040A
:10A3C000A0904A04B0904B04C301B2010E940F97C1
:10A3D00020E030E040EA50E40E946E9720E030E058
:10A3E00040E85AE30E946E9720E030E048E452E4EF
:10A3F0000E945F99A50194010E94989820E030E0A6
:10A4000040E751E40E946E972B013C01A5019401A5
:10A410006AE979E989E390E40E9498989B01AC018C
:10A42000C301B2010E945F9920E030E0A9010E94BF
:10A43000999820E030E040E251E40E946E975B0181
:10A440008C01232D3D854E85522D0E944E9A181663
:10A4500024F43A2CBD860E87212E20E030E0A9019D
:10A46000B501C8010E94099787FF04C0A12CB12C37
:10A4700000E010E022E0A501B801CE0101960E94A3
:10A48000016DBE016F5F7F4FCE0107960E948F6DF9
:10A490006BED7AE0CE0107960E940F6CBC0184E25E
:10A4A00091E10E94B86CCE0107960E94CD6CCE015E
:10A4B00001960E94CD6C64E271E1CE0101960E948A
:10A4C0008F6D4AE050E060E070E0CE010196B4D4B8
:10A4D000CE0101960E94CD6C0E94F64940906F0C0F
:10A4E0005090700C6090710C7090720C930182010E
:10A4F0000C591F4F2F4F3F4F0617170728073907D3
:10A5000008F4CEC00E94F6490E940D974B015C01F1
:10A51000C301B2010E940F9720E030E048EC51E403
:10A520000E9499989B01AC01C501B4010E94099752
:10A5300087FDB6C06CE370E080E090E00E94BE4909
:10A540009FEFC91AD90AE90AF90A8F859889A9895A
:10A55000BA898C159D05AE05BF050CF014CF64E6D5
:10A5600070E080E090E00E94BE4916D464E670E09E
:10A5700080E090E00E94BE4967E47CE084E291E1E3
:10A580000E945E6C64E271E1CE0101960E948F6DC3
:10A5900044E150E060E070E0CE0101967ED5CE014E
:10A5A00001960E94CD6C22E0432D5D856E85722D53
:10A5B000CE0101960E94016DBE016F5F7F4FCE01FB
:10A5C00007960E948F6D6BED7AE0CE0107960E9490
:10A5D0000F6CBC0184E291E10E94B86CCE01079639
:10A5E0000E94CD6CCE0101960E94CD6C64E271E1B7
:10A5F000CE0101960E948F6D42E350E06FEF7FEF36
:10A60000CE01019619D4CE0101960E94CD6C64E171
:10A6100070E080E090E00E94BE4900D46EE170E0FE
:10A6200080E090E00E94BE496EE170E080E090E042
:10A630000E94BE4960EE7AE0CE0101960E94976DBD
:10A6400064E271E1CE0101960E94266C64EE7AE02C
:10A650000E940F6C6AE271E10E94266CBC018AE2E2
:10A6600091E10E94B86CCE0101960E94CD6C639678
:10A670000FB6F894DEBF0FBECDBFDF91CF911F9113
:10A680000F91FF90EF90DF90CF90BF90AF909F9091
:10A690008F907F906F905F904F903F902F90089594
:10A6A000BDD348CF4F925F926F927F92AF92BF928D
:10A6B000CF92DF92FF920F931F93CF93DF9300D03F
:10A6C00000D0CDB7DEB75C0185E09FE00E943E7010
:10A6D00040E052EC61E070E085E09FE00E94255E82
:10A6E0008CED95E0A0E0B0E08093090F90930A0F05
:10A6F000A0930B0FB0930C0F64E670E080E090E045
:10A700000E94BE49C12CD12CF12CCA14DB040CF0E0
:10A7100051C065E070E080E090E00E94BE4900E03A
:10A7200010E0412C512C3201F1100FC085E09FE068
:10A730000E94F769892B31F485E1481651046104C0
:10A7400071041CF40330110554F08FEFC81AD80AB5
:10A7500064E670E080E090E00E94BE49D6CF85E0DC
:10A760009FE00E94F769892B69F085E09FE00E94D5
:10A77000D569E1E0F0E0EC0FFD1FE00FF11F8083F1
:10A780000F5F1F4F65E070E080E090E00E94BE49DF
:10A79000023011054CF089818B3B31F4FF24F39496
:10A7A0008A818A3A09F0F12C8FEF481A580A680A10
:10A7B000780ABACF8F2D26960FB6F894DEBF0FBE5B
:10A7C000CDBFDF91CF911F910F91FF90DF90CF9080
:10A7D000BF90AF907F906F905F904F9008953F92A1
:10A7E0004F925F926F927F928F929F92AF92BF92A1
:10A7F000CF92DF92EF92FF920F931F93CF93DF934D
:10A80000CDB7DEB7EB970FB6F894DEBF0FBECDBF66
:10A810002B013C0188E69EE00E943E7064E670E0F9
:10A8200080E090E00E94BE4940E855E260E070E0C0
:10A8300088E69EE00E94255E64E670E080E090E09D
:10A840000E94BE496BE37CE084E291E10E945E6C71
:10A8500064E271E1CE0101960E948F6D42E350E007
:10A860006FEF7FEFCE01019618D4CE0101960E94C2
:10A87000CD6C60E37CE084E291E10E945E6C64E276
:10A8800071E1CE0101960E948F6D42E350E06FEFBF
:10A890007FEFCE010196D0D2CE0101960E94CD6C01
:10A8A0008091390C90913A0C8D7F312CC12CD12C98
:10A8B000E12CF12C00E010E0019709F46CC0CE010E
:10A8C000809699AF88AFDE015E96BBAFAAAF0E94BB
:10A8D000F649DC01CB0184199509A609B709883B23
:10A8E0009B40A105B10508F056C088E69EE00E9495
:10A8F000F769892B09F448C08CED95E0A0E0B0E041
:10A9000080936C0E90936D0EA0936E0EB0936F0EAD
:10A910000E94FD6197FD06C082349105C9F780E071
:10A9200090E002C08FEF9FEF892B71F5DE01119649
:10A930004D015D010E94FD6197FF06C089818D3444
:10A9400019F520E030E009C0D5018D935D01E8AD37
:10A95000F9ADAE17BF0771F7F1CFD4018D914D015D
:10A96000280F311DEAADFBADAE17BF07B1F72E5B67
:10A970003F4F8E8D90E0982F88274F8D840F911D2B
:10A980002817390709F4FCC062E370E080E090E02A
:10A990000E94BE499CCF0E94F649DC01CB0184197C
:10A9A0009509A609B709883B9B40A105B10510F49C
:10A9B0003110BEC0F1D164E271E1CE0180960E94F7
:10A9C0008F6D42E350E066E070E0CE01809665D383
:10A9D000CE0180960E94CD6C332009F4E9C082E05C
:10A9E00090E090933A0C8093390C4AE0B601CE0186
:10A9F000C2960E945C6D4AE0B701CE018C960E941F
:10AA00005C6D4AE0B801CE0180960E945C6DBE018B
:10AA1000605E7F4FCE0186960E948F6D68E278E07F
:10AA2000CE0186960E940F6CBE01645D7F4F0E942E
:10AA3000266C68E278E00E940F6CBE016E5C7F4F6E
:10AA40000E94266CBC018AE291E10E94B86CCE01A2
:10AA500086960E94CD6CCE0180960E94CD6CCE0170
:10AA60008C960E94CD6CCE01C2960E94CD6C6AE29B
:10AA700071E1CE0180960E948F6D4AE050E06FEF49
:10AA80007FEFCE018096D8D1CE0180960E94CD6C0A
:10AA90006AE27CE08BE292E10E94046E4AE0B60139
:10AAA000CE01C2960E945C6D4AE0B701CE018C9641
:10AAB0000E945C6D4AE0B801CE0186960E945C6DF2
:10AAC00068EE7AE0CE0180960E94976DBE016A5DC5
:10AAD0007F4FCE0180960E94266C6AEC79E00E943E
:10AAE0000F6CBE01645D7F4F0E94266C6AEC79E0BA
:10AAF0000E940F6CBE016E5C7F4F0E94266C68EF57
:10AB00007AE00E940F6CBC018AE291E10E94B86C6D
:10AB1000CE0180960E94CD6CCE0186960E94CD6CAF
:10AB2000CE018C960E94CD6CCE01C2960E94CD6C57
:10AB300062E370E080E090E00E94BE4988E69EE01B
:10AB40000E943E7062E370E080E090E00E94BE49A7
:10AB5000EB960FB6F894DEBF0FBECDBFDF91CF915D
:10AB60001F910F91FF90EF90DF90CF90BF90AF902B
:10AB70009F908F907F906F905F904F903F9008953F
:10AB80000C8110E0102F00278D81080F111DEE8021
:10AB9000F12CFE2CEE248F81E80EF11CC884D12C00
:10ABA000DC2CCC248985C80ED11C33243394ECCE04
:10ABB0006FE17CE08AE291E10E945E6C6AE271E101
:10ABC000CE0180960E948F6D4AE050E060E070E018
:10ABD000CE01809631D1CE0180960E94CD6C6CE082
:10ABE0007CE08AE291E10E945E6C8091390C909148
:10ABF0003A0C029709F09CCF10923A0C1092390C43
:10AC000097CFCF92DF92EF92FF92CF93DF93CDB7A2
:10AC1000DEB72C970FB6F894DEBF0FBECDBF9927D5
:10AC200043DBBC01990F880B990B0E940F972DE015
:10AC300038E643E55BE30E946E976B017C0120914F
:10AC4000A8043091A9044091AA045091AB040E9439
:10AC5000099718164CF060919004709191048091BE
:10AC60009204909193041BC02091BC043091BD04C8
:10AC70004091BE045091BF04C701B6010E944E9A94
:10AC800087FF05C0C701B6010E94666108C06091D8
:10AC9000A4047091A5048091A6049091A70420E0DB
:10ACA00030E048EC52E40E946E9720E030E048EA41
:10ACB00051E40E946E9720914C0430914D044091D4
:10ACC0004E0450914F040E945F996B017C0164E037
:10ACD0007CE084E291E10E945E6C64E271E1CE016D
:10ACE00001960E948F6D42E350E060E070E0CE017B
:10ACF0000196D3D1CE0101960E94CD6C22E0B7011E
:10AD0000A601CE0107960E94016D6AE579E0CE01A9
:10AD100001960E94976DBE01695F7F4FCE0101963B
:10AD20000E94266C6EEF7AE00E940F6CBC018AE2F2
:10AD300091E10E94B86CCE0101960E94CD6CCE01CB
:10AD400007960E94CD6C6AE271E1CE0101960E94E5
:10AD50008F6D42E350E06FEF7FEFCE0101966CD034
:10AD6000CE0101960E94CD6C8091B912882331F0FA
:10AD700060E273E080E090E00E94BE492C960FB63E
:10AD8000F894DEBF0FBECDBFDF91CF91FF90EF9063
:10AD9000DF90CF9008950895809112028823F9F0F2
:10ADA0008091E2048823D9F081E00E94055F8BE363
:10ADB0009FE10197F1F760E080E00E94165F6CE68A
:10ADC0007DE08BE292E10E94046E61E080E00E94EF
:10ADD000165F6CE57DE08BE292E10C94046E0895C1
:10ADE000CF93DF93209112022223A9F02091E20455
:10ADF000222389F0EC016FED8BE292E10E94EF6D6E
:10AE00008C819D81892B39F0BE018BE292E1DF912B
:10AE1000CF910C94F66DDF91CF910895809112023D
:10AE2000882349F08091E204882329F060E08BE2D6
:10AE300092E10C94ED4D08958F929F92AF92BF9244
:10AE4000EF92FF920F931F93CF93DF937C01EB015F
:10AE50008A0180911202882309F45EC08091E20485
:10AE6000882309F459C077FF16C0C095D09561E0DA
:10AE70008C2FDCD7B7018BE292E10E94F66D6BE478
:10AE80007DE08BE292E10E94046EF701848161E033
:10AE90008C0FCCD731C00E94F64980906F0C9090F7
:10AEA000700CA090710CB090720C24E6820E911C74
:10AEB000A11CB11C86169706A806B90668F561E0C4
:10AEC0008C2FB4D7B7018BE292E10E94F66D6AE352
:10AED0007DE08BE292E10E94046EF701848161E0E3
:10AEE0008C0FA4D70E94F64960936F0C7093700C7E
:10AEF0008093710C9093720CB801110F880B990B11
:10AF0000DF91CF911F910F91FF90EF90BF90AF9085
:10AF10009F908F900C94BE49DF91CF911F910F911C
:10AF2000FF90EF90BF90AF909F908F900895AF9259
:10AF3000BF92CF92DF92EF92FF920F931F93CF9326
:10AF4000DF93CDB7DEB762970FB6F894DEBF0FBEC2
:10AF5000CDBF20911202222309F48EC02091E20479
:10AF6000222309F489C06A017B015C010E94F64931
:10AF70000091830C1091840C2091850C3091860CEB
:10AF80000C591F4F2F4F3F4F061717072807390738
:10AF900008F072C0F7FE07C087010095109560E0C9
:10AFA000802F44D749C060E080E040D70E94F64936
:10AFB00028EE33E040E050E00E943B98CA01B9011E
:10AFC00020E831E541E050E00E943B98AB01BC0134
:10AFD0002AE0CE0101960E94306DBE016F5F7F4F67
:10AFE000CE0107960E948F6D6CE576E0CE01079644
:10AFF0000E940F6CBC01CE010D960E948F6DCE0198
:10B0000007960E94CD6CCE0101960E94CD6CBE01C8
:10B01000635F7F4F8BE292E10E94F66D09891A8986
:10B02000E114F10429F00E0D1F1D60E0802FFED603
:10B03000CE010D960E94CD6CB5018BE292E10E948B
:10B04000F66D69E27DE08BE292E10E94046EF5010B
:10B05000848160E0800FEAD60E94F6496093830CF9
:10B060007093840C8093850C9093860CB601DD0C54
:10B07000880B990B0E94BE4962960FB6F894DEBF0A
:10B080000FBECDBFDF91CF911F910F91FF90EF9039
:10B09000DF90CF90BF90AF900895BF92CF92DF9294
:10B0A000EF92FF920F931F93CF93DF93CDB7DEB74D
:10B0B00062970FB6F894DEBF0FBECDBF6C018B0157
:10B0C0007A0180911202882309F478C08091E20409
:10B0D000882309F473C077FF06C00095109560E0DF
:10B0E000802FA4D64BC060E080E0A0D60E94F64935
:10B0F00028EE33E040E050E00E943B98CA01B901DD
:10B1000020E831E541E050E00E943B98AB01BC01F2
:10B110002AE0CE0101960E94306DBE016F5F7F4F25
:10B12000CE0107960E948F6D6CE576E0CE01079602
:10B130000E940F6CBC01CE010D960E948F6DCE0156
:10B1400007960E94CD6CCE0101960E94CD6CBE0187
:10B15000635F7F4F8BE292E10E94F66DB98860E0F9
:10B160008B2D64D60115110511F40B2D03C060E081
:10B17000802F5CD6CE010D960E94CD6CB6018BE27D
:10B1800092E10E94F66D68E17DE08BE292E10E941F
:10B19000046EF601848160E0800F48D60E94F64973
:10B1A0006093830C7093840C8093850C9093860C31
:10B1B000B701FF0C880B990B0E94BE4962960FB62F
:10B1C000F894DEBF0FBECDBFDF91CF911F910F91DD
:10B1D000FF90EF90DF90CF90BF9008950F931F9353
:10B1E000CF93DF9300D000D0CDB7DEB720913B0CDA
:10B1F0002223A9F08C016CE97AE0CE0101960E942D
:10B20000976DB801CE0101960E94266CBC0182EABE
:10B210009FE00E94E56ECE0101960E94CD6C2696BD
:10B220000FB6F894DEBF0FBECDBFDF91CF911F9157
:10B230000F9108954F925F926F927F928F929F929B
:10B24000AF92BF92CF92DF92EF92FF920F931F9334
:10B25000CF93DF93CDB7DEB7CA54D1090FB6F894B8
:10B26000DEBF0FBECDBF8C0167E57BE0CE018B96C4
:10B270000E94976D67E57BE0CE0185960E94976DF1
:10B28000BE016F5F7F4F8FE591E10E94E8478D8897
:10B290009E88AF88B88C498C5A8C6B8C7C8C8D8D39
:10B2A0009E8DAF8DB8A127968CAF9DAFAEAFBFAFCF
:10B2B0002797C8010197039708F0D4C1A301920111
:10B2C000C501B40190580E940C992BED3FE049EC68
:10B2D0005FE30E94999820916C0430916D04409135
:10B2E0006E0450916F040E9499986B017C0120E0DC
:10B2F00030E0A9010E94099787FD09C0C0927F0C28
:10B30000D092800CE092810CF092820C10C02BED58
:10B310003FE049EC50E4C701B6010E949998609360
:10B320007F0C7093800C8093810C9093820CC09062
:10B330007F0CD090800CE090810CF090820C2BED73
:10B340003FE049EC50E4C701B6010E944E9A18163E
:10B3500084F42BED3FE049EC50E4C701B6010E94B4
:10B36000989860937F0C7093800C8093810C9093DD
:10B37000820C20E030E044E353E460917F0C709154
:10B38000800C8091810C9091820C0E946E972BED25
:10B390003FE049E450E40E945F9960937B0C709316
:10B3A0007C0C80937D0C90937E0C0E94F8994AE06F
:10B3B000CE01C7960E945C6D63E07BE0CE01C19632
:10B3C0000E94976DBE01695C7F4FCE01C1960E94BD
:10B3D000266C6DE07BE00E940F6CBC0180E391E184
:10B3E0000E94B86CCE01C1960E94CD6CCE01C7966A
:10B3F0000E94CD6CC0907B0CD0907C0CE0907D0CBA
:10B40000F0907E0C20E030E044EB52E4C701B6013E
:10B410000E940997181694F020E030E040E05FE3C6
:10B42000C701B6010E9499980E94F8994AE0CE019E
:10B43000C7960E945C6D64E17BE023C020E030E0B1
:10B4400044E353E4C701B6010E9409971816A4F11A
:10B45000A701960160E070E884E393E40E94989865
:10B4600060937B0C70937C0C80937D0C90937E0C8E
:10B470000E94F8994AE0CE01C7960E945C6D67E190
:10B480007BE0CE01C1960E94976DBE01695C7F4F43
:10B49000CE01C1960E94266CBC01CE018B960E9403
:10B4A000B86CCE01C1960E94CD6CCE01C7960E94A9
:10B4B000CD6C6CE07AE063C020E030E047E853E414
:10B4C000C701B6010E940997181604F120E030E088
:10B4D00044E353E4C701B6010E94989820E030E0AD
:10B4E00040E05FE30E94999860937B0C70937C0C22
:10B4F00080937D0C90937E0C0E94F8994AE0CE01D7
:10B50000C7960E945C6D67E17BE01FC0A7019601B2
:10B5100060E070E084EB93E40E94989820E030E0D3
:10B5200040E05FE30E94999860937B0C70937C0CE1
:10B5300080937D0C90937E0C0E94F8994AE0CE0196
:10B54000C7960E945C6D64E17BE0CE01C1960E94CB
:10B55000976DBE01695C7F4FCE01C1960E94266C3B
:10B56000BC01CE018B960E94B86CCE01C1960E94A0
:10B57000CD6CCE01C7960E94CD6C6AE17BE0CE0116
:10B5800085960E94A36CBE01655D7F4FCE01C1967A
:10B590000E948F6D4AE050E060E070E0CE01C196FD
:10B5A0007CDDCE01C1960E94CD6C0E94F6492091AF
:10B5B000830C3091840C4091850C5091860C69016C
:10B5C0007A01A4E6CA0ED11CE11CF11CC616D706EE
:10B5D000E806F90608F435C228962FAF2897299671
:10B5E0003FAF29972A964FAF2A972B965FAF2B979D
:10B5F0000E94F6490E940D976B017C0128962FADA1
:10B60000289729963FAD29972A964FAD2A972B96D2
:10B610005FAD2B97CA01B9010E940F9720E030E07F
:10B6200048EC51E40E9499989B01AC01C701B60116
:10B630000E94099787FD05C26AEC79E0CE01C196A8
:10B640000E94976DBE016B5D7F4FCE01C1960E9437
:10B65000266CBC01CE018B960E94586CCE01C1961F
:10B660000E94CD6CC8010297029708F0C4C120E087
:10B6700030E040E251E4C501B4010E946E976B01D5
:10B680007C0120E030E040E251E4C301B2010E94BD
:10B690006E974B015C0120E030E040E251E42796D8
:10B6A0006CAD7DAD8EAD9FAD27970E946E972B013F
:10B6B0003C010E94F6492091080C3091090C409100
:10B6C0000A0C50910B0C621B730B840B950B0E94A0
:10B6D0000D9720E030E04AE754E40E945F99AB0107
:10B6E000BC0123E0CE01C7960E94016D65E27BE0BC
:10B6F000CE01C1960E94976DBE01695C7F4FCE015D
:10B70000C1960E94266C6CE576E00E940F6CBC012D
:10B710008EE191E10E94B86CCE01C1960E94CD6C81
:10B72000CE01C7960E94CD6C6EE171E1CE01C1964B
:10B730000E948F6D60E371E1CE01C1960E94266C7C
:10B74000BE01655D7F4F0E94266CBC01CE018B96C9
:10B750000E94B86CCE01C1960E94CD6C6DE07DE078
:10B760008AE291E10E945E6C21E0B701A601CE0160
:10B77000C1960E94016DBE016F5C7F4F8AE291E12C
:10B780000E94586CCE01C1960E94CD6C21E0B3019D
:10B79000A201CE01CD960E94016D21E0B501A40168
:10B7A000CE01C7960E94016D6AEC79E0CE01C19688
:10B7B0000E94976DBE01695C7F4FCE01C1960E94C9
:10B7C000266C6AEC79E00E940F6CBE01635C7F4FCF
:10B7D0000E94266C6CE17BE00E940F6CBC018AE247
:10B7E00091E10E94586CCE01C1960E94CD6CCE01B1
:10B7F000C7960E94CD6CCE01CD960E94CD6CA7015C
:10B800009601C701B6010E946E976B017C01A501EC
:10B810009401C501B4010E946E979B01AC01C70160
:10B82000B6010E9499986B017C01A3019201C301AA
:10B83000B2010E946E979B01AC01C701B6010E9444
:10B8400099980E945D9B6B017C016093770C7093CB
:10B85000780C8093790C90937A0C60E27BE08AE21A
:10B8600091E10E944A6C21E0B701A601CE01C19688
:10B870000E94016DBE016F5C7F4FCE01C7960E9492
:10B880008F6D61E37BE0CE01C7960E940F6CBC0117
:10B8900080E391E10E94B86CCE01C7960E94CD6C06
:10B8A000CE01C1960E94CD6C60E371E18AE291E124
:10B8B0000E94586CC090770CD090780CE090790C76
:10B8C000F0907A0C20E030E04AE754E4C701B6017A
:10B8D0000E944E9A87FD29C020E030E04AE754E4F8
:10B8E000C701B6010E945F99AB01BC0123E0CE0104
:10B8F000C1960E94D26CBE016F5C7F4FCE01C7968D
:10B900000E948F6D62E37BE0CE01C7960E940F6CB0
:10B91000BC0180E391E10E94B86CCE01C7960E9401
:10B92000CD6CCE01C1960E94CD6C20E030E64AE697
:10B9300056E46091770C7091780C8091790C90911D
:10B940007A0C0E940997BE01655D7F4F87FF4FC04B
:10B95000CE01C1960E948F6D64E27BE0CE01C1965C
:10B960000E940F6C6AE271E10E94266CBC018AE2BF
:10B9700091E10E94B86CCE01C1960E94CD6C03305B
:10B980001105A1F46AE271E1CE01C1960E948F6DAA
:10B99000CE01C1960E949E7CCE01C1960E94CD6CC4
:10B9A00067E57BE08AE291E10E94A36C67E27BE0BD
:10B9B000CE01C1960E94976D60E371E1CE01C19600
:10B9C0000E94266CBC01CE01C7960E948F6D4AE092
:10B9D00050E06FEF7FEFCE01C7962EDACE01C7960B
:10B9E0000E94CD6CCE01C1960E94CD6C04C08AE24B
:10B9F00091E10E94B86C6AE070E080E090E00E9403
:10BA0000BE49CE0185960E94CD6CCE018B960E94D8
:10BA1000CD6CC65BDF4F0FB6F894DEBF0FBECDBF57
:10BA2000DF91CF911F910F91FF90EF90DF90CF901A
:10BA3000BF90AF909F908F907F906F905F904F904E
:10BA4000089567E57BE0CE01C1960E94976DCE0117
:10BA5000C196C6D9CE01C1960E94CD6CBE016B5D68
:10BA60007F4F8BE292E10E94F66DE6CD1F93CF935C
:10BA7000DF93CDB7DEB7A8970FB6F894DEBF0FBE41
:10BA8000CDBF182FDDD28EE1B6D162E08FE390E119
:10BA9000E0D660E08FE390E1DCD6A7D18EE1ABD1B8
:10BAA00061E08FE390E1D5D660E28FE390E1D1D6FB
:10BAB0009CD180E290E0909363118093621180E0CA
:10BAC00090E8A9E8B4E48093810490938204A09361
:10BAD0008304B093840480E090E0A5E7B4E480930D
:10BAE0007D0490937E04A0937F04B0938004BE01F4
:10BAF0006F5F7F4F8FE591E10E949B47112309F40F
:10BB000094C062EE7CE082EA9FE00E94046E82EACA
:10BB10009FE00E94D26E62ED7CE082EA9FE00E948C
:10BB2000046EBE016F5F7F4F82EA9FE00E94D56E78
:10BB300062EC7CE082EA9FE00E94046E4D855E85A7
:10BB40006F8578892AE030E082EA9FE00E94856E66
:10BB500082EA9FE00E94D26E62EB7CE082EA9FE084
:10BB60000E94046E49895A896B897C892AE030E0F9
:10BB700082EA9FE00E94856E82EA9FE00E94D26E78
:10BB800062EA7CE082EA9FE00E94046E20E030E0FE
:10BB900040E251E4698D7A8D8B8D9C8D0E946E9769
:10BBA00042E050E04CD260E37BE082EA9FE00E94FA
:10BBB000D56E62E97CE082EA9FE00E94046E20E09C
:10BBC00030E040E251E46D8D7E8D8F8D98A10E9412
:10BBD0006E9742E050E033D260E37BE082EA9FE080
:10BBE0000E94D56E62E87CE082EA9FE00E94046ECB
:10BBF00020E030E040E251E469A17AA18BA19CA150
:10BC00000E946E9742E050E01AD260E37BE082EA45
:10BC10009FE00E94D56E6CE57CE082EA9FE00E9486
:10BC2000046E82EA9FE00E94D26E64EF71E080E0D1
:10BC300090E00E94BE49A8960FB6F894DEBF0FBEF2
:10BC4000CDBFDF91CF911F910895CF92DF92EF92F8
:10BC5000FF920F931F93CF93DF93EC016A017B0157
:10BC6000E889F98982E080834115514E61057105AB
:10BC7000B1F060E079E08DE390E0A70196010E94C9
:10BC8000679889019A0101501109210931093695F6
:10BC9000279517950795980101151041A8F0E88997
:10BCA000F989108260E874E88EE190E0A7019601BE
:10BCB0000E946798DA01C9010197A109B109B695F7
:10BCC000A795979587959C01EC85FD853083EE853A
:10BCD000FF852083188EEC89FD8986E08083EA89C0
:10BCE000FB89808180618083EA89FB89808188600B
:10BCF0008083EA89FB89808180688083EA89FB8967
:10BD000080818F7D8083DF91CF911F910F91FF9074
:10BD1000EF90DF90CF900895CF93DF93EC01FB017C
:10BD2000248135810E94AB6DCE01DF91CF910895C2
:10BD3000382F2091CA0D90913712213208F049C056
:10BD40008091A70D8111FCCF42E04093A70D309365
:10BD5000A60D3FEF3093A50D1092A40D2093A30DD7
:10BD6000AAEABDE043E85DE0FA013E2F341B32173A
:10BD700018F43D913193F9CF1092820D2091820DEC
:10BD8000990F922B9093820D9091810D913061F4D7
:10BD90001092810D9091820D9093BB009091BC0008
:10BDA00093FDF8CF95EC01C095EE9093BC00909177
:10BDB000A70D9230E1F39091A50D9F3F79F080910E
:10BDC000A50D803241F08091A50D803331F084E0E3
:10BDD00005C081E003C082E001C083E01092A90D9C
:10BDE0001092CA0D1092A80D089581E0A1CF682F7E
:10BDF0008FE390E12EC591E09093A80D80933712C8
:10BE00001092A90D1092CA0D0895CF93C82F682FD4
:10BE1000607F8BE292E10E94D74D80E1C89FB00124
:10BE200011248BE292E1CF910C94D74DCF93DF9305
:10BE3000CDB7DEB728970FB6F894DEBF0FBECDBFE3
:10BE400098E0E5E0F5E0DE01119601900D929A95FB
:10BE5000E1F790913412961710F46FEF690FFE011D
:10BE60003196E60FF11DE60FF11D9081890F806874
:10BE700028960FB6F894DEBF0FBECDBFDF91CF91ED
:10BE8000C4CF4F925F926F927F928F929F92AF92A8
:10BE9000BF92CF92DF92EF92FF926B017C01B42EA2
:10BEA0009B01AC010E949E9B882319F063E47BE018
:10BEB00027C026013701E89477F82FEF3FEF4FE7CF
:10BEC0005FE7C301B2010E949E9B81110DC02FEF5D
:10BED0003FEF4FE75FE7C301B2010E9409971816D1
:10BEE0001CF467E47BE00CC02FEF3FEF4FE75FE40B
:10BEF000C701B6010E944E9A181694F46BE47BE0D9
:10BF000082EA9FE0FF90EF90DF90CF90BF90AF90DC
:10BF10009F908F907F906F905F904F900C94286EC1
:10BF20002FEF3FEF4FE75FECC701B6010E94099783
:10BF300087FDE4CF20E030E0A901C701B6010E94EF
:10BF4000099787FF0BC06DE282EA9FE00E94EF6DC8
:10BF50004C01F7FAF094F7F8F09402C0812C912C80
:10BF6000A12C60E070E080E09FE3AB1441F020E0A2
:10BF700030E040E251E40E945F99A394F6CF9B0128
:10BF8000AC01C701B6010E9499982B013C010E94A7
:10BF9000FD996B017C010E940D979B01AC01C301CF
:10BFA000B2010E9498982B013C012AE0B701A6013A
:10BFB00082EA9FE00E943D6E7C01E80CF91CBB20E8
:10BFC00039F06EE282EA9FE00E94EF6DE80EF91E02
:10BFD000DB2CDD2031F120E030E040E251E4C30110
:10BFE000B2010E946E972B013C010E94FD994B010A
:10BFF000A12CB12C2AE0B501A40182EA9FE00E94A5
:10C000003D6EE80EF91EC501B4010E940D979B011B
:10C01000AC01C301B2010E9498982B013C01DA9453
:10C02000D8CFC701FF90EF90DF90CF90BF90AF9037
:10C030009F908F907F906F905F904F90089521CF49
:10C040001092800D10927F0D1092A90D1092CA0DC2
:10C050001092A70D81E08093A60D1092810D61E0F2
:10C0600084E10E94034961E085E10E940349E9EB14
:10C07000F0E080818E7F808380818D7F808388E463
:10C080008093B80085E48093BC0008952F923F927E
:10C090004F925F926F927F928F929F92AF92BF92D8
:10C0A000CF92DF92EF92FF920F931F93CF93DF9384
:10C0B000CDB7DEB728970FB6F894DEBF0FBECDBF61
:10C0C00040912F0D5091300DC090310DD090320D18
:10C0D0004C155D052CF03C2D2D2D6A01432F522F60
:10C0E000E3E3FDE060E070E0CB0101911191041702
:10C0F000150754F44A01550FAA08BB08680D791DAD
:10C100008A1D9B1DA80115C0C016D10654F40D2C24
:10C11000000CEE08FF086C0D7D1D8E1D9F1D680133
:10C1200008C0012E000C220B330B600F711F821F01
:10C13000931F2DE0EF37F207C1F60E940F9720E022
:10C1400030E048E152E40E945F996B017C010FE20C
:10C150001DE0812C912C5401D8016D917D918D01B0
:10C16000072E000C880B990B0E940F97A7019601D0
:10C170000E9498989B01AC010E946E979B01AC01B4
:10C18000C501B4010E9499984B015C01BDE00F37D5
:10C190001B0711F720E030E04CE152E40E945F9968
:10C1A0000E945D9B4B015C0120E030E040E85FE3D2
:10C1B0000E944E9A18160CF06EC00FE21DE0212C62
:10C1C000312C19821A821B821C82F8018191919173
:10C1D0008F019C01990F440B550B2D833E834F8398
:10C1E0005887CA01B9010E940F97A70196010E94C2
:10C1F00098982B013C0120E030E0A9010E944E9A62
:10C20000181624F077FA709477F87094A5019401C9
:10C21000C301B2010E94099787FF13C089819A81E7
:10C22000AB81BC812D813E814F815885820F931F48
:10C23000A41FB51F89839A83AB83BC833FEF231A66
:10C24000330A4DE00F37140709F0BFCF20E030E08C
:10C2500040EC5FE3C501B4010E946E974B015C01A5
:10C2600055E0251631040CF4A8CF69817A818B81C1
:10C270009C810E940F976B017C01B101330C880BEC
:10C28000990B0E940F979B01AC01C701B6010E9458
:10C290005F996B017C01C701B60128960FB6F8942F
:10C2A000DEBF0FBECDBFDF91CF911F910F91FF90E9
:10C2B000EF90DF90CF90BF90AF909F908F907F9046
:10C2C0006F905F904F903F902F9008954F925F92A4
:10C2D0006F927F928F929F92AF92BF92CF92DF9296
:10C2E000EF92FF920F931F93CF93DF9300D01F9293
:10C2F000CDB7DEB76B017C0111E0A12EB12C450159
:10C30000880C991C880C991CF401E855FB4F40805F
:10C31000518062807380A3019201C701B6010E941F
:10C320004E9A181614F41F5FE8CFA3019201C701BB
:10C33000B6010E940997840100571B4F811106C066
:10C34000D8016D917D918D919C9142C0C501815024
:10C35000904C880F991F880F991FFC01E855FB4FDF
:10C36000208131814281538129833A834B835C83CD
:10C37000FC01E057FB4F80809180A280B380C70111
:10C38000B6010E9498986B017C01A5019401D80127
:10C390006D917D918D919C910E9498989B01AC012B
:10C3A000C701B6010E946E976B017C0129813A8119
:10C3B0004B815C81C301B2010E9498989B01AC0142
:10C3C000C701B6010E945F99A50194010E94999846
:10C3D0000F900F900F900F90DF91CF911F910F91C1
:10C3E000FF90EF90DF90CF90BF90AF909F908F9095
:10C3F0007F906F905F904F9008950F931F930E94CE
:10C40000F6496093700E7093710E8093720E909344
:10C41000730EE091680EF091690E0284F385E02DB1
:10C4200088E69EE0199597FF1FC00E94F64900918B
:10C43000700E1091710E2091720E3091730EDC010E
:10C44000CB01801B910BA20BB30B00916C0E1091D2
:10C450006D0E20916E0E30916F0E80179107A2071E
:10C46000B307B8F28FEF9FEF1F910F910895CF920E
:10C47000DF92EF92FF920F931F93CF93DF931F9260
:10C48000CDB7DEB76C0109EA1CE07C0186E8E80E56
:10C49000F11CF80161918F01C60169830E94259802
:10C4A0006981681719F0C6010E942D98FFEFCF1A15
:10C4B000DF0ACE14DF0469F789EA9CE00F90DF9170
:10C4C000CF911F910F91FF90EF90DF90CF90089543
:10C4D000CF93DF931F92CDB7DEB76091A70C8EED9F
:10C4E00093E069830E9425986981681721F08EED99
:10C4F00093E00E942D986091A80C8FED93E06983E2
:10C500000E9425986981681721F08FED93E00E94C1
:10C510002D9887EA9CE00F90DF91CF9108953F928C
:10C520004F925F926F927F928F929F92AF92BF9243
:10C53000CF92DF92EF92FF920F931F93CF93DF93EF
:10C5400000D01F921F92CDB7DEB7982E0E94F649F9
:10C550002B013C0120ED420E27E0521E611C711C94
:10C5600060E0809115120E94034935E0832ECE01D0
:10C5700001966C01AA24A394B12C55E0352E380EF7
:10C58000F601282D11922A95E9F7860127E0E22E7F
:10C59000F12C809116120E94D948019739F40E941B
:10C5A000F649641575058605970598F3809116126E
:10C5B0000E94D948892B39F40E94F6496415750503
:10C5C0008605970598F3809117120E94D948892B08
:10C5D00051F0F8012081C5010E2C01C0880F0A948A
:10C5E000EAF7822B8083F1E0EF1AF10890F60F5FF3
:10C5F0001F4F3012CBCF0E94F64964157505860592
:10C60000970550F061E0809115120E94034960E0A7
:10C6100070E080EC9FE72CC089818911B1CF9B81AC
:10C620008A81980F990D8C818913AACF8D818D30C5
:10C6300009F0A6CF61E0809115120E9403496A813A
:10C640008B8170E0762F6627680F711D072E000C16
:10C65000880B990B0E940F9720E030E040E85DE3E3
:10C660000E946E9723E333E948E853E40E949898C8
:10C670000F900F900F900F900F90DF91CF911F911F
:10C680000F91FF90EF90DF90CF90BF90AF909F9071
:10C690008F907F906F905F904F903F900895909112
:10C6A000A70D9111FCCF91E09093A70D9093A60D4B
:10C6B0002FEF2093A50D1092A40D260F2093A30D0C
:10C6C0009093820D9091820D880F892B8093820D1B
:10C6D0008091810D813061F41092810D8091820DE5
:10C6E0008093BB008091BC0083FDF8CF85EC01C036
:10C6F00085EE8093BC008091A70D8130E1F380919D
:10C70000A40D861710F46091A40DA3E8BDE027E8FE
:10C710003CE0F9018E2F821B861718F48D918193CE
:10C72000F9CF862F0895613208F060E2B8DF1092E9
:10C73000800D80937F0D089585ED8093BC008091DE
:10C74000BC0084FDFCCF1092A70D089540915B12B0
:10C75000262F30E0240F311D21323105DCF42091E9
:10C76000A70D2430C9F4FC0180E090E0861758F44E
:10C7700030915B122191DC01A75CBD4EA30FB11D6E
:10C780002C930196F3CF80915B12680F60935B123C
:10C7900080E0089581E0089582E008950895E09191
:10C7A000800D80917F0DE81730F4F0E0E957F34FEA
:10C7B000808190E008958FEF9FEF08959091800D14
:10C7C00080917F0D981750F4E92FF0E0E957F34F6F
:10C7D000208130E09F5F9093800D02C02FEF3FEFEC
:10C7E000C901089580917F0D90E02091800D821BFA
:10C7F00091090895CF92DF92EF92FF920F931F93CA
:10C80000CF93DF937C01262F972F8A018091A80D6B
:10C81000882391F0C62FD72F6E01C40ED51ECC15DC
:10C82000DD0569F06991D701ED91FC910190F081EE
:10C83000E02DC7011995F3CF642F822F87DFC80140
:10C84000DF91CF911F910F91FF90EF90DF90CF90EC
:10C850000895CF93DF931F92CDB7DEB76983209100
:10C86000A80D2223D1F02091CA0D203240F021E002
:10C8700030E0FC013383228380E090E014C080919B
:10C88000A90DE82FF0E0E655F24F998190838F5F74
:10C890008093A90D8093CA0D04C061E0CE0101967A
:10C8A00055DF81E090E00F90DF91CF9108950895DA
:10C8B00080E090E008951F920F920FB60F9211241E
:10C8C0000BB60F922F933F934F935F936F937F938A
:10C8D0008F939F93AF93BF93EF93FF9380914C10EF
:10C8E0000E94D94820915010309151102F5F3F4F36
:10C8F000309351102093501090914F10953618F0AE
:10C9000096E090934B1090914B109430C9F128F41D
:10C91000923069F09330D1F05EC0953009F451C087
:10C92000963009F058C091E090931C1151C08111CC
:10C9300052C020915010309151102436310508F426
:10C9400042C010921C1110924F101CC0813009F08F
:10C9500042C0E0914F1091E09E0F90934F10F0E095
:10C960002091501030915110EE0FFF1FE55BFF4EEC
:10C9700030872783109251101092501094E029C0F4
:10C98000811117C0E0914F1091E09E0F90934F10CE
:10C99000F0E02091501030915110EE0FFF1FE55B39
:10C9A000FF4E30872783109251101092501093E061
:10C9B00010C020915010309151102536310558F09B
:10C9C00007C0811108C0109251101092501003C07E
:10C9D00095E090934B1090914E109923B9F08111EE
:10C9E0000AC080914D10882321F080914D1061E0A4
:10C9F00009C02F9A0BC080914D10882331F080918F
:10CA00004D1060E00E94034901C02F98FF91EF9103
:10CA1000BF91AF919F918F917F916F915F914F9156
:10CA20003F912F910F900BBE0F900FBE0F901F9054
:10CA30001895CF92DF92EF92FF92CF93DF93EC01A4
:10CA4000072E000C880B990B0E940F976B017C013D
:10CA500020E030E040E45FE30E946E9720E030E0A9
:10CA600048E452E40E945F990E94F899C617D707DC
:10CA7000D4F020E030E040EA5FE3C701B6010E9455
:10CA80006E9720E030E048E452E40E945F9920E095
:10CA900030E040E85FE30E9499980E94F89921E015
:10CAA0006C177D070CF420E0822F90E0DF91CF918E
:10CAB000FF90EF90DF90CF9008950F931F93CF9347
:10CAC000DF93082F6DE779E082EA9FE00E94F56E20
:10CAD000C7E0D0E010E0B8010C2E02C07595679554
:10CAE0000A94E2F76170772742E050E082EA9FE023
:10CAF0000E94CC6E219778F7DF91CF911F910F9113
:10CB000008951F920F920FB60F9211240BB60F9239
:10CB10002F933F934F935F936F937F938F939F9345
:10CB2000AF93BF93EF93FF938091B900887F8036D6
:10CB300009F49CC068F5883209F45BC090F4803138
:10CB400009F454C038F4882309F4F6C0883009F495
:10CB50004DC0F5C0883109F44CC0803209F45DC085
:10CB6000EEC0803409F468C048F4803309F455C03D
:10CB7000883309F0E4C08093A50DD8C0803509F44E
:10CB80004FC0883509F45DC0883409F0D8C0D6C0DC
:10CB9000883909F4C7C0A8F4883709F467C038F4A5
:10CBA000883609F463C0803709F460C0C8C088388B
:10CBB00009F4B8C0803909F45FC0803809F0BFC0FB
:10CBC0005BC0803B09F486C038F4803A09F466C043
:10CBD000883A09F47FC0B3C0803C09F4A7C0883C00
:10CBE00009F4A4C0883B09F48AC0A9C08091820DD1
:10CBF00010C09091A40D8091A30D981770F5E0914D
:10CC0000A40D81E08E0F8093A40DF0E0ED57F24F5C
:10CC100080818093BB0085EC86C08093A50D8EC07B
:10CC2000E091A40D81E08E0F8093A40D8091BB0054
:10CC3000F0E0ED57F24F80839091A40D8091A30D09
:10CC40006EC0E091A40D81E08E0F8093A40D8091C1
:10CC5000BB00F0E0ED57F24F80838091A60D81116B
:10CC60006DC081E08093810D84EA61C083E0809390
:10CC7000A70D10927F12CFCF80917F12803208F0E3
:10CC800051C0E0917F1281E08E0F80937F128091DE
:10CC9000BB00F0E0E15AFD4E8083BDCF85EC809370
:10CCA000BC001092A70D80917F12803230F4E09189
:10CCB0007F12F0E0E15AFD4E108260917F1270E029
:10CCC000E0915D12F0915E128FE592E1199510925C
:10CCD0007F1235C084E08093A70D10925C121092F1
:10CCE0005B12E0915912F0915A12199580915B12E2
:10CCF000811105C081E080935B1210923912E0919E
:10CD00005C1281E08E0F80935C12F0E0E75CFD4ED8
:10CD100080818093BB0090915C1280915B12981788
:10CD200008F479CF85E88093BC0009C085EC809336
:10CD3000BC001092A70D03C01092A50DFDDCFF9161
:10CD4000EF91BF91AF919F918F917F916F915F9183
:10CD50004F913F912F910F900BBE0F900FBE0F90F0
:10CD60001F9018953F924F925F926F927F928F9291
:10CD70009F92AF92BF92CF92DF92EF92FF920F936A
:10CD80001F93CF93DF93CDB7DEB7AC970FB6F89470
:10CD9000DEBF0FBECDBF81E08093381200E010E00F
:10CDA00088EE882E83E0982EA12CB12C90E8C92E15
:10CDB00091E5D92EEE24E394F12C22E0322E0E30B0
:10CDC000110508F074C2F8018827E754FF4F8F4F10
:10CDD0000C94ED9B80911F0D9091200D892BE1F417
:10CDE00069EF79E0CE010796A2D66FE172E1CE013C
:10CDF00007962CD5BC01CE01019691D648EC50E0A7
:10CE00006FEF7FEFCE0101960E944D58CE01019643
:10CE1000C4D5CE010796C1D580911F0D9091200DEC
:10CE20000197E1F465EE79E0CE01079680D66FE1D7
:10CE300072E1CE0107960AD5BC01CE0101966FD6EC
:10CE400048EC50E06FEF7FEFCE0101960E944D5805
:10CE5000CE010196A2D5CE0107969FD580911F0DD8
:10CE60009091200D0297E1F46EE07AE0CE010796F2
:10CE70005ED66FE172E1CE010796E8D4BC01CE0127
:10CE800001964DD648EC50E06FEF7FEFCE01019652
:10CE90000E944D58CE01019680D5CE0107967DD5D2
:10CEA00063E17AE0CE01079642D669E172E1CE01F4
:10CEB0000796CCD4BC01CE01019631D640ED57E0A7
:10CEC0006FEF7FEFCE0101960E941C57CE010196B5
:10CED00064D5CE01079661D580911F0D9091200DEC
:10CEE0000197C9F5CE0107960E946C768B859C85CB
:10CEF000009771F1EF81F8852081222349F107978E
:10CF000038F169EE7EE0CE01019601D648EC50E0A2
:10CF10006FEF7FEFCE0101960E949757CE010196E9
:10CF20003CD5BE01695F7F4FCE010196F8D548EC34
:10CF300050E06FEF7FEFCE0101960E941C57CE01AB
:10CF400001962BD560ED77E080E090E00E94BE492D
:10CF5000CE01079622D564E670E080E090E00E9462
:10CF6000BE4930924B1010924F10A1C16DED7EE082
:10CF7000CE010196CCD548EC50E06FEF7FEFCE01AB
:10CF800001960E949757CE01019607D50E94F64957
:10CF90006DA37EA38FA398A70E94F649A5019401D3
:10CFA0000E946798CA01B901A70196010E9467987B
:10CFB00020E13EE040E050E00E943B9829013A0128
:10CFC0002CE330E040E050E00E943B9829A73AA7CC
:10CFD0004BA75CA7AB01BC012AE0CE01019640D56E
:10CFE0002AE049A55AA56BA57CA5CE01079638D5A0
:10CFF0002AE0B301A201CE010D9632D56DA17EA12A
:10D000008FA198A5A50194010E946798CA01B90152
:10D01000A70196010E946798BA01A9012AE0CE01F2
:10D0200049961ED5BE01675E7F4FCE01439677D5E8
:10D030006FE47BE0CE014396F2D3BE01635F7F4F86
:10D0400005D462E57BE0EBD3BE01695F7F4FFED381
:10D0500063E279E0E4D3BE016F5F7F4FF7D36CEEFC
:10D0600078E0DDD3BC01CE014F9659D5CE01439671
:10D0700094D4CE01499691D4CE010D968ED4CE0192
:10D0800007968BD4CE01019688D440ED57E06FEF20
:10D090007FEFCE014F960E941C57CE014F9606C1DE
:10D0A0008091390C90913A0C019719F46EEC7EE066
:10D0B00002C060EC7EE0CE01019629D548EC50E03C
:10D0C0006FEF7FEFCE0101960E949757CE01019638
:10D0D00064D460EB7EE0DDC060EA7EE0CE010196C4
:10D0E00016D548EC50E06FEF7FEFCE0101960E941D
:10D0F0009757CE01019651D463E97EE0CAC066E835
:10D100007EE0CE01019603D548EC50E06FEF7FEF53
:10D11000CE0101960E949757CE0101963ED46BE74F
:10D120007EE0B7C06FE67EE0CE010196F0D448EC19
:10D1300050E06FEF7FEFCE0101960E949757CE012E
:10D1400001962BD46EE57EE0A4C08091390C9091BD
:10D150003A0C039719F463E57EE002C069E47EE0CF
:10D16000CE010196D4D448EC50E06FEF7FEFCE01B2
:10D1700001960E949757CE0101960FD46EE37EE090
:10D1800088C061E37EE0CE010196C1D448EC50E056
:10D190006FEF7FEFCE0101960E949757CE01019667
:10D1A000FCD362E27EE075C067E17EE0CE010196CD
:10D1B000AED448EC50E06FEF7FEFCE0101960E94B5
:10D1C0009757CE010196E9D36AE07EE062C0809174
:10D1D000390C90913A0C029719F469EF7DE002C086
:10D1E00069EE7DE0CE01019692D448EC50E06FEFFD
:10D1F0007FEFCE0101960E949757CE010196CDD3C5
:10D200006CED7DE046C060ED7DE0CE0101967FD4FF
:10D2100048EC50E06FEF7FEFCE0101960E949757E8
:10D22000CE010196BAD360EC7DE033C065EB7DE0C2
:10D23000CE0101966CD448EC50E06FEF7FEFCE0149
:10D2400001960E94975730C065EA7DE0CE010196B5
:10D250005ED448EC50E06FEF7FEFCE0101960E9464
:10D260009757CE01019699D368E97DE012C06CE82A
:10D270007DE0CE0101964BD448EC50E06FEF7FEF9C
:10D28000CE0101960E949757CE01019686D36CE796
:10D290007DE0CE0101963BD440ED57E06FEF7FEF8C
:10D2A000CE0101960E941C57CE01019676D30E94B2
:10D2B000CA45882319F0109238120BC001D780910B
:10D2C0003812882331F00F5F1F4F0F30110509F01E
:10D2D00076CDAC960FB6F894DEBF0FBECDBFDF9112
:10D2E000CF911F910F91FF90EF90DF90CF90BF9063
:10D2F000AF909F908F907F906F905F904F903F90F6
:10D3000008950895CF92DF92EF92FF920F931F93AB
:10D31000CF93DF936C017A018B01C0E0D0E0CE1592
:10D32000DF0589F0D8016D918D01D601ED91FC9159
:10D330000190F081E02DC6011995892B11F47E0131
:10D3400002C02196ECCFC701DF91CF911F910F91C1
:10D35000FF90EF90DF90CF900895FC01A089B189F4
:10D360008C91A689B78982FD0FC09C91818D8F5FBA
:10D370008F73228D821749F0218DDF01A20FB11D1D
:10D380005D969C93818F08958C910895FC01538D37
:10D39000448D252F30E0842F90E0821B930B54178F
:10D3A00010F0CF96089501970895FC01918D828D1C
:10D3B000981761F0828DDF01A80FB11D5D968C91E9
:10D3C000928D9F5F9F73928F90E008958FEF9FEFF4
:10D3D0000895FC01918D828D981731F0828DE80FB0
:10D3E000F11D858D90E008958FEF9FEF0895FC016A
:10D3F000918D228D892F90E0805C9F4F821B910937
:10D400008F73992708958BEC9DE0F1DF21E0892B44
:10D4100009F420E0822F089588E69EE0E8DF21E00D
:10D42000892B09F420E0822F089585E09FE0DFDF5B
:10D4300021E0892B09F420E0822F089582EA9FE001
:10D44000D6DF21E0892B09F420E0822F0895FC012A
:10D45000848DDF01A80FB11DA35ABF4F2C91848D7D
:10D4600090E001968F739927848FA689B7892C93B2
:10D47000A089B1898C9180648C93938D848D98134D
:10D4800006C00288F389E02D80818F7D8083089516
:10D49000EF92FF920F931F93CF93DF93EC0181E004
:10D4A000888F9B8D8C8D981305C0E889F9898081C0
:10D4B00085FD23C0F62E0B8D10E00F5F1F4F0F73FD
:10D4C0001127E02E8C8DE8120BC00FB607FCFACFA7
:10D4D000E889F989808185FFF5CFCE01B8DFF2CFE9
:10D4E0008B8DFE01E80FF11DE35AFF4FF0820B8F89
:10D4F000EA89FB898081806207C0EE89FF896083A9
:10D50000E889F98980818064808381E090E0DF91FF
:10D51000CF911F910F91FF90EF900895CF93DF93DC
:10D52000EC01888D8823C1F0EA89FB89808185FD23
:10D5300005C0A889B9898C9186FD0EC00FB607FC7D
:10D54000F5CF808185FFF2CFA889B9898C9185FFBD
:10D55000EDCFCE017CDFE8CFDF91CF91089580E061
:10D5600090E0892B19F06ADF811116C080E090E00D
:10D57000892B19F05ADF811112C080E090E0892BCD
:10D5800019F04ADF81110EC080E090E0892B79F01C
:10D590003ADF81110AC008950E940000E7CF0E947F
:10D5A0000000EBCF0E940000EFCF0C940000089524
:10D5B0000E943D9ECF93DF93EC0188819981009773
:10D5C00011F00E94C19C198218821D821C821B824C
:10D5D0001A82DF91CF910895FC018081918100979B
:10D5E00011F00C945D9260E070E0CB010895AF9271
:10D5F000BF92CF92DF92EF92FF920F931F93CF9340
:10D60000DF93DC01CD90DC901197C114D10409F4B3
:10D6100042C01496CD91DC9115972097E1F18C01D1
:10D6200056017501BFEFAB1ABB0AF7018081082EC6
:10D63000000C990B0E94D996892B99F72197CC0D54
:10D64000DD1D8881082E000C990B0E94D996892B2C
:10D6500091F4AE014F5F5F4F4E195F09D8011596E7
:10D660005C934E931497CE14DF0450F4B701C601B7
:10D670000E94529E05C0CE15DF0558F32197E1CFD9
:10D68000D801ED91FC91119714968D919C9115976D
:10D69000E80FF91F1082DF91CF911F910F91FF903A
:10D6A000EF90DF90CF90BF90AF900895FC01248160
:10D6B00035816217730748F480819181009729F0C2
:10D6C000FC01E60FF71F8081089580E00895FB01BB
:10D6D00044815581FC01248135812417350778F078
:10D6E00080819181009759F0FB0160817181611502
:10D6F000710529F00E946B9E21E0892B09F020E042
:10D70000822F08950F931F93CF93DF938C01EB012A
:10D71000FC01808191810097B1F068817981611568
:10D72000710579F0428153812C813D814217530765
:10D7300040F00E94649E8C819D81F80195838483D2
:10D7400013C00E94C19C88819981F80191838083D4
:10D750008A819B81938382838C819D81958384833D
:10D76000198218821B821A821D821C82DF91CF913E
:10D770001F910F9108950F931F93CF93DF93EC01A7
:10D7800088819981009729F02A813B8126173707E4
:10D7900088F48B016F5F7F4F0E94599D009761F065
:10D7A000998388831B830A832C813D81232B11F469
:10D7B000FC01108281E001C080E0DF91CF911F91D8
:10D7C0000F910895EF92FF920F931F93CF93DF93E2
:10D7D000FC01248135816115710511F480E018C0C8
:10D7E00041155105A1F07B01EC018A01020F131FC5
:10D7F000B801C1DF882391F3288139818C819D8113
:10D80000B701820F931F0E94649E1D830C8381E0E9
:10D81000DF91CF911F910F91FF90EF900895CF93DB
:10D82000DF93EC016115710559F0FB0101900020B7
:10D83000E9F73197AF01461B570BC4DF811102C0D6
:10D84000CE01B8DECE01DF91CF910895CF93DF9363
:10D85000EC01FB014481558160817181B3DF81114D
:10D8600002C0CE01A7DECE01DF91CF910895CF9304
:10D87000DF931F921F92CDB7DEB769831A8241E012
:10D8800050E0BE016F5F7F4F9DDF0F900F90DF91E3
:10D89000CF9108956115710549F0FB0101900020B9
:10D8A000E9F73197AF01461B570B8CCF80E0089505
:10D8B000FB01448155816081718184CFEF92FF9299
:10D8C0000F931F93CF93DF93EC018B0161157105CB
:10D8D00049F0CB010E948A927C01BC01CE014BDF52
:10D8E000811103C0CE0166DE07C0FD82EC82B80163
:10D8F000888199810E948392CE01DF91CF911F91FF
:10D900000F91FF90EF900895EF92FF920F931F9366
:10D91000CF93DF93EC017B018A01BA012CDF8111E7
:10D9200003C0CE0147DE07C01D830C83B701888189
:10D9300099810E94649ECE01DF91CF911F910F913A
:10D94000FF90EF900895CF93DF93EC01611571057F
:10D9500051F0FB0101900020E9F73197AF01461B20
:10D96000570BD2DF01C026DECE01DF91CF910895A3
:10D97000CF93DF93EC01FB018617970751F060818D
:10D9800071816115710521F044815581BDDF01C0B0
:10D9900011DECE01DF91CF910895FC01808191814C
:10D9A0000C94C19CEF92FF920F931F93CF93DF9340
:10D9B000CDB7DEB7A1970FB6F894DEBF0FBECDBFCF
:10D9C0007C01CB01BA01F70111821082138212820D
:10D9D0001582148242E0420F8E010F5F1F4F0E949A
:10D9E0003B92BC01C701AFDFA1960FB6F894DEBF32
:10D9F0000FBECDBFDF91CF911F910F91FF90EF90A0
:10DA00000895EF92FF920F931F93CF93DF93CDB7BB
:10DA1000DEB7A1970FB6F894DEBF0FBECDBF7C0175
:10DA2000CB01BA01F7011182108213821282158292
:10DA3000148242E0420F8E010F5F1F4F0E943B9203
:10DA4000BC01C70180DFA1960FB6F894DEBF0FBE00
:10DA5000CDBFDF91CF911F910F91FF90EF9008956F
:10DA60000F931F93CF93DF93CDB7DEB7A2970FB677
:10DA7000F894DEBF0FBECDBF8C01CB01BA01F80117
:10DA800011821082138212821582148230E0AE015C
:10DA90004F5F5F4F0E94A792BE016F5F7F4FC8012B
:10DAA00052DFA2960FB6F894DEBF0FBECDBFDF9156
:10DAB000CF911F910F9108950F931F93CF93DF93F1
:10DAC000CDB7DEB762970FB6F894DEBF0FBECDBFFD
:10DAD0008C01CB01F801118210821382128215820F
:10DAE000148250E0BE016F5F7F4F0E949392BE018F
:10DAF0006F5F7F4FC80127DF62960FB6F894DEBFD5
:10DB00000FBECDBFDF91CF911F910F910895FC0102
:10DB1000118210821382128215821482CFCEFC01F0
:10DB200011821082138212821582148221CFFC018D
:10DB3000118210821382128215821482611571057E
:10DB400049F0FB0101900020E9F73197AF01461B36
:10DB5000570BDACE0895BF92CF92DF92EF92FF92E9
:10DB60000F931F93CF93DF937C016B018A01E9012F
:10DB70002417350720F4812F8901C42FD82F67E59A
:10DB80007BE0C701D4DFD60114968D919C91159747
:10DB900008171907C8F48C179D0708F4EC01D60183
:10DBA000ED91FC911197EC0FFD1FB08010824D910B
:10DBB0005C91BA01600F711FC701C5DED601ED91FE
:10DBC000FC91EC0FFD1FB082C701DF91CF911F9137
:10DBD0000F91FF90EF90DF90CF90BF900895DC0100
:10DBE000ED91FC910190F081E02D1994DC01ED9113
:10DBF000FC91DB0114964D915C9115976D917C9190
:10DC00000280F381E02D1994EF92FF920F931F93FE
:10DC1000CF93DF938C017B01C0E0D0E0F701EC0FE4
:10DC2000FD1F6491662361F0D801ED91FC91019094
:10DC3000F081E02DC8011995892B11F02196EECFC6
:10DC4000CE01DF91CF911F910F91FF90EF9008953A
:10DC50006115710579F0FB0101900020E9F731971A
:10DC6000AF01461B570BDC01ED91FC910280F38163
:10DC7000E02D199480E090E008954F925F926F92AA
:10DC80007F92EF92FF920F931F93CF93DF93CDB7C5
:10DC9000DEB7A1970FB6F894DEBF0FBECDBF7C01F3
:10DCA000FA01CB0119A2223008F42AE08E010F5D9F
:10DCB0001F4F422E512C612C712CBF01A3019201E8
:10DCC0000E946798F901CA01015011096A3014F4E1
:10DCD000605D01C0695CD8016C93232B242B252B3C
:10DCE00061F7B801C701B4DFA1960FB6F894DEBFA3
:10DCF0000FBECDBFDF91CF911F910F91FF90EF909D
:10DD00007F906F905F904F900895CF92DF92EF9247
:10DD1000FF920F931F93CF93DF93EC016A017B0176
:10DD20002115310579F4E881F9810190F081E02D28
:10DD3000642FDF91CF911F910F91FF90EF90DF90B3
:10DD4000CF9019942A303105D9F477FF18C06DE2CD
:10DD500046DF8C0144275527BA014C195D096E092D
:10DD60007F092AE0CE0189DF800F911FDF91CF91DB
:10DD70001F910F91FF90EF90DF90CF9008952AE0D0
:10DD8000B701A601CE01DF91CF911F910F91FF90B6
:10DD9000EF90DF90CF9071CF9A01AB01770F660BB8
:10DDA000770BB3CF65E57BE053CF0F931F93CF93F2
:10DDB000DF93EC014DDF8C01CE01F4DF800F911F6A
:10DDC000DF91CF911F910F9108950F931F93CF93E0
:10DDD000DF93EC010BDF8C01CE01E4DF800F911F9C
:10DDE000DF91CF911F910F91089532CF1F920F9223
:10DDF0000FB60F9211240BB60F922F933F934F93B0
:10DE00005F936F937F938F939F93AF93BF93EF93A2
:10DE1000FF938BEC9DE01BDBFF91EF91BF91AF91E6
:10DE20009F918F917F916F915F914F913F912F9132
:10DE30000F900BBE0F900FBE0F901F9018951F9262
:10DE40000F920FB60F9211240BB60F922F933F93A0
:10DE50004F935F936F937F938F939F93AF93BF93F2
:10DE6000EF93FF938BEC9DE078DAFF91EF91BF91F8
:10DE7000AF919F918F917F916F915F914F913F9162
:10DE80002F910F900BBE0F900FBE0F901F90189503
:10DE90001F920F920FB60F9211240BB60F922F9371
:10DEA0003F934F935F936F937F938F939F93AF9322
:10DEB000BF93EF93FF9388E69EE0C9DAFF91EF915D
:10DEC000BF91AF919F918F917F916F915F914F9192
:10DED0003F912F910F900BBE0F900FBE0F901F9090
:10DEE00018951F920F920FB60F9211240BB60F9236
:10DEF0002F933F934F935F936F937F938F939F9352
:10DF0000AF93BF93EF93FF9388E69EE026DAFF91ED
:10DF1000EF91BF91AF919F918F917F916F915F91A1
:10DF20004F913F912F910F900BBE0F900FBE0F900E
:10DF30001F9018951F920F920FB60F9211240BB6D7
:10DF40000F922F933F934F935F936F937F938F9392
:10DF50009F93AF93BF93EF93FF9385E09FE077DAB2
:10DF6000FF91EF91BF91AF919F918F917F916F91B1
:10DF70005F914F913F912F910F900BBE0F900FBE6D
:10DF80000F901F9018951F920F920FB60F921124A9
:10DF90000BB60F922F933F934F935F936F937F93A3
:10DFA0008F939F93AF93BF93EF93FF9385E09FE091
:10DFB000D4D9FF91EF91BF91AF919F918F917F91B4
:10DFC0006F915F914F913F912F910F900BBE0F90EA
:10DFD0000FBE0F901F9018951F920F920FB60F92C1
:10DFE00011240BB60F922F933F934F935F936F9330
:10DFF0007F938F939F93AF93BF93EF93FF9382EAA7
:10E000009FE025DAFF91EF91BF91AF919F918F91A2
:10E010007F916F915F914F913F912F910F900BBE28
:10E020000F900FBE0F901F9018951F920F920FB672
:10E030000F9211240BB60F922F933F934F935F9340
:10E040006F937F938F939F93AF93BF93EF93FF93C0
:10E0500082EA9FE082D9FF91EF91BF91AF919F91AA
:10E060008F917F916F915F914F913F912F910F9081
:10E070000BBE0F900FBE0F901F901895CF93DF939C
:10E08000EC01E881F9810680F781E02D1995EA8994
:10E09000FB8980818F7E8083EA89FB898081877FED
:10E0A0008083EA89FB8980818F778083EA89FB8975
:10E0B00080818F7D80838A8D898FDF91CF910895B4
:10E0C000CF92DF92EF92FF920F931F93CF93DF9344
:10E0D000CDB7DEB762970FB6F894DEBF0FBECDBFE7
:10E0E00081E08093130284E992E10E943233892B0C
:10E0F00009F48CC280913812882319F010923812DA
:10E10000DCC51092381280913B0C882391F16CE9A8
:10E110007AE0CE0101960BDDBE016F5F7F4F82EA90
:10E120009FE064DDBE016F5F7F4F8BEC9DE05EDDA5
:10E13000CE01019632DC4091981250919912609173
:10E140009A1270919B1220E182EA9FE096DD82EAAA
:10E150009FE028DE409198125091991260919A1296
:10E1600070919B1220E18BEC9DE087DD8BEC9DE0B4
:10E1700019DE8091981290919912A0919A12B09103
:10E180009B12883025E09207A105B10509F4D2C1A0
:10E1900008F08DC0893421E09207A105B10509F48A
:10E1A000D1C1E0F5843421E09207A105B10509F45D
:10E1B000A1C1E8F4813421E09207A105B10509F479
:10E1C00081C138F480349140A105B10509F46DC1D5
:10E1D0000BC2823421E09207A105B10509F47AC18E
:10E1E00083349140A105B10509F47CC1FDC1863499
:10E1F00021E09207A105B10509F48CC108F482C1A0
:10E20000873421E09207A105B10509F48BC1883458
:10E210009140A105B10509F48DC1E6C1823025E028
:10E220009207A105B10509F455C1E8F4843721E04E
:10E230009207A105B10509F409C138F4823791406C
:10E24000A105B10509F40CC1CFC1811525E09207E4
:10E25000A105B10509F429C181309540A105B10599
:10E2600009F430C1C1C1853025E09207A105B1058F
:10E2700009F448C170F4833025E09207A105B10587
:10E2800009F430C184309540A105B10509F432C1CB
:10E29000ABC1863025E09207A105B10509F43AC16A
:10E2A00087309540A105B10509F43CC19DC18D3B66
:10E2B00022E492072FEFA207B10509F4E9C008F0A4
:10E2C0004AC08F3E20E192072FEFA207B10509F463
:10E2D00029C110F5823325E09207A105B10509F4A3
:10E2E000BFC038F489309540A105B10509F42AC1B1
:10E2F0007BC1843325E09207A105B10509F4A6C0CE
:10E300008D3F9240AF4FB10509F06EC163E87BE0ED
:10E3100082E491E118DB95C08D3D22E292072FEF58
:10E32000A207B10509F492C038F4873E9841AF4F77
:10E33000B10509F4E7C058C18F3C20E392072FEFE5
:10E34000A207B10509F4D6C0873C9843AF4FB10589
:10E3500009F4F0C049C1873928E692072FEFA207D8
:10E36000B10509F4AFC038F58D3A22E592072FEFD9
:10E37000A207B10509F47FC038F4853B9A44AF4F3A
:10E38000B10509F492C030C1853A2AE592072FEF12
:10E39000A207B10509F4D6C08D399246AF4FB10539
:10E3A00009F022C163E87BE082E491E1CCDA81E00C
:10E3B0008093B91246C0873528EA92072FEFA2074B
:10E3C000B105F1F078F485382AE792072FEFA2071C
:10E3D000B10509F49FC087369849AF4FB10509F4DC
:10E3E00079C002C18F3420EB92072FEFA207B1054D
:10E3F00009F478C08D33924CAF4FB10589F1F4C068
:10E400006CE271E080E090E00E94BE4982E080937F
:10E410004B1010924F1000E010E084E892E10E944F
:10E420003233892B09F096C00F5F1F4F0536110557
:10E4300009F490C06EE170E080E090E00E94BE4977
:10E44000ECCF8BEF9FEF0E94BA1DD4C066E87BE053
:10E4500082E491E178DA1092B9128CEF9FEFF3CF5A
:10E4600069E87BE082E491E16EDA81E08093B912A1
:10E470008DEF9FEFE8CF6CE87BE082E491E163DA17
:10E480006CE87BE082E491E15EDA8EEF9FEFDBCF18
:10E490006FE87BE082E491E156DA6FE87BE082E4AA
:10E4A00091E151DA8FEF9FEFCECF62EC7BE086E314
:10E4B00091E149DA62EC7BE082E491E144DA80E0C8
:10E4C00090E0C1CF60E97BE086E391E13CDA81E056
:10E4D00090E0B9CF6DE87BE086E391E134DA82E049
:10E4E00090E0B1CF6AE87BE086E391E12CDA83E04B
:10E4F00090E0A9CF67E87BE086E391E124DA84E04D
:10E5000090E0A1CF64E87BE086E391E11CDA85E04E
:10E5100090E099CF69E57BE086E391E114DA86E04B
:10E5200090E091CF6CE57BE086E391E10CDA87E047
:10E5300090E089CF6FE57BE086E391E104DA88E043
:10E5400090E081CF62E67BE086E391E1FCD989E04F
:10E5500090E079CF80913B0C8823A1F062E07FE0CE
:10E5600082EA9FE051DB40918812509189126091BC
:10E570008A1270918B122AE082EA9FE07EDB82EAA7
:10E580009FE010DC8091881290918912A0918A12EC
:10E59000B0918B12873025E09207A105B10509F4EF
:10E5A0005AC208F07CC1893421E09207A105B10567
:10E5B00009F463C208F037C1843421E09207A10551
:10E5C000B10509F42DC208F017C1813421E092078A
:10E5D000A105B10509F409C208F000C180349140D9
:10E5E000A105B10509F4F8C164E670E080E090E0AF
:10E5F0000E94BE496CE271E080E090E00E94BE495A
:10E6000082E080934B1010924F1045C067E57BE08D
:10E6100082E491E198D91092811267E57BE0CE0106
:10E620000D9685DA67E57BE082E491E18CD911E013
:10E6300082EA9FE00E94F76920918112181619065C
:10E640000CF066C2211164C22AC20E94CA45182F6A
:10E65000882309F4A1C28091381281114FCD67E55A
:10E660007BE086E391E16FD980913B0C882361F0D8
:10E6700065E17FE082EA9FE0C7DA612F82EA9FE0EE
:10E68000AEDA82EA9FE08EDB812F0E9464851A3227
:10E6900011F0109238120E94F6496093040C7093A6
:10E6A000050C8093060C9093070C8CC08BEC9DE0BE
:10E6B0000E94D569809380128A3009F435C28D306A
:10E6C00009F432C29091811291112EC2682FCE01AD
:10E6D0000D96CDD80F5F1F4F65E070E080E090E0B1
:10E6E0000E94BE498BEC9DE00E94F769181619063E
:10E6F000ECF264E170E080E090E00E94BE49012B02
:10E7000009F01AC22091811289899A89222309F479
:10E7100002C2019709F03EC06CEE78E0CE0101968E
:10E7200006DABE016F5F7F4FCE010D960E94676BC8
:10E73000811130C26BE97BE0CE010796F8D9BE01AA
:10E74000695F7F4FCE010D960E94676B11E08111CA
:10E7500010E0CE01079621D9CE0101961ED91123D2
:10E7600099F040E050E0BE01635F7F4FCE0101961B
:10E770000E948C5EBE016F5F7F4F86E391E10E9435
:10E78000826BCE01019609D964E170E080E090E0EF
:10E790000E94BE49BE01635F7F4F82E491E1E8D8E9
:10E7A000CE010D96FAD86AE070E080E090E00E9419
:10E7B000BE498091461190914711892B09F445CFAC
:10E7C0000E9457088091B912882309F476C264E642
:10E7D00070E080E090E00E94BE496FC2823421E088
:10E7E0009207A105B10509F409C183349140A1053F
:10E7F000B10509F40CC1F8CE863421E09207A105D9
:10E80000B10509F41FC108F414C1873421E092074F
:10E81000A105B10509F41FC188349140A105B105D6
:10E8200009F422C1E1CE823025E09207A105B105AD
:10E8300009F4E4C0E8F4843721E09207A105B105AA
:10E8400009F424C138F482379140A105B10509F4D7
:10E85000D1CECACE811525E09207A105B10509F4F4
:10E86000BBC081309540A105B10509F4BEC0BCCE46
:10E87000843025E09207A105B10509F4D1C008F460
:10E88000C6C0853025E09207A105B10509F4D1C0C5
:10E8900086309540A105B10509F4D4C0A5CE873CCA
:10E8A00028E392072FEFA207B10509F4DDC008F0B5
:10E8B0003FC08D3F22E092072FEFA207B10509F478
:10E8C00099CEB8F4893025E09207A105B10509F485
:10E8D000D4C008F4C9C0823325E09207A105B10570
:10E8E00009F488CE84339540A105B10509F4CEC062
:10E8F0007BCE873E28E192072FEFA207B10509F4EE
:10E9000098C038F48F3E9041AF4FB10509F4A3C0D1
:10E910006BCE8D3D22E292072FEFA207B10509F4DD
:10E92000B5C08F3C9043AF4FB10509F479C05CCEC0
:10E930008D3922E692072FEFA207B10509F45ACECE
:10E9400038F5853B2AE492072FEFA207B10509F4B9
:10E9500043C078F48D3B9244AF4FB10509F044CEEB
:10E9600060E87BE082E491E10E94A36C84E190E0A6
:10E970006ACD8D3A22E592072FEFA207B10509F47F
:10E9800039CE853A9A45AF4FB10509F476C02CCE01
:10E99000873628E992072FEFA207B10579F170F4C5
:10E9A000873928E692072FEFA207B105F1F08538E5
:10E9B0009A47AF4FB10509F445C016CE8F3420EB0E
:10E9C00092072FEFA207B10511F18D33924CAF4F93
:10E9D000B10509F40FCE08CE68E57BE086E391E14E
:10E9E0000E94A36C8AEF9FEF2ECD6BE57BE086E360
:10E9F00091E10E94A36C89EF9FEF25CD6EE57BE04E
:10EA000086E391E10E94A36C88EF9FEF1CCD61E645
:10EA10007BE086E391E10E94A36C87EF9FEF13CD2B
:10EA200064E67BE086E391E10E94A36C86EF9FEFB2
:10EA30000ACD68E67BE086E391E10E94A36C85EF56
:10EA40009FEF01CD6CE67BE086E391E10E94A36C31
:10EA500084EF9FEFF8CC60E77BE086E391E10E94D2
:10EA6000A36C83EF9FEFEFCC64E77BE086E391E15B
:10EA70000E94A36C82EF9FEFE6CC68E77BE086E321
:10EA800091E10E94A36C81EF9FEFDDCC6CE77BE00E
:10EA900082E491E10E94A36C88EE9FEFD4CC82EADD
:10EAA0009FE00E94D569809380128A3041F08D30BA
:10EAB00031F0682FCE010D960E94376C22C08989F3
:10EAC0009A89892BF1F01093811262E97BE0CE01E3
:10EAD00007962DD8BE01635F7F4FCE0107960E9437
:10EAE000266CBC01CE0101961AD8CE0101960E9477
:10EAF000EE58CE0101960E94CD6CCE0107960E9481
:10EB0000CD6C6AE070E080E090E00E94BE4990CD5C
:10EB10002111F8CD04C0009709F0FBCD88C000E0BA
:10EB200010E0FF24F394DECD89899A89892B09F4BA
:10EB3000D3CDF0928112D0CD89899A89892B09F49D
:10EB4000E1CD6DE97BE0CE0107960E94976DBE0195
:10EB5000635F7F4FCE0107960E94266CBC01CE01F9
:10EB600001960E948F6DCE0101960E94EE58CE0153
:10EB700001960E94CD6CCE0107960E94CD6C8BEC65
:10EB80009DE00E948E6A64E170E080E090E00E9467
:10EB9000BE49B8CD10E0E0CD8091B912882309F4C8
:10EBA0006CC00E94F64928EEC22E23E0D22EE12C42
:10EBB000F12CA70196010E946798CA01B9010E9431
:10EBC0000D972091000C3091010C4091020C509156
:10EBD000030C0E94989820911802309119024091DC
:10EBE0001A0250911B020E944E9A18160CF045C052
:10EBF0000E94F649A70196010E946798CA01B901CF
:10EC00000E940D976093000C7093010C8093020C8E
:10EC10009093030C80918212909183120E94BA1DEE
:10EC200064E170E080E090E00E94BE49CBCD64E6F4
:10EC300070E080E090E00E94BE490E94F649CB015E
:10EC400068EE73E00E94DA9BCB0164E670E00E94FC
:10EC5000DA9B823691050CF4A3CD8091B912811113
:10EC60009FCD86E391E10E94EC6A613071058105D8
:10EC7000910509F095CD8FD393CD0E94F64900916F
:10EC8000040C1091050C2091060C3091070CDC014E
:10EC9000CB01801B910BA20BB30B88349E4EA105B8
:10ECA000B10508F48FCD1092361260E08BE292E14C
:10ECB0000E94BC4D1092E20485CD62960FB6F89486
:10ECC000DEBF0FBECDBFDF91CF911F910F91FF909F
:10ECD000EF90DF90CF900895AF92BF92CF92DF92E6
:10ECE000EF92FF920F931F93CF93DF93CDB7DEB7D1
:10ECF00062970FB6F894DEBF0FBECDBF7C01809146
:10ED00001F0D9091200D019731F067E57BE0C70161
:10ED10000E94976DF7C063EA7BE0CE0101960E94E6
:10ED2000976DBE016F5F7F4F8BEC9DE00E94F66D8B
:10ED300068EE73E080E090E00E94BE4916D664EF72
:10ED400071E080E090E00E94BE4984E6C82ED12C9C
:10ED50006EEA7BE0CE0107960E94976D8091461186
:10ED600090914711892B79F0A0904211B0904311F6
:10ED70006F817885C5010E94889E009721F08C01E3
:10ED80000A191B0902C00FEF1FEFCE0107960E9460
:10ED9000CD6CA8014F5F5F4F62E471E1CE01079631
:10EDA0000E948C5EBE01695F7F4FCE0101960E947A
:10EDB000826BCE0107960E94CD6C8D819E81892B3E
:10EDC00069F060E070E0CE0101960E94566B082E5B
:10EDD000000C990BC0970A9708F47DC010E062EF11
:10EDE0007EE0CE0107960E94876D44E150E06FEF10
:10EDF0007FEFCE0107960E949757CE0107960E949B
:10EE0000CD6C62E370E080E090E00E94BE4981E05A
:10EE1000C81AD10819F0112309F49ACF80913B0C3C
:10EE20008823E9F06CE97AE0CE0107960E94976D9D
:10EE3000BE016F5F7F4FCE0107960E94266CBC011A
:10EE4000CE010D960E948F6DCE010D9677D5CE0125
:10EE50000D960E94CD6CCE0107960E94CD6C8D81DF
:10EE60009E81892B61F060E070E0CE0101960E94E6
:10EE7000566B082E000C990BC0970A9730F060EB88
:10EE80007BE0C7010E94976D21C06CEB7BE0CE0157
:10EE900007960E94976DBE01695F7F4FCE01019674
:10EEA0000E94676B182FCE0107960E94CD6C11113E
:10EEB000E6CFF7011182108213821282158214822A
:10EEC000BE016F5F7F4FC7010E94826BCE0101962A
:10EED0000E94CD6C17C06CEB7BE0CE0107960E94C0
:10EEE000976DBE01695F7F4FCE0101960E94676BEF
:10EEF000082FCE0107960E94CD6C11E0002309F483
:10EF00006ECF6CCFC70162960FB6F894DEBF0FBE0E
:10EF1000CDBFDF91CF911F910F91FF90EF90DF90C8
:10EF2000CF90BF90AF9008958F929F92AF92BF9273
:10EF3000CF92DF92EF92FF920F931F93CF93DF93C5
:10EF40007C01862F9BE0E916F10409F070C09091D6
:10EF50009111992309F0F89462E10E94B342EC0107
:10EF600080919111882309F07894209709F074C05A
:10EF7000D0908C11C0908D116D2D70E080E090E0EC
:10EF80000E940F974B015C016C2D70E080E090E0D7
:10EF90000E940F972DEC3CEC4CEC5DE30E946E97C9
:10EFA0009B01AC01C501B4010E9499986093841142
:10EFB00070938511809386119093871110918E1113
:10EFC00000918F11612F6F7770E080E090E00E94D8
:10EFD0000F974B015C01602F70E080E090E00E9491
:10EFE0000F972DEC3CEC4CEC5DE30E946E979B017F
:10EFF000AC01C501B4010E94999817FD09C0609346
:10F0000088117093891180938A1190938B110BC092
:10F01000DC01CB01B0588093881190938911A093A3
:10F020008A11B0938B11DC0C1D0D100F6FC096E18F
:10F03000E916F10409F071C090919111992309F03A
:10F04000F89461E00E94B342EC0180919111882311
:10F0500009F078942097A9F080E090ECA9E7B4EC4F
:10F060008093841190938511A0938611B09387119A
:10F070008093881190938911A0938A11B0938B117A
:10F080004FC000918D11D0908C11602F70E07D29C0
:10F0900080E090E00E940D972DEC3CEC4CEC5DE3A1
:10F0A0000E946E97609384117093851180938611EE
:10F0B00090938711C0908F1110918E11812F8F77AF
:10F0C0006C2D70E0782B80E090E00E940D972DEC85
:10F0D0003CEC4CEC5DE30E946E9717FD09C0609319
:10F0E00088117093891180938A1190938B110BC0B2
:10F0F000DC01CB01B0588093881190938911A093C3
:10F100008A11B0938B110D0DC00E1C0D80919011C2
:10F11000811731F0CFEFDFEF03C0CFEFDFEF48C053
:10F12000CF3F9FEFD90709F411C1209709F01DC106
:10F130008090841190908511A0908611B0908711D5
:10F1400020E030E048EC52E4C501B4010E944E9A40
:10F1500018160CF007C1CBEFDFEF20E030E0A9017B
:10F16000C501B4010E94099787FF02C0CAEFDFEF13
:10F170008090881190908911A0908A11B0908B1185
:10F1800020E030E048EC52ECC501B4010E94099740
:10F1900087FF02C0C9EFDFEF20E030E040EF52E42C
:10F1A000C501B4010E944E9A181614F4C8EFDFEF9F
:10F1B0008CE0E816F10409F0E0C08CE50E94FB5EEB
:10F1C00080E090E00E94F75E0E94F55E65E08CE5CD
:10F1D0000E949363C82FD0E02097B1F0C530D105CD
:10F1E00084F000E010E08FE390E10E94DE63F8011C
:10F1F000EC55FD4E80870F5F1F4F0C171D079CF3CA
:10F2000006C0CDEFDFEFB9C0CEEFDFEFB6C0C091E3
:10F21000AC120091AD126C2F70E080E090E00E9483
:10F220000F976B017C01602F70E080E090E00E94FE
:10F230000F972DEC3CEC4CEC5DE30E946E979B012C
:10F24000AC01C701B6010E9499986093A412709313
:10F25000A5128093A6129093A712D091AE1210918E
:10F26000AF126D2F6F7770E080E090E00E940F97F3
:10F270006B017C01612F70E080E090E00E940F97AD
:10F280002DEC3CEC4CEC5DE30E946E979B01AC01D5
:10F29000C701B6010E949998D7FF5BC0DC01CB0182
:10F2A000B0588093A8129093A912A093AA12B09379
:10F2B000AB12802F8C0FC82FCD0FC10F8091B012D1
:10F2C0008C1344C0C090A412D090A512E090A61256
:10F2D000F090A71220E030E048EC52E4C701B601FC
:10F2E0000E944E9A18161CF4CBEFDFEF02C0C0E06C
:10F2F000D0E020E030E040EA50E4C701B6010E94CF
:10F30000099787FF02C0CAEFDFEFC090A812D09024
:10F31000A912E090AA12F090AB1220E030E040EF8A
:10F3200051ECC701B6010E94099787FF02C0C9EFDF
:10F33000DFEF20E030E040EF52E4C701B6010E9469
:10F340004E9A1816D4F4C8EFDFEF17C0CFEFDFEFF7
:10F3500014C06093A8127093A9128093AA1290937C
:10F36000AB12A7CFC0E0D0E0F8CE229619F0CCEFD8
:10F37000DFEF1ECFCEEFDFEF1BCFCE01DF91CF91BE
:10F380001F910F91FF90EF90DF90CF90BF90AF90C3
:10F390009F908F9008958F929F92AF92BF92CF923D
:10F3A000DF92EF92FF92CF93DF93CDB7DEB72C972A
:10F3B0000FB6F894DEBF0FBECDBF60ED7FE0CE018B
:10F3C00001960E94876D4CE251E06FEF7FEFCE0116
:10F3D00001960E941C57CE0101960E94CD6C60914F
:10F3E0008C0470918D0480914604909147049CDDBB
:10F3F00084E1882E912CA12CB12CE12CF12C8FEFE3
:10F40000E81AF80AC501B4010E94BE4960918C0453
:10F4100070918D04809146049091470485DD23E02E
:10F42000E216F10434F424E1820E911CA11CB11CFB
:10F43000E6CF2AE0E216F1041CF4892BA1F703C001
:10F44000892B09F08CC180914604909147048B3040
:10F450009105C9F48091881190918911A0918A1128
:10F46000B0918B118093B5129093B612A093B712FE
:10F47000B093B8128091841190918511A09186115A
:10F48000B09187111DC08631910521F30C9701F5CC
:10F490008091A8129091A912A091AA12B091AB12DA
:10F4A0008093B5129093B612A093B712B093B8128E
:10F4B0008091A4129091A512A091A612B091A712CA
:10F4C0008093B1129093B212A093B312B093B4127E
:10F4D0004091B5125091B6126091B7127091B81266
:10F4E00021E0CE0107960E94016D69E379E0CE012B
:10F4F00001960E94976DBE01695F7F4FCE01019614
:10F500000E94266CBC018AE291E10E94B86CCE0197
:10F5100001960E94CD6CCE0107960E94CD6C409161
:10F52000B1125091B2126091B3127091B41221E0F5
:10F53000CE0107960E94016D6FE779E0CE0101963A
:10F540000E94976DBE01695F7F4FCE0101960E94B8
:10F55000266CBC018AE291E10E94586CCE010196B2
:10F560000E94CD6CCE0107960E94CD6C61E07BE0DD
:10F570008AE291E10E944A6C67E57BE0CE01019648
:10F580000E94976D44E150E060E070E0CE0101968A
:10F590000E944D58CE0101960E94CD6CC090B512CC
:10F5A000D090B612E090B712F090B81220E030E0A0
:10F5B000A901C701B6010E944E9A20E030E040E068
:10F5C0005FE387FD05C0C701B6010E94999804C09A
:10F5D000C701B6010E9498980E94F8992AE0AB01F1
:10F5E000BC01CE0101960E94306DBE016F5F7F4F5E
:10F5F00084E291E10E94826BCE0101960E94CD6C63
:10F6000060E087E00E94165F64E271E18BE292E1C4
:10F610000E94F66D6FED8BE292E10E94EF6D65E85E
:10F6200079E08BE292E10E94F56E6091B1127091E7
:10F63000B2128091B3129091B4120E94F8994AE0EC
:10F6400050E08BE292E10E94CC6E61E07BE08BE2C5
:10F6500092E10E94F56E64E670E080E090E00E9426
:10F66000BE49C090B512D090B612E090B712F0909B
:10F67000B81220E030E040EF51E4C701B6010E942B
:10F680004E9A87FD03C061EC7FE054C020E030E07B
:10F6900040ED51E4C701B6010E944E9A87FD1FC09C
:10F6A00061EB7FE0CE0101960E94876D4AE050E059
:10F6B0006FEF7FEFCE0101960E941C57CE0101969D
:10F6C0000E94CD6C80917404882331F06CED75E05C
:10F6D00080E090E00E94BE4961EA7FE02BC020E01C
:10F6E00030E040EB51E4C701B6010E944E9A87FD1D
:10F6F00003C063E97FE01EC064E87FE0CE010196AD
:10F700000E94876D4AE050E06FEF7FEFCE010196D7
:10F710000E941C57CE0101960E94CD6C809174040A
:10F72000882331F06CED75E080E090E00E94BE49E6
:10F7300066E77FE0CE0101960E94876D4AE050E0C7
:10F740006FEF7FEFCE0101960E941C57CE0101960C
:10F750000E94CD6C62E370E080E090E0DCC00E942B
:10F76000CC566EE170E080E090E00E94BE490E94BD
:10F7700054426B017C0164E670E080E090E00E94FE
:10F78000BE4969E379E08AE291E10E94A36C21E03D
:10F79000B701A601CE0101960E94016DBE016F5F07
:10F7A0007F4F8AE291E10E94586CCE0101960E943F
:10F7B000CD6C6AE271E1CE0101960E948F6D4AE044
:10F7C00050E060E070E0CE0101960E944D58CE01FD
:10F7D00001960E94CD6C80911202882379F080916D
:10F7E000E204882359F06FED8BE292E10E94EF6D05
:10F7F00066ED79E08BE292E10E94F56E65ED79E0CD
:10F800008AE291E10E944A6CC092B512D092B6127F
:10F81000E092B712F092B81220E030E040EF51E4ED
:10F82000C701B6010E944E9A87FD03C066E67FE0DD
:10F8300054C020E030E040ED51E4C701B6010E9421
:10F840004E9A87FD1FC066E57FE0CE0101960E94BB
:10F85000876D4AE050E06FEF7FEFCE0101960E9486
:10F860001C57CE0101960E94CD6C809174048823B0
:10F8700031F06CED75E080E090E00E94BE4966E4F6
:10F880007FE02BC020E030E040EB51E4C701B6013F
:10F890000E944E9A87FD03C068E37FE01EC069E2C4
:10F8A0007FE0CE0101960E94876D4AE050E06FEF45
:10F8B0007FEFCE0101960E941C57CE0101960E9457
:10F8C000CD6C80917404882331F06CED75E080E09C
:10F8D00090E00E94BE496BE17FE0CE0101960E945C
:10F8E000876D4AE050E06FEF7FEFCE0101960E94F6
:10F8F0001C57CE0101960E94CD6C6CE271E080E055
:10F9000090E00E94BE4980917404882331F068EE33
:10F9100073E080E090E00E94BE492C960FB6F89408
:10F92000DEBF0FBECDBFDF91CF91FF90EF90DF9094
:10F93000CF90BF90AF909F908F900895CF93DF931B
:10F94000FC0124813581232B69F0EC01BC0182EAA2
:10F950009FE00E94E56EBE018BEC9DE0DF91CF91B0
:10F960000C94E56EDF91CF910895FF920F931F9352
:10F97000CF93DF93CDB7DEB72C970FB6F894DEBFE9
:10F980000FBECDBF1092811267E57BE0CE010196DC
:10F990000E94976D67E57BE082E491E10E94A36C91
:10F9A00000E010E0FF24F3948BEC9DE00E94F769E7
:10F9B000181619062CF480918112882309F443C08B
:10F9C00062E370E080E090E00E94BE49012B51F0BC
:10F9D0008BEC9DE00E948E6A64E670E080E090E02F
:10F9E0000E94BE4980918112811104C08D819E8147
:10F9F000892BC9F080913B0C882371F0BE016F5FA9
:10FA00007F4FCE0107960E948F6DCE01079696DF3D
:10FA1000CE0107960E94CD6CBE016F5F7F4F82E4DE
:10FA200091E10E94B86CCE0101960E94CD6C2C969B
:10FA30000FB6F894DEBF0FBECDBFDF91CF911F91FF
:10FA40000F91FF9008958BEC9DE00E94D569809303
:10FA500080128A3071F08D3061F090918112911195
:10FA600008C0682FCE0101960E94376C0F5F1F4FB0
:10FA700006C08D819E81892B11F0F09281126FE07A
:10FA800070E080E090E00E94BE498ECF1F93CF933C
:10FA9000DF93182FCFE2DDE0812F0E947449899314
:10FAA00099936CE370E080E090E00E94BE498DE0A5
:10FAB000CF37D80789F70E94466020E030E040EA5F
:10FAC00050E40E946E9720E030E040E85AE30E9444
:10FAD0006E97DF91CF911F9108952F923F924F9291
:10FAE0005F926F927F928F929F92AF92BF92CF92CE
:10FAF000DF92EF92FF920F931F93CF93DF93CDB7D7
:10FB0000DEB7C954D1090FB6F894DEBF0FBECDBF22
:10FB10002B013C0127962FAF279728963FAF2897B8
:10FB200029964FAF29972A965FAF2A970E94F649E8
:10FB300022966CAF7DAF8EAF9FAF229727962FADE9
:10FB4000279728963FAD289729964FAD29972A9653
:10FB50005FAD2A9780E9481681E058066104710478
:10FB600034F060E9462E55245394612C712C2031D9
:10FB700097E23907410551052CF42DA73EA74FA761
:10FB800058AB0AC090E1C92E97E2D92EE12CF12C96
:10FB9000CDA6DEA6EFA6F8AA8091B912882321F09F
:10FBA0002DA73EA74FA758AB22966CAD7DAD8EAD6D
:10FBB0009FAD229728EE33E040E050E00E943B9852
:10FBC00026962CAF3DAF4EAF5FAF269721E02DAB11
:10FBD00019A61AA61BA61CA68E01035F1F4FCC24D4
:10FBE000DD247601C418D508E608F708C9AADAAA00
:10FBF000EBAAFCAAC9A4DAA4EBA4FCA42DA53EA5FB
:10FC00004FA558A9C216D306E406F5060CF031C379
:10FC100069A57AA58BA59CA50E940F9720E030E0EE
:10FC20004AE754E40E945F99AB01BC0123E0C8019C
:10FC30000E94016DB80184E291E10E94826BC801CB
:10FC40000E94CD6C2DA53EA54FA558A92A3031059F
:10FC50004105510594F42AE026964CAD5DAD6EAD9C
:10FC60007FAD2697C8010E94306DB80184E291E112
:10FC70000E94826BC8010E94CD6CCE0101960E9449
:10FC8000FB4366EE7FE08AE291E10E945E6CAE018A
:10FC90004F5F5F4F1A01C12CD12C7601D1018D909D
:10FCA0009D90AD90BD901D01A5019401C501B401C9
:10FCB0000E946E979B01AC01C701B6010E94999802
:10FCC0006B017C0123E0B501A401C8010E94D26C44
:10FCD000B801CE0143960E948F6D6AEC79E0CE01A7
:10FCE00043960E940F6CBC018AE291E10E94586C1D
:10FCF000CE0143960E94CD6CC8010E94CD6C2016A7
:10FD0000310661F6C701B6010E945D9B6B017C0163
:10FD1000BDE24B16B1E05B066104710434F00E9451
:10FD2000CC5660E080E00E94165F23E0B701A60198
:10FD3000CE0143960E94016D64E27BE0C8010E94FF
:10FD4000976D64E271E1C8010E94266C64EC7BE06F
:10FD50000E940F6CBE016D5E7F4F0E94266C69ECA5
:10FD60007BE00E940F6CBC018AE291E10E94586C1A
:10FD7000C8010E94CD6CCE0143960E94CD6C2DEC43
:10FD80003CEC4CE45FE3C701B6010E944E9A298126
:10FD90003A814B815C812DA33EA34FA358A718162F
:10FDA0000CF0ABC12AE939E949E95FE3C701B601C3
:10FDB0000E94099787FFA1C1CDA8CC2009F49DC15D
:10FDC00089849A84AB84BC8420E030E0A901C50119
:10FDD000B4010E940997CD80DE80EF80F8848823EB
:10FDE00009F12DA13EA14FA158A5CA01B9010E9458
:10FDF0006E976EAB7FAB88AF99AFA7019601C70135
:10FE0000B6010E946E979B01AC016EA97FA988ADD7
:10FE100099AD0E9499980E945D9BA50194010E9452
:10FE20000C9904C06BED7FE089EC9FE320EE3EE28D
:10FE300045E652E40E946E976EAB7FAB88AF99AFF8
:10FE400020E030E0A901C701B6010E94099788238C
:10FE500009F12DA13EA14FA158A5CA01B9010E94E7
:10FE60006E976AAF7BAF8CAF9DAFA5019401C501C2
:10FE7000B4010E946E979B01AC016AAD7BAD8CAD65
:10FE80009DAD0E9499980E945D9BA70196010E94DA
:10FE90000C9904C06BED7FE089EC9FE320EE3EE21D
:10FEA00045E652E40E946E976AAF7BAF8CAF9DAF80
:10FEB00020E030E0A9016DA17EA18FA198A50E944C
:10FEC00009978823F9F0A5019401C501B4010E94A6
:10FED0006E974B015C01A7019601C701B6010E9414
:10FEE0006E979B01AC01C501B4010E9499980E94D4
:10FEF0005D9B2DA13EA14FA158A50E940C996B01BD
:10FF00007C0108C08BEDC82E8FE0D82E89ECE82E3E
:10FF10008FE3F82E65E27BE0C8010E94976D64E2F2
:10FF200071E1C8010E94266C6CEC7BE00E940F6CB2
:10FF3000BC018AE291E10E94B86CC8010E94CD6CBC
:10FF400065E27BE0C8010E94976D64E271E1C8013F
:10FF50000E94266C66EE7BE00E940F6CBC0184E27E
:10FF600091E10E94B86CC8010E94CD6C21E04EA9BD
:10FF70005FA968AD79ADCE014F960E94016D21E079
:10FF80004AAD5BAD6CAD7DADCE0149960E94016D71
:10FF900020EE3EE245E652E4C701B6010E946E97AC
:10FFA000AB01BC0121E0C8010E94016DB801CE0186
:10FFB00043960E948F6D6AEC79E0CE0143960E94D1
:10FFC0000F6CBE01675E7F4F0E94266C6AEC79E081
:10FFD0000E940F6CBE01615E7F4F0E94266CBC01C7
:10FFE0008EE191E10E94B86CCE0143960E94CD6CE7
:10FFF000C8010E94CD6CCE0149960E94CD6CCE0105
:020000021000EC
:100000004F960E94CD6C2DE2421621E0520661040B
:10001000710474F469A57AA58BA59CA525E030E050
:1000200040E050E00E943B98672B682B692BC1F59C
:1000300064E271E1C8010E948F6D45E050E06FEF0E
:100040007FEFC8010E949757C8010E94CD6C6FEEE8
:100050007BE0C8010E94976D45E050E061EF7FEFC3
:10006000C8010E944D58C8010E94CD6C67E57BE035
:10007000C8010E94976DC8010E94F056C8010E94F5
:10008000CD6C6EE171E1C8010E948F6D45E050E0DA
:1000900060E070E0C8010E941C57C8010E94CD6C4E
:1000A0006EE171E18AE291E10E94586C3FE14316F2
:1000B00051046104710434F4C9A4DAA4EBA4FCA4CF
:1000C000F7FC10C06AE271E1C8010E948F6DC8019F
:1000D00035DCC8010E94CD6C67E57BE08AE291E1E6
:1000E0000E94A36CB201C30177FE04C069A97AA97A
:1000F0008BA99CA90E94BE49A9C023E04DA15EA185
:100100006FA178A5CE0143960E94016D65E27BE068
:10011000C8010E94976D64E271E1C8010E94266CDB
:1001200061EF7BE00E940F6CBE016D5E7F4F0E940D
:10013000266C6AEC7BE00E940F6CBC0184E291E1CA
:100140000E94B86CC8010E94CD6CCE0143960E94FB
:10015000CD6C49855A856B857C8523E0CE01499617
:100160000E94D26C4D815E816F81788523E0C80149
:100170000E94D26CB801CE0143960E948F6D66EF4B
:100180007BE0CE0143960E940F6CBE01675E7F4FFD
:100190000E94266C6AEC7BE00E940F6CBC018EE131
:1001A00091E10E94B86CCE0143960E94CD6CC801CB
:1001B0000E94CD6CCE0149960E94CD6C2DE2421674
:1001C00021E052066104710474F469A57AA58BA537
:1001D0009CA525E030E040E050E00E943B98672B72
:1001E000682B692BF1F464E271E1C8010E948F6D04
:1001F0004AE050E06FEF7FEFC8010E949757C801B7
:100200000E94CD6C6EE171E1C8010E948F6D4AE0E1
:1002100050E060E070E0C8010E941C57C8010E94D5
:10022000CD6C6AE271E1C8010E948F6DC80186DB66
:10023000C8010E94CD6C67E57BE08AE291E10E94F3
:10024000A36CC301B2010E94BE491DAA0E94F649D7
:100250006B017C0122962CAD3DAD4EAD5FAD22977A
:10026000C21AD30AE40AF50AC9A6DAA6EBA6FCA6C6
:10027000C1CC64E271E1CE010D960E948F6D4AE01F
:1002800050E06FEF7FEFCE010D960E944D58CE01EA
:100290000D960E94CD6CCDA8CC20B1F16FEE7BE025
:1002A000CE010D960E94976D45E050E061EF7FEF23
:1002B000CE010D960E944D58CE010D960E94CD6C38
:1002C0008091B912882391F06EED7FE0CE010D96FA
:1002D0000E94876D45E050E060E070E0CE010D9631
:1002E0000E944D58CE010D960E94CD6C67E57BE0D3
:1002F000CE010D960E94976DCE010D960E94F0568C
:10030000CE010D960E94CD6C6EE171E1CE010D968D
:100310000E948F6D4AE050E06FEF7FEFCE010D96A7
:100320000E941C57CE010D960E94CD6CC75BDF4F1B
:100330000FB6F894DEBF0FBECDBFDF91CF911F91F6
:100340000F91FF90EF90DF90CF90BF90AF909F9074
:100350008F907F906F905F904F903F902F90089577
:100360000C94C19CCF92DF92EF92FF920F931F9358
:10037000CF93DF93CDB7DEB72C970FB6F894DEBFDF
:100380000FBECDBF88E69EE00E943E7064E670E03E
:1003900080E090E00E94BE4967E370E184E291E171
:1003A0000E945E6C64E271E1CE0101960E948F6D45
:1003B00044E150E060E070E0CE0101960E944D58AB
:1003C000CE0101960E94CD6C68E270E184E291E179
:1003D0000E945E6C64E271E1CE0101960E948F6D15
:1003E00044E150E06FEF7FEFCE0101960E941C5771
:1003F000CE0101960E94CD6C8CE40E948F626B014D
:100400007C0104E010E0A7019601C701B6010E943B
:100410009E9B882309F484C00150110961F068ECA7
:1004200070E080E090E00E94BE498CE40E948F6200
:100430006B017C01E8CF6DE170E184E291E10E9403
:100440005E6C64E271E1CE0101960E948F6D4AE01C
:1004500050E060E070E0CE0101960E944D58CE0160
:1004600001960E94CD6C6AEB79E0CE0101960E9464
:10047000976D64E271E1CE0101960E94266CBC0189
:100480008AE291E10E94B86CCE0101960E94CD6C87
:100490008091390C90913A0C039721F410923A0C08
:1004A0001092390C82E090E09093330480933204F0
:1004B00025C067E57BE080E391E10E94A36C60E3E7
:1004C00071E1CE0101960E948F6D6AEC79E0CE0158
:1004D00001960E940F6C6AE271E10E94266CBC01D9
:1004E0008AE291E10E94B86CCE0101960E94CD6C27
:1004F00083E090E090933A0C8093390C64E670E0CE
:1005000080E090E00E94BE498091B912882309F4EE
:10051000CAC060E273E080E090E00E94BE49C3C0C0
:1005200021E0B701A601CE0101960E94016D6CEC9D
:1005300079E0CE0107960E94976DBE016F5F7F4FF5
:10054000CE0107960E94266CBC018AE291E10E94CE
:10055000B86CCE0107960E94CD6CCE0101960E9428
:10056000CD6C6AE271E1CE0101960E948F6D42E38B
:1005700050E06FEF7FEFCE0101960E941C57CE0135
:1005800001960E94CD6C66ED79E0CE0101960E9445
:10059000976DCE0101960E94F056CE0101960E9401
:1005A000CD6C65ED79E08AE291E10E944A6C86E6C5
:1005B0000E948F626B017C0104E010E0A7019601AC
:1005C000C701B6010E949E9B882381F0015011094A
:1005D00009F46FCF68EC70E080E090E00E94BE49C3
:1005E00086E60E948F626B017C01E8CF21E0B701B3
:1005F000A601CE0101960E94016D69E379E0CE016A
:1006000007960E94976DBE016F5F7F4FCE010796E0
:100610000E94266CBC0180E391E10E94B86CCE017F
:1006200007960E94CD6CCE0101960E94CD6C6AECBB
:1006300079E0CE0101960E94976D60E371E1CE01F1
:1006400001960E94266CBC0184E291E10E94B86C84
:10065000CE0101960E94CD6C64E271E1CE0101965B
:100660000E948F6D4AE050E06FEF7FEFCE01019660
:100670000E949757CE0101960E94CD6C66ED79E0FD
:10068000CE0101960E94976DCE0101960E94F05610
:10069000CE0101960E94CD6C65ED79E080E391E199
:1006A0000E944A6C0CCF2C960FB6F894DEBF0FBE9A
:1006B000CDBFDF91CF911F910F91FF90EF90DF9011
:1006C000CF9008950895CF93DF930E9420601092F9
:1006D000301280913412823018F098E090933012EA
:1006E00090913512992339F0813029F4809130129C
:1006F00084608093301262E370E080E090E00E94BA
:10070000BE49609136128BE292E10E94BC4D68EEC8
:1007100073E080E090E00E94BE4960E38BE292E1EA
:100720000E94D74DCBE4D6E4CE010197F1F760E308
:100730008BE292E10E94D74D2197F1F760E38BE2C3
:1007400092E10E94D74D83E592E00197F1F760E2D4
:100750008BE292E10E94D74D8091301280620E941C
:10076000055F84E0809331128CE00E94055F81E098
:100770000E94055FCBE3DFE1CE010197F1F782E054
:100780008093321286E00E94055F82E00E94055F3E
:100790002197F1F7DF91CF910895FF920F931F9367
:1007A000CF93DF93CDB7DEB72B970FB6F894DEBFAC
:1007B0000FBECDBF85E09FE00E943E7040E855E24D
:1007C00060E070E085E09FE00E94255E64E670E0F6
:1007D00080E090E00E94BE498CED95E0A0E0B0E0A2
:1007E0008093090F90930A0FA0930B0FB0930C0FF7
:1007F00064E670E080E090E00E94BE498FEF89835C
:1008000081E08A8386E88B831C821D821E821F8280
:10081000188689E7898785E09FE00E948E6A62E3F7
:1008200070E080E090E00E94BE4985E09FE00E9479
:10083000C66908974CF049E050E0BE016F5F7F4FFA
:1008400085E09FE00E94826962E370E080E090E0D2
:100850000E94BE4985E09FE00E94F769892B09F15B
:1008600085E09FE00E94C66908978CF465E070E01F
:1008700080E090E00E94BE4900E010E0F12C85E0AD
:100880009FE00E94F76902301105ACF50CC049E009
:1008900050E0BE016F5F7F4F85E09FE00E9482695C
:1008A000E5CFF12C28C085E09FE00E94F769892BF5
:1008B000A1F465E070E080E090E00E94BE49023063
:1008C0001105E9F69A8589819813D9CF9B858B818B
:1008D0009813D5CFFF24F394D2CF85E09FE00E94F8
:1008E000D569EAE0F0E0EC0FFD1FE00FF11F808317
:1008F0000F5F1F4FDECF62E370E080E090E00E9468
:10090000BE4985E09FE00E943E708F2D2B960FB66A
:10091000F894DEBF0FBECDBFDF91CF911F910F9135
:10092000FF9008958091241190912511009711F066
:100930000C945A9260E070E0CB010895AF92BF92A0
:10094000CF92DF92EF92FF920F931F93CF93DF939B
:100950002091461130914711FC0144815581890154
:10096000041B150B4115510559F12115310541F1B4
:100970002417350728F10217130718F089010150D1
:1009800011097C01A0904211B0904311C501DFEF25
:10099000CFEF6501C00ED11EC816D906A0F0F70131
:1009A000608171810E94889E009769F09C012A19DC
:1009B0003B090217130710F0D22FC32F0196ECCF7B
:1009C0008FEF9FEF02C08D2F9C2FDF91CF911F9152
:1009D0000F91FF90EF90DF90CF90BF90AF90089570
:1009E0008F929F92AF92BF92CF92DF92EF92FF923F
:1009F0000F931F93CF93DF93DB01CD91DC91DC014B
:100A00001C96ED91FC911D97CE17DF070CF04AC0A4
:100A1000FE01EE0FFF1F1A968D919C911B97E80F18
:100A2000F91F80809180C170DD27B1E0CB2720972E
:100A300019F404E610E002C00CE91FEF79015A0135
:100A40006B01020F131FB801C4010E941965892BA5
:100A500099F40E0D1F1DB801C4010E941965892B60
:100A600071F4B8016E0D7F1DC4010E941965892BB8
:100A7000E1F023E030E005C021E030E002C022E0F8
:100A800030E0F5018081918101968217930734F05F
:100A900011821082F6018081918101969183808379
:100AA000CE0105C081E090E002C08FEF9FEFDF91A3
:100AB000CF911F910F91FF90EF90DF90CF90BF905B
:100AC000AF909F908F900895CF92DF92EF92FF9218
:100AD0000F931F93CF93DF93CDB7DEB728970FB651
:100AE000F894DEBF0FBECDBF823409F441C0CCF410
:100AF000803309F45DC07CF4833209F450C08A323B
:100B000009F076C06FE87BE082E491E10E94A36C7B
:100B10008FEF9FEF6AC0813309F459C08134E9F047
:100B200067C08136D1F02CF4833469F1843439F014
:100B30005FC0833641F1E4F0843609F059C08091FA
:100B40003A1190913B11892B09F4F1C086E391E1B0
:100B50000E94EC6A97FF81C0EAC063E87BE082E410
:100B600091E10E94A36C8091330C9091340C3DC0B4
:100B700066E87BE082E491E10E94A36C1092B912D6
:100B80008CEF9FEF32C069E87BE082E491E10E9444
:100B9000A36C81E08093B9128DEF9FEF26C06CE8C3
:100BA0007BE082E491E10E94A36C8EEF9FEF1DC079
:100BB00062EC7BE086E391E10E94A36C62EC7BE057
:100BC00082E491E10E94A36C80E090E00EC060E9B5
:100BD0007BE086E391E10E94A36C60E97BE082E424
:100BE00091E10E94A36C81E090E00E94BA1DA5C033
:100BF0001A8219821C821B821E821D828F83188694
:100C0000BE01695F7F4FCE0101960E94A36CBE01B9
:100C10006F5F7F4F86E391E10E94826BCE01019668
:100C20000E94CD6C60E070E086E391E10E94566B1B
:100C3000082E000C990B0E94419E892B39F086E307
:100C400091E10E94EC6ACB010E94BA1D64E670E05B
:100C500080E090E00E94BE4970C080913B0C8823E8
:100C600061F069EF7BE082EA9FE00E94F56E66E347
:100C700071E182EA9FE00E94E56E86E391E10E94C5
:100C8000EC6A0AEF1FEF2FEF3FEF68017901C61AF8
:100C9000D70AE80AF90AB701A6012AE0CE010196AF
:100CA0000E94306D33C08FEFE81AF80A85E6E81627
:100CB000F10459F06EE170E080E090E00E94BE49DE
:100CC0000E94CA45182F112371F380913B0C882391
:100CD00079F069EF7BE082EA9FE00E94F56E612F78
:100CE00082EA9FE00E94EF6D82EA9FE00E94D26E4E
:100CF00010330CF414516AE270E0611B710917FDA6
:100D000073954AE0CE0101960E945C6DBE016F5F53
:100D10007F4F86E391E10E94826BCE0101960E9493
:100D2000CD6C86E391E10E94EC6ACB015ECF0E941C
:100D3000CA45182FE12CF12CC6CF28960FB6F8948F
:100D4000DEBF0FBECDBFDF91CF911F910F91FF90FE
:100D5000EF90DF90CF900895CF92DF92EF92FF92C5
:100D60000F931F93E82FF92F05C001501109210996
:100D7000310961F1908196239417B9F305C00150B0
:100D800011092109310911F1908196239413F7CFAC
:100D9000C12CD12CE12CF12C0AC08FEFC81AD80A33
:100DA000E80AF80A0C151D052E053F0579F080812B
:100DB0008623841791F36C2D7D2D8E2D9F2D1F91F1
:100DC0000F91FF90EF90DF90CF90089560E070E07A
:100DD00080E090E01F910F91FF90EF90DF90CF9017
:100DE0000895CF93DF93CDB7DEB762970FB6F8942F
:100DF000DEBF0FBECDBF789484B5826084BD84B55C
:100E0000816084BD85B5826085BD85B5816085BD05
:100E100080916E00816080936E00109281008091BD
:100E20008100826080938100809181008160809345
:100E30008100809180008160809380008091B1006A
:100E400084608093B1008091B00081608093B00095
:100E500080919100826080939100809191008160E7
:100E600080939100809190008160809390008091A8
:100E7000A10082608093A1008091A1008160809395
:100E8000A1008091A00081608093A0008091210149
:100E900082608093210180912101816080932101F2
:100EA0008091200181608093200180917A0084608C
:100EB00080937A0080917A00826080937A0080919A
:100EC0007A00816080937A0080917A0080688093B4
:100ED0007A001092C10061E089E10E94354961E029
:100EE00089E10E9403490E9420606FE17AE082EA72
:100EF0009FE00E94D56E37E2C32ED12CE12CF12C5D
:100F000000E010E08C2D0E94FB5E0E94F55E8111D6
:100F100027C06BE27AE082EA9FE00E94F56E20E152
:100F2000B701A60182EA9FE00E943D6E82EA9FE03F
:100F30000E94D26EC0922F1267E47AE082EA9FE0AC
:100F40000E94F56E20E1B701A60182EA9FE00E94AF
:100F50003D6E82EA9FE00E94D26E0F5F1F4F13C06A
:100F6000843089F461E67AE082EA9FE00E94F56EBF
:100F700020E1B701A60182EA9FE00E943D6E82EA6D
:100F80009FE00E94D26E8FEFC81AD80AE80AF80ACA
:100F9000E0E4CE16D104E104F10409F0B3CF012B53
:100FA00019F46CE77AE002C062E97AE082EA9FE035
:100FB0000E94D56E88DB80E40E94055F05E714E09F
:100FC000F80161918F018BE292E10E94ED4DF4E016
:100FD0000D371F07A9F70E94CC560E94C44E8EED14
:100FE00093E09093650C8093640C0E942598809305
:100FF000A70C8FED93E00E9425988093A80C809118
:10100000A70C9091A80C1816190654F410927404A9
:10101000019731F41092A80C1092A70C0E946862FC
:1010200063EB7AE0CE0101960E94876D4AE050E0C2
:101030006FEF7FEFCE0101960E944D58CE010196D1
:101040000E94CD6C40E052EC61E070E082EA9FE0EB
:101050000E94255E80917404882331F068EE73E06D
:1010600080E090E00E94BE4982EA9FE00E94D5693C
:10107000182F823709F4B6C11092650C1092640CD7
:1010800029EAC22E2CE0D22EE12CF12CC7010E94BD
:101090002598F60181936F01FFEFEF1AFF0A86E8AA
:1010A000E816F10499F78091A90C9091AA0CA091EF
:1010B000AB0CB091AC0C85369105A105B1050CF4D3
:1010C00091C18093700490937104A0937204B093C3
:1010D00073048091AD0C9091AE0CA091AF0CB091C7
:1010E000B00C80936C0490936D04A0936E04B09345
:1010F0006F048091B10C9091B20CA091B30CB0919F
:10110000B40C8093680490936904A0936A04B0932C
:101110006B0465EC7CE0CE0101960E94976DBE01E8
:101120006F5F7F4F85E292E10E94826BCE01019654
:101130000E94CD6C63E27DE0CE0101960E94976D26
:10114000BE016F5F7F4F8FE192E10E94826BCE0103
:1011500001960E94CD6C23E030E040E050E065E273
:1011600072E1CE0101960E94AB6D23E030E040E0D9
:1011700050E06FE172E1CE0107960E94AB6D2B85C6
:101180003C858D819E812817390729F58F819885A7
:1011900069817A81009719F061157105B9F46115BB
:1011A000710559F02115310541F0FB01208130E036
:1011B00088279927821B930B0BC0009771F0232B74
:1011C00061F0FC019081892F90E002C00E945B9E3B
:1011D00001E0892B19F000E001C001E0CE01079683
:1011E0000E94CD6CCE0101960E94CD6C011106C00B
:1011F00065E272E18FE192E10E94B86C8091B50CDA
:101200009091B60CA091B70CB091B80C8093640487
:1012100090936504A0936604B09367048091B90C21
:101220009091BA0CA091BB0CB091BC0C809360045F
:1012300090936104A0936204B09363048091BD0C09
:101240009091BE0CA091BF0CB091C00C80935C0437
:1012500090935D04A0935E04B0935F048091C10CF1
:101260009091C20CA091C30CB091C40C809358040F
:1012700090935904A0935A04B0935B048091CD0CD1
:101280009091CE0CA091CF0CB091D00C8093C4045F
:101290009093C504A093C604B093C7048091D10C69
:1012A0009091D20CA091D30CB091D40C8093C00437
:1012B0009093C104A093C204B093C3048091D50C51
:1012C0009091D60CA091D70CB091D80C8093540477
:1012D00090935504A0935604B09357048091D90C71
:1012E0009091DA0CA091DB0CB091DC0C809350044F
:1012F00090935104A0935204B09353048091DD0C59
:101300009091DE0CA091DF0CB091E00C80934C0426
:1013100090934D04A0934E04B0934F04C090F30CEF
:10132000D090F40CE090F50CF090F60CA70196012B
:10133000C701B6010E949E9B811108C0C09248045B
:10134000D0924904E0924A04F0924B0460911F0D40
:101350007091200D072E000C880B990B0E940F979F
:101360009B01AC010E949E9B882321F01092200DCE
:1013700010921F0DE090210DF090220DB7010F2C5F
:10138000000C880B990B0E940F979B01AC010E94E7
:101390009E9B811104C0F0924704E0924604E12C28
:1013A000F12CF701E950F34F80809180A280B38047
:1013B000A5019401C501B4010E949E9B811107C043
:1013C000F701E45CF34F80829182A282B382F4E061
:1013D000EF0EF11C88E2E816F10419F781E090E0C5
:1013E0000E9417500EE8010F023080F01E3671F097
:1013F0008091A90C9091AA0CA091AB0CB091AC0C6F
:1014000085369105A105B1050CF053C1809170049A
:1014100090917104A0917204B09173048093A90C0F
:101420009093AA0CA093AB0CB093AC0C80916C047D
:1014300090916D04A0916E04B0916F048093AD0CF7
:101440009093AE0CA093AF0CB093B00C8091680455
:1014500090916904A0916A04B0916B048093B10CDF
:101460009093B20CA093B30CB093B40C1337B1F0BB
:1014700085EC9CE0009739F048E050E0BC0185E243
:1014800092E10E940B4783E29DE0009739F04CE027
:1014900050E0BC018FE192E10E940B47809164040F
:1014A00090916504A0916604B09167048093B50C97
:1014B0009093B60CA093B70CB093B80C80916004D5
:1014C00090916104A0916204B09163048093B90C7F
:1014D0009093BA0CA093BB0CB093BC0C80915C04AD
:1014E00090915D04A0915E04B0915F048093BD0C67
:1014F0009093BE0CA093BF0CB093C00C8091580485
:1015000090915904A0915A04B0915B048093C10C4E
:101510009093C20CA093C30CB093C40C8091C404EC
:101520009091C504A091C604B091C7048093CD0CDE
:101530009093CE0CA093CF0CB093D00C8091C004AC
:101540009091C104A091C204B091C3048093D10CC6
:101550009093D20CA093D30CB093D40C80915404EC
:1015600090915504A0915604B09157048093D50CE6
:101570009093D60CA093D70CB093D80C80915004C4
:1015800090915104A0915204B09153048093D90CCE
:101590009093DA0CA093DB0CB093DC0C80914C049C
:1015A00090914D04A0914E04B0914F048093DD0CB6
:1015B0009093DE0CA093DF0CB093E00C8091480474
:1015C00090914904A0914A04B0914B048093F30C8C
:1015D0009093F40CA093F50CB093F60C8091460414
:1015E000909147049093220D8093210DECE3FCE051
:1015F000A7EFBCE041915191619171914D935D9341
:101600006D937D938CE0E436F807A1F76DE97AE0FD
:10161000CE0101960E94876DCE0101960E94EE5880
:10162000CE0101960E94CD6C84E3C82E84E0D82EB2
:1016300091EEA92E9CE0B92EE12CF12C809134047E
:10164000909135048E159F0554F1F60180819181AA
:10165000F501819391935F0180913B0C8823C1F048
:101660006CE97AE082EA9FE00E94F56E4AE050E081
:10167000B70182EA9FE00E94CC6E69E97AE082EAD3
:101680009FE00E94F56EF601808191810E94774370
:10169000FFEFEF1AFF0A82E0C80ED11CCFCF023055
:1016A00040F41092650C1092640C80E090E00E946F
:1016B000376280911F0D9091200D8D7F892B41F411
:1016C00040E855E260E070E08BEC9DE00E94255E12
:1016D00080911F0D9091200D019741F440E052EC54
:1016E00061E070E08BEC9DE00E94255E64E670E0B6
:1016F00080E090E00E94BE4980911F0D9091200DE6
:10170000892B09F0B7C01E3671F08091A90C909119
:10171000AA0CA091AB0CB091AC0C85369105A1053B
:10172000B1050CF0A7C067E57BE0CE0107960E94EB
:10173000976D62E677E0CE0101960E94976D6FE1AA
:1017400072E1CE0101960E94266CBC01CE01079683
:101750000E94B86CCE0101960E94CD6CBE01695FFB
:101760007F4F8BEC9DE00E94F66D68EB7BE080E0A4
:1017700090E00E94BE49BE01695F7F4FCE01019695
:101780000E948F6DCE0101960E94EE58CE01019607
:101790000E94CD6C6CE271E080E090E00E94BE4956
:1017A0004091231250912412425051096FE172E18D
:1017B000CE0101960E948C5EBE016F5F7F4FCE010D
:1017C00007960E94826BCE0101960E94CD6CBE01ED
:1017D000695F7F4FCE0101960E948F6DBE01695FE8
:1017E0007F4FCE0101960E94266CBC01CE01079668
:1017F0000E94B86CCE0101960E94CD6C65EA77E03C
:10180000CE0101960E94976DBE01695F7F4FCE01A8
:1018100001960E94266CBC01CE0107960E94B86C0E
:10182000CE0101960E94CD6CBE01695F7F4F8BECAB
:101830009DE00E94F66D68EB7BE080E090E00E9406
:10184000BE49BE01695F7F4FCE0101960E948F6D38
:10185000CE0101960E94EE58CE0101960E94CD6CF9
:101860006CE271E080E090E00E94BE49CE010796F4
:101870000E94CD6C64E670E080E090E00E94BE497A
:10188000F89482E08093B0008093B10094E6909346
:10189000B3001092B20080937000789480934B1044
:1018A00010924F1080914C1060E00E9435496DE815
:1018B0007AE0CE0101960E94876D4AE050E06FEF1A
:1018C0007FEFCE0101960E944D58CE0101960E94F5
:1018D000CD6C80911F0D9091200D892B09F569EF3A
:1018E00079E0CE0107960E94976D6FE172E1CE011B
:1018F00007960E94266CBC01CE0101960E948F6D56
:101900004AE050E06FEF7FEFCE0101960E941C5736
:10191000CE0101960E94CD6CCE0107960E94CD6C3F
:1019200080911F0D9091200D019709F565EE79E0EA
:10193000CE0107960E94976D6FE172E1CE01079686
:101940000E94266CBC01CE0101960E948F6D4AE078
:1019500050E06FEF7FEFCE0101960E941C57CE0141
:1019600001960E94CD6CCE0107960E94CD6C8091AD
:101970001F0D9091200D029709F56EE07AE0CE01DF
:1019800007960E94976D6FE172E1CE0107960E9463
:10199000266CBC01CE0101960E948F6D4AE050E09A
:1019A0006FEF7FEFCE0101960E941C57CE0101968A
:1019B0000E94CD6CCE0107960E94CD6C80911F0DC8
:1019C0009091200D019709F059C0CE010D960E940B
:1019D0006C7689899A89009709F44CC0ED85FE855B
:1019E0002081222309F446C0079708F443C06EE91A
:1019F0007AE0CE0107960E94976DBE01635F7F4F2C
:101A0000CE0107960E94266CBC01CE0101960E9471
:101A10008F6DCE0101960E949E7CCE0101960E94A0
:101A2000CD6CCE0107960E94CD6C64E87AE0CE01C1
:101A300001960E94876D48EC50E06FEF7FEFCE017A
:101A400001960E949757CE0101960E94CD6CBE016F
:101A5000635F7F4FCE0101960E948F6D48EC50E08E
:101A60006FEF7FEFCE0101960E941C57CE010196C9
:101A70000E94CD6CCE010D960E94CD6C6CE97AE08F
:101A8000CE0107960E94976D6FE172E1CE01079635
:101A90000E94266C61EB7AE00E940F6CBC01CE01C3
:101AA00001960E948F6DCE0101960E949E7CCE0110
:101AB00001960E94CD6CCE0107960E94CD6C64E623
:101AC00070E080E090E00E94BE490E94206064E6E1
:101AD00070E080E090E00E94BE4983E20E94FB5EDD
:101AE00081E090E00E94F75E0E94F55E83E090E066
:101AF00090933A0C8093390C8CE40E948F626B01B6
:101B00007C0162E370E080E090E00E94BE49A701A2
:101B10009601C701B6010E949E9B882309F449C023
:101B200086E60E948F626B017C0162E370E080E0D8
:101B300090E00E94BE49A7019601C701B6010E942C
:101B40009E9B8823B1F110923A0C1092390C88E6D2
:101B50009EE00E943E7064E670E080E090E00E94AB
:101B6000BE4940E855E260E070E088E69EE00E94F1
:101B7000255E88E69EE00E94F769892BD1F06AE62F
:101B80007AE0CE0101960E94876DCE0101960E94F7
:101B9000EE58CE0101960E94CD6C82E090E09093C9
:101BA0003A0C8093390C64E670E080E090E00E948B
:101BB000BE498091390C90913A0C039779F465E510
:101BC0007AE0CE0101960E94876DCE0101960E94B7
:101BD000EE58CE0101960E94CD6C10C00E94ED3FE0
:101BE00020E030E048E453E40E94099787FF06C0F4
:101BF00082E090E0909333048093320483E08093FA
:101C000048110E94206080ED0E940B40853509F04C
